:020000040800F2
:1000000000000120B513060839140608D93F02087C
:1000100039140608391406083914060800000000CF
:100020000000000000000000000000003914060875
:100030003914060800000000391406083159010877
:100040003914060839140608391406083914060844
:1000500039140608391406086120010865200108D2
:10006000692001086D20010871200108ADB6000863
:10007000C1B60008D5B60008E9B60008FDB600080C
:1000800011B7000825B70008391406083914060806
:1000900039140608391406083914060875200108B1
:1000A00085BF0008A9BE000899BF000895BE0008DA
:1000B000D1BE0008E5BE0008F9BE0008B1AC0008DA
:1000C000A5AC0008C9AC0008BDAC0008391406088E
:1000D0003914060861C200086DC2000879C2000820
:1000E000792001083914060839140608ADBF000844
:1000F00035BF00085DBF000821BF000839B7000800
:1001000039140608391406080DBF0008391406080A
:1001100085C20008391406083914060875D000088D
:100120004DB7000861B7000875B7000889B7000827
:100130009DB7000800000000000000000000000063
:100140000000000000000000000000000BC40008D8
:10015000B1B70008C5B70008D9B7000891C20008B8
:10016000E1AC0008D5AC00083914060839140608BB
:1001700039140608391406080000000000000000C9
:100180003914060839140608391406083914060803
:10019000391406083914060800000000391406084E
:1001A00000000000000000000000000039140608F4
:1001B0003914060839140608000000000000000089
:1001C000000000000000000000000000000000002F
:1001D00000000000000000000000000039140608C4
:0801E000000F06000100000001
:1001E800D04102200201000007002200F041022055
:1001F8000202000102003F0010420220010B000031
:100208000000760030420220010F00000000760056
:1002180050420220010C01000000770070420220C9
:100228000111000000007600904202200113000036
:1002380000001E00B04202200119000000000D005D
:10024800D04202200115000000000C00F0420220FC
:10025800011A000000000E0010430220011B0000DC
:1002680000001E00304302200116000000000C00B0
:10027800504302200117000000000E0070430220C6
:100288000118000000000C00904302200127010023
:1002980000001800B0430220011F000000004800C1
:1002A800D04302200120000000004900F043022052
:1002B8000121000000004A00104402200122000031
:1002C80000004B00304402200123000000004C00D5
:1002D800504402200124000000004D007044022018
:1002E8000125000000004E00904402200126000075
:1002F80000004F00B0440220012A0000000029003D
:10030800D0440220012B010000002900F044022003
:10031800012C01000000700010450220012D010091
:100328000000520030450220012E01000000280084
:10033800504502200228010000012C0070450220CF
:10034800022F000000024200904502200131000007
:1003580000003C00B04502200134000000002000ED
:10800000836B1A6C12F0500F21D11A6C42F400727B
:108010001A641A68916811F0405F1BD19969C9B957
:10802000D16A11F4700F02D09168490512D45168D9
:1080300021F0200151601A6C22F480721A641A6CCB
:10804000D20407D41A6C42F001021A6470479B6B89
:10805000DB6C184770477047836B40221A645A6C78
:1080600042F004025A64704790F83530022B03D076
:1080700080234365012070470268052380F835306E
:108080000020136823F00103136070470268436BFC
:108090009169126803B118477047836B19684A6881
:1080A00042F400424A600022996B0A65D96B0A6566
:1080B00093F84120602A02D1202283F841207047A2
:1080C000F0B5059D06680C4FB46931EA04040CBF95
:1080D00001240024944201D000200CE03C68641B81
:1080E0009C42F1D9202380F84130002380F84230AF
:1080F00080F840300320F0BD4022012030B50468F4
:10810000039D60682B4320F07F700B4320F45930AF
:1081100043EA024320F47F7020F0030003436360CE
:1081200030BD836B0022A3F85A20A3F85220704779
:10813000436ADA0710B506D50168846A4A6822F4F2
:10814000003222434A609C0706D50168C46A4A6827
:1081500022F4803222434A60590706D50168046B35
:108160004A6822F4802222434A601A0706D5016831
:10817000446B4A6822F4004222434A60DC0606D57A
:108180000168846B8A6822F4805222438A609906CF
:1081900006D50168C46B8A6822F4005222438A60C3
:1081A0005A0610D50168046C4A68B4F5801F22F4A1
:1081B000801242EA04024A6005D14A68446C22F403
:1081C000C00222434A601B0606D50268816C5368D0
:1081D00023F400230B43536010BD0F4B984215D07E
:1081E000A3F57843984213D003F58063984211D0E9
:1081F00003F57843984208D10323084A142101FB70
:108200000322138A01339BB2138270470023F4E7E1
:108210000123F2E70223F0E70030014000000120D3
:10822000036920221F2B70B544682DD9A3F12005C6
:108230006168AA400A4226D08069027C022A01D1E4
:108240000022027445681F2B134A2969C1F30321D8
:1082500002EB81018968565CC1684868815921F048
:108260000101815128686D79C16802EB4502128DC8
:1082700002F4F05221EA0202C2604FF0200206D955
:10828000203B9A40E26070BD21689A40D2E702FA32
:1082900003F3A360F7E700BF686F0608D0E9072380
:1082A0009A422FBFD01AC0688018C01A7047D0E910
:1082B000092300699A4238BF12180138D31AC01A2C
:1082C0007047D0E90902131A5842584170470246D4
:1082D000036A4169C85C0133D1688B4228BF00231F
:1082E00013627047436A8269D154436A0269013359
:1082F000934228BF0023426B4362136843F080031C
:1083000013607047436BD86910F0100002D0102240
:1083100001201A6270477047704701207047014B77
:108320005868704740220120034B93F80402C31E93
:1083300058425841704700BF40220120012380F875
:108340004930704708B5D0F814320BB9022008BD87
:108350001B6898470028FAD0F8E7D0F818321BB10C
:108360000020C3F81402704702207047D0F8302272
:1083700001F00F01D0F8183210B51C2404FB0122C3
:1083800003F50371B2F81022C3F80C22D0F81C22B6
:10839000D3F80402D2689047002010BDD0F81C32F8
:1083A00010B56BB1D0F8184294F80002FF2807D03E
:1083B0009B68214694F801229847FF2384F80032F5
:1083C000002010BD43230380004870475000012067
:1083D0004323038000487047940001204323038017
:1083E00000487047D80001200A23038000487047E6
:1083F0001C01012020230380004870472801012030
:108400002023038000487047480101202023038077
:1084100000487047680101200A2303800048704724
:1084200088010120042301480B807047940101203A
:10843000002370B54D1C1E46040FB0F1204F4FEACB
:10844000001034BF3034373401F8134005F813609E
:108450000133DCB2A242EFD870BD1A2310B50B80F5
:10846000094BD3F8100AD3F8182A80180AD0D3F889
:10847000144A08220549FFF7DBFF04221031204689
:10848000FFF7D6FF024810BD0070F01F9A010120CF
:108490009801012000207047212808B51CD022280F
:1084A0002CD0202816D1A9B1072A13D11A4B08794C
:1084B0000A6883F8B80148798979C3F8B42183F848
:1084C000B90183F8BA11154BD3F83C3213B11146F8
:1084D00000209847002008BD0029FBD0072AF9D1C9
:1084E0000D4BD3F8B4210A6093F8B8210A7193F8C0
:1084F000B92193F8BA314A718B71EBE70029E9D0C1
:10850000022AE7D1054BD3F84032002BE2D009888C
:1085100000209847DEE700BF000001204022012034
:10852000064AD2E99132934203F1FF338CBF002017
:1085300001209B1A03EB0030704700BF402201204E
:10854000EEE74FF4007300201380024BD3F858324B
:108550000B607047402201200020704701207047C7
:10856000012070470020704730B414461A69A242B7
:1085700009D30D199B69AA4238BF111B0A46E1189D
:1085800030BC5EF003B930BC704738B500250446F6
:1085900080F8425090F84130292B0AD1282301213C
:1085A00080F841302123036357F04EFE84F8405099
:1085B00038BD90F841302A2BFAD12823022180F8C7
:1085C000413022230363EFE7154B202210B5C3622D
:1085D000002304460363436380F8412080F842305F
:1085E0004B0711D503685A6A436A591C41621A70D5
:1085F000038D4BB1013B0385438D013B9BB243850A
:10860000436C43F0040343640721204657F01CFEEB
:1086100023681022DA61002384F8403010BD00BFC7
:108620000000FFFF0022304B10B580F842200446C6
:10863000C3624285436C1943416490F84130282B52
:1086400007D090F84130292B03D090F841302A2BE5
:1086500021D10321204657F0F7FD282384F841302B
:1086600000232363214B6363236819681A6811F49C
:1086700080411DD022F48042A06B1A601C4B036520
:10868000002384F84030FFF7EFFC58B3A06B036D74
:10869000BDE810401847072157F0D6FD94F8413047
:1086A000602B02D0202384F8413000232363DAE7D3
:1086B00012F400420DD01A68E06B22F400421A60F6
:1086C0000B4B036584F84010FFF7CEFC50B1E06B14
:1086D000DDE794F84130602B02D1202384F841304B
:1086E00084F8402010BD00BF0000FFFFF1A100088A
:1086F0009B800008036899691A6810B4CC0508D5F6
:10870000140606D5446C44F0010444644FF48074AC
:10871000DC614C0508D5140606D5446C44F0080409
:1087200044644FF48064DC61890508D5120606D5DF
:10873000426C42F0020242644FF40072DA61436C10
:1087400013F00B0F03D0416C5DF8044B6AE75DF842
:10875000044B704703682DE9F04F13F0010885B012
:1087600000F0C881AC4A916821F400019160C16AAF
:1087700094680C43B1FA81F14909946013F400261E
:1087800000F0BA81A44D426BD5F88C40B2F5801F41
:1087900024F4401444EA0204C5F88C4000F0AE8191
:1087A000B2FA82F2520913F48014019411D0DFF866
:1087B00068C2856BDCF88C40B5F5800F24F440046A
:1087C00044EA0504CCF88C4000F09B81002D08BFE2
:1087D00001229F0638D5904CDFF844C2256C45F045
:1087E00080552564246C04F080540394039C8B4CC6
:1087F000256845F480752560DCF800E02568ED0506
:1088000040F18181844C856AD4F870E005F44079A8
:108810001EF4407E40F08281B9F5407F7E4C40F0EE
:10882000A981D4F808C025F0704E2CF4F81C2EF461
:10883000407E4CEA0E0CC4F808C0C5F30B05D4F812
:1088400070C045EA0C052567DC060CD5724DD5F8DD
:108850008C4024F08074C5F88C40D5F88C40076BB0
:108860003C43C5F88C405F0409D5DFF8ACC1C46D4A
:10887000DCF8905025F440352C43CCF890401D0492
:1088800009D5DFF894C1046EDCF8905025F440253A
:108890002C43CCF89040DC0309D5DFF87CC1446E52
:1088A000DCF8905025F440152C43CCF890405F063E
:1088B00009D5DFF864C1C46BDCF8905025F00305DE
:1088C0002C43CCF890401D0609D5DFF84CC1046C50
:1088D000DCF8905025F00C052C43CCF89040DC05DA
:1088E00009D5DFF834C1446CDCF8905025F0300530
:1088F0002C43CCF890409F0509D5DFF81CC1846C4F
:10890000DCF8905025F0C0052C43CCF890405D0574
:1089100009D5DFF804C1C46CDCF8905025F440752B
:108920002C43CCF890401C0509D5DFF8ECC0046D51
:10893000DCF8905025F440652C43CCF89040DF04DF
:1089400009D5DFF8D4C0446DDCF8905025F44055CB
:108950002C43CCF890409D0409D5DFF8BCC0846D51
:10896000DCF8905025F440452C43CCF8904013F4AB
:1089700000150FD0DFF8A0E0D0F874C0DEF890400A
:10898000BCF1006F24F0006408BF012244EA0C042B
:10899000CEF890405C030AD5DFF87CE0DEF890402A
:1089A00024F0407CC46E4CEA0404CEF890401F02D0
:1089B0000AD5DFF864E0DEF8904024F0805C846F34
:1089C0004CEA0404CEF890405C0140F1D880DFF816
:1089D00048E0DEF8904024F0005CC46F4CEA0404E8
:1089E000CEF89040002940F0CF80012A40F08080EE
:1089F000094B0B491A6822F080521A600C681A68F9
:108A0000970000F178810EB1426B5AB1019A002AA9
:108A100038D0826BB2BB05E00038024000700040E5
:108A200040220120D3F888404FF4403696FAA6FE43
:108A300047F6C072BEFA8EFE92FAA2F2B2FA82F73E
:108A400096FAA6F64FF0706CB6FA86F69CFAACFC75
:108A50000269BCFA8CFC04F44034BA40476924FA39
:108A60000EF407FA0CF7B4403A432243C3F88820C7
:108A7000D3F88C20046A22F4F852013C42EA042222
:108A8000C3F88C2055B3436FB3F1006F26D1A04DCE
:108A90004FF0706CD5F888209CFAACF747F6C0739D
:108AA000B7FA87F793FAA3F34FF44034B3FA83F697
:108AB00094FAA4F4B4FA84F49CFAACFC036902F0CE
:108AC00070628069BCFA8CFCB340FA4000FA04F48E
:108AD00002FA0CF223431343C5F888308C4B1A6812
:108AE00042F080521A6008681A68920040F10981C9
:108AF000002010E0414641E6324654E600220121C2
:108B000051E6012165E6DCF80050A5EB0E05642D69
:108B10007FF674AE032005B0BDE8F08FF1453FF459
:108B20007BAED4F870E0D4F870A02EF4407E4AF406
:108B3000803AC4F870A0D4F870A02AF4803AC4F83F
:108B400070A0C4F870E0D4F870E01EF0010F3FF49C
:108B500063AEDCF800A041F2883BD4F870E01EF070
:108B6000020F7FF459AEDCF800E0AEEB0A0EDE45F2
:108B7000F3D9CFE7D4F808C02CF4F81C5BE619B998
:108B8000B3F1007F7FF431AFDFF884E1DFF884C117
:108B9000DEF8001021F08061CEF80010DCF8004013
:108BA000DEF800100F0100F19F80B8F1000F2AD00D
:108BB000C16A41BBDEF884404FF0706898FAA8F9AA
:108BC00047F6C07BB9FA89F99BFAABFBBBFA8BFB82
:108BD00098FAA8F84FF0E04AB8FA88F89AFAAAFA90
:108BE0004168BAFA8AFA04F0706401FA0BFB8168F2
:108BF00024FA09F401FA0AF104FA08F44BEA010133
:108C00002143CEF884101EB1416BB1F5801F05D011
:108C10000199B9B3816BB1F5800F33D1DFF8F0E082
:108C20004FF0E048DEF8844098FAA8F947F6C07B98
:108C3000B9FA89F99BFAABFB4FF0706ABBFA8BFB70
:108C40009AFAAAFABAFA8AFA98FAA8F8416804F0E5
:108C5000E044B8FA88F801FA0BFBC16824FA09F479
:108C600001FA0AF104FA08F44BEA01012143CEF8B3
:108C70008410DEF88C40C16924F01F0401392143BF
:108C8000CEF88C109C011ED547F6C07393FAA3F35F
:108C90004FF07061B3FA83F491FAA1F14FF0E04E16
:108CA000B1FA81F19EFAAEFE4368BEFA8EFEA34091
:108CB000C46804FA01F10B43816801FA0EF10B4319
:108CC0001349C1F88430124B196841F08061196072
:108CD000DCF80040196809013FF587AEDCF80010A8
:108CE000091B6429F6D915E7DCF80010091B642973
:108CF0007FF656AF0EE70A68121B642A7FF67FAE36
:108D000008E70A68121A642A7FF6EEAE02E700BF8F
:108D100000380240402201202DE9F347066905464C
:108D2000C3680C464FF0004901F150071E4001F1A5
:108D3000380816B902B0BDE8F087B6FA86F329FA0A
:108D400003F21B3BD24316402A61002C42D0042B75
:108D5000EFD8DFE803F03B36302903002369D5F86C
:108D60002CA033B19B6823B11FFA8AF104F10800EB
:108D70009847A36A33B19B6823B11FFA8AF104F1C3
:108D800020009847236C2BB19B681BB11FFA8AF116
:108D900040469847A36D002BCBD09B68002BC8D0D2
:108DA0001FFA8AF1384604E0236904F10800696B70
:108DB0005B689847BDE7A36A04F12000A96B5B6874
:108DC000F7E7236C4046E96B5B68F2E7A36D296C1B
:108DD0005B68E7E7042B06D8DFE803F00D0B090713
:108DE0000300EB6A0193019BA3E76B6BFAE7AB6BA4
:108DF000F8E7EB6BF6E72B6CF4E737B5224B002571
:108E0000224C234AC4F8883242F20F7304F52270D0
:108E1000C4F89852C4F894321E4BC4F89052D3F858
:108E2000BC31B3FBF2F3013BC4F88C3257F07CF950
:108E3000194B062137201A6C42F020021A641B6C71
:108E400003F020030193019B54F068FC134B4FF493
:108E5000000228465A60D4F88832DA6842F00102EB
:108E6000DA601A6842F001021A60D4F820320C4A23
:108E7000C3F81052C3F808220A4AC4E98F55C3F850
:108E8000042203B030BD00BF001400404022012086
:108E900080841E00000001200038024000E100E054
:108EA0000C6301200C53012010B501200C460BF07F
:108EB000CBFB054B122103F11402218002280CBFC9
:108EC0001846104610BD00BFC0010120436BDA698F
:108ED000910670B5044613D5586AE36AC0B2002BF8
:108EE0004AD0216B9847636B1A6822F480721A602B
:108EF0009A6822F001029A609A6942F008029A6127
:108F0000636BDA69D20701D501221A62DA69960722
:108F100001D502221A62DA69550701D504221A62C4
:108F2000DA69100701D508221A62DA6911060ED52E
:108F300094F89D20212A0AD0D4E909128A4227D127
:108F40000022A4F886201A6822F080021A60DA69EA
:108F5000520640F19380DA6904F13400196816076B
:108F60009D6821D1960640F18A808D0640F1878068
:108F7000BDE8704056F01ABFE3696269D054E369F6
:108F8000E2680133B3FBF2F102FB1133E361AAE7BC
:108F9000A169895C0132C9B299622169B2FBF1F021
:108FA00001FB1022A262D2E705F0010501F49076E0
:108FB0002E4364D0D60709D5CE0507D501261E62FB
:108FC000D4F8A06046F00106C4F8A060960708D562
:108FD0003DB102261E62D4F8A06046F00406C4F833
:108FE000A060560708D53DB104261E62D4F8A060E3
:108FF00046F00206C4F8A06016070AD501F0200664
:10900000354306D008251D62D4F8A0302B43C4F8A0
:10901000A030D4F8A030002B30D0960603D58D06B2
:1090200001D556F0C3FED4F8A020636B110703D41A
:109030009A6812F040021FD01A6822F490721A60E7
:109040009A6822F001029A60202284F89E209A6891
:10905000520613D59A68D4F8980022F040029A601C
:1090600060B1254B0365FEF7FFFF38B1D4F89800D7
:10907000BDE87040036D1847C4F8A02070BD160607
:109080002ED50D062CD594F89D20212AF6D1B4F8C2
:10909000862092B242B91A6822F080021A601A68D9
:1090A00042F040021A60E9E7E16BD4F88020B1F5A4
:1090B000805F0FD1616C69B932F8021BC1F30801FE
:1090C0009962C4F88020B4F88630013B9BB2A4F8C2
:1090D0008630D3E7511CC4F8801012789A62F2E708
:1090E0005006CBD54A06C9D51A6822F040021A604C
:1090F000202384F89D30C1E72381000870B5002645
:109100000E4CD4F8C8329BB9FEE712F8016B013B54
:109110004FF00105C4F8C822636007D156F0C5FAC4
:109120006368D4F8C8222BB1002DEED0304670BD54
:109130000025F5E7002DE3D0F8E700BF402201202D
:1091400008B5054A0B68C2F8C80253600BB956F05F
:10915000ACFA002008BD00BF4022012090F8482052
:10916000531C0244DBB280F8483082F8341090F887
:1091700049200AB1132B01D956F076BB7047002263
:1091800080F8492056F070BBF8B50446D0F830029C
:10919000237C93BB4FF400730222812156F0FAFA2C
:1091A0004FF4007302220121D4F8300256F0F2FA93
:1091B000082303228221D4F8300256F0EBFA4FF450
:1091C00007705DF0F3FC0546C4F8180230B3D4F81C
:1091D0001C3200271B689847267CC5F81472C5F816
:1091E00018728EB94FF40073D5F804220121D4F817
:1091F000300256F038FA3046F8BD40230222812171
:1092000056F0C8FA4023CDE74023D5F804220121C7
:10921000D4F830023E4656F026FAECE70126EAE79B
:1092200010B504468121D0F8300256F070FA0121C1
:10923000D4F8300256F06BFA8221D4F8300256F09E
:1092400066FAD4F8183253B1D4F81C325B689847E8
:10925000D4F818025DF0B2FC0023C4F818320020E4
:1092600010BD10B504460121D0F8300256F04FFA77
:109270008121D4F8300256F04AFAD4F828025DF081
:109280009DFC0020C4F8280210BD37B50B780446B9
:109290000D4613F060022BD0202A21D1CA884878CD
:1092A0000AB31B06D4F818120AD5D4F81C3201915F
:1092B0009B689847EA880199204656F0CAFA0FE061
:1092C000032381F8012281F80002C4F8F431134627
:1092D000D4F83002C4E942220A46002156F0C3F90C
:1092E000002003B030BDD4F81C329B689847F7E7E4
:1092F0004B780A2BF4D101220049DEE70C2501202E
:1093000070B50446D0F83002237C93BB4FF4007351
:109310000222012156F03EFA4FF40073022281210D
:10932000D4F8300256F036FA4FF41B705DF03EFC74
:109330000646C4F8280218B30025D4F82C3205815B
:10934000A0F85C5228461B6898470121D4F83002E7
:1093500056F0DFFC8121D4F8300256F0DAFCD4F864
:1093600030021F2306F50372012156F07CF92846CE
:1093700070BD40230222012156F00CFA4023CDE7B4
:109380000120F5E770B5D0F82852044695F8183258
:109390004BB9D5F8143233B16B7A23B90121D0F827
:1093A000300256F0B2FA8121D4F8300256F0ADFA0C
:1093B0006B7A022B09D105F50372D4F830021F2312
:1093C0000121BDE8704056F04EB970BD70B50E4B2E
:1093D0000446D0F82852C5F82C32002385F83812FC
:1093E00005F50B722B7281210D23D0F8300256F057
:1093F0006FF905F50372D4F830021F230121BDE88F
:10940000704056F030B900BF555342532DE9F0413A
:109410000B7804460D46D0F8287213F0600635D05C
:10942000202E7ED14A78FE2A07D0FF2A18D0D4F801
:109430003002022656F0A8FA25E04E88002EF6D11A
:10944000CD88012DF3D11A06F1D5D0F82C329B69C5
:1094500098472A4638603946204656F0FAF912E015
:109460004A88002AE3D1CE88002EE0D11B06DED444
:109470004FF4807307F5037201213B811F23D0F85D
:10948000300256F0F0F83046BDE8F08191F80180E6
:10949000B8F10A0F2AD0B8F10B0F2AD0B8F1010F9A
:1094A000F1D10979D0F8300256F033FCD4F830020B
:1094B000297956F02CF995F90430D4F83002002BB4
:1094C000237C1BDAC3B94FF400730222812156F0CA
:1094D00061F9D4F828727B7A022B17D18121D4F854
:1094E000300256F012FA00237B72CCE70122391DBC
:1094F000B3E78B787B60C6E74023E6E723B94FF4F8
:10950000007302224146E2E74023FAE795F904207E
:10951000002AB8DA012BB6D001212046FFF756FF0A
:10952000B1E70026AFE72DE9F743137806460D466D
:1095300017462F2BD0F828423CD8192B08D8032BDC
:109540005ED0122B00F08680002B3ED02022F0E16E
:109550001A3B152BFAD801A252F823F09396000873
:109560008D9600084D9500084D9500088D960008D1
:109570004D9500084D9500084D9500084D95000843
:10958000A79600084D950008F59600084D9500082F
:109590004D9500082F9700084D9500080998000880
:1095A0004D9500084D9500084D9500084D95000813
:1095B000299900085A2BC9D10823B94A6381D2F8E6
:1095C0003F30E360D2F843306BE0D4F81432002B24
:1095D000BCD1D0F82C3208469B689847054650B15C
:1095E0003A220221D6F8280254F012FA05232372F7
:1095F0004FF0FF3500E06081284603B0BDE8F083FE
:109600001222002104F10C005DF00AFB702394F893
:109610005D2223730C23E37494F85C329A4211D0D8
:1096200004EBC302013392F83C12DBB2A173042BAA
:1096300092F8411208BF0023217692F8402284F864
:109640005C326276122363813B79122B98BF63816F
:109650000025D1E75378DB0715D4D0F82C3201EB85
:10966000C1051279DB6903EB85052B79053393423C
:1096700028BF13466381002BEAD0013B9BB2E95C13
:10968000E2181173F7E70723864DF3E700206081A6
:10969000DEE70823824A6381D2F83730E360D2F8EC
:1096A0003B302361D4E700230DF1020201A9E360FE
:1096B00023616361D0F82C3228465B6898470546E1
:1096C00020B13A220221D6F82802CAE00823E37327
:1096D000019B013B1A0EE37422741A0C62741A0A7D
:1096E000BDF80230A27402225BBAA282E3820C238C
:1096F000638181E7D0F82C3204F25E22284604F51B
:1097000018715B68984705460028DAD1D4F86032B2
:109710002082013B1A0EE37322731A0C62731A0A39
:10972000B4F85E32A2735BBA63820823E0E7237A5F
:109730006BBB94F91832002BBFF608AFD0F82C326F
:1097400008469B6898470028BBD1D7F80220D6F876
:10975000280212BAD0F86012C4F86422B7F80730B1
:109760005BBA9BB29F18C4F868328F4277D8022147
:109770002172B4F85E124A434B43C4F86422D4F811
:109780001422C4F86832934201D0202268E04FF4DA
:109790000073D6F82C026381D6F82842D0F81090D6
:1097A0002846D4F8687204F10C08B4F85E229F428F
:1097B000D4F8641228BF1F46B7FBF2F3B1FBF2F2F4
:1097C0009BB24146C847002802DA112204217AE7F9
:1097D000BBB2D6F830024246812155F079FFD4F869
:1097E0006432D4F868023B44C51BC4F86432D4F830
:1097F0003432C4F86852DB1BC4F83432002D7FF4D5
:1098000027AF03232372F7E6237A002B4CD194F978
:109810001832002BFFF69AAED0F82C3208469B681F
:10982000984700287FF44DAFD6F82C322846DB68E5
:109830009847054608B1272244E7D7F80220D6F812
:10984000280212BAD0F86012C4F86422B7F80730C0
:109850005BBA9BB2D718C4F868328F4204D9212270
:10986000052154F0D5F8C3E6B4F85E124A434B43E1
:10987000C4F86422D4F81422C4F86832934284D124
:10988000B3F5007F4FF0010104F10C0228BF4FF443
:1098900000732172D6F830029BB255F0E4FEABE6BD
:1098A000686F0608986F0608D4F8687204F10C080F
:1098B000B4F85E22B7F5007FD4F86412D0F82C0219
:1098C00028BF4FF40077D0F814902846B7FBF2F386
:1098D000B1FBF2F29BB24146C847002801DA0322ED
:1098E00074E7D4F86432D4F868523B44ED1BC4F8F2
:1098F0006432D4F83432C4F86852DB1BC4F8343212
:1099000025B929463046FFF761FD75E6B5F5007FBC
:1099100042464FF00101D6F8300228BF4FF40075DF
:10992000ABB255F0A0FE93E6787810F0020003D0B9
:1099300024220521204694E7D4F86422B4F8683242
:109940001344D4F8602293427FF6A1AE2122F0E7BF
:10995000D0F8281210B50B7A0446022B07D0033B2F
:10996000012B02D80021FFF731FD002010BD01F2CC
:109970001B2291F81912FFF7D6FD0028F5DA012114
:109980002046F0E770B5D0F828420546267A1EB189
:10999000012E55D0002070BDD4F81032C4F83032FA
:1099A000D4F81432C4F83432D0F83032B3F82C3250
:1099B0001F2B0DD1D4F80C22264B9A4208D194F8D3
:1099C0001912012904D894F81A32013B0F2B0AD935
:1099D00020220521204654F01BF8022363722846FA
:1099E000FFF7D0FCD6E704F21B22FFF79CFD00280E
:1099F000237A06DA052BF2D101212846FFF7E6FC8F
:109A0000C8E7013B022BC5D961890029F5D0D5F8FB
:109A10002832D3F8142283F83862914228BF1146C5
:109A2000D3F83422521AC3F8342204221A728BB2A9
:109A300004F10C028121D5F8300255F049FEA9E766
:109A400004F21B2294F81912FFF76DFD0028A1DA29
:109A5000D2E700BF5553424308B520B9034853F03D
:109A600023FB034808BD0348F9E700BF300C070893
:109A700010250120510C0708024808B553F014FBCB
:109A8000014808BD720C070810250120024808B5DE
:109A900053F00AFB014808BD770C07081025012088
:109AA000024808B553F000FB014808BD820C0708C6
:109AB00010250120002108B5084609F0E7FE002026
:109AC00008BD2DE9F843089D0E46174600212022C7
:109AD000044698465DF0A4F84DB12B681A0CE3815A
:109AE0006B682282E3821A0C6B8922836382304680
:109AF00056F088FCFB0604D400F1FF39B9F1FF3FB2
:109B000042D1082802464FF0FF394FF00005A8BFA8
:109B100008224FF0203331462046236063605CF01A
:109B200035FE04F10803224A09F101011846228199
:109B30003144A2722A465CF029FE621E0346E01DF3
:109B400012F8011FA1F16105192D9CBF2039117078
:109B50008242F5D1184604F10B0210F8013BA3F143
:109B6000610119299CBF203B00F8013C9042F4D1CF
:109B70001823E772A4F81A8023734FEA1843A382CC
:109B8000099BE361BDE8F88316F809302E2B02D05B
:109B900009F1FF39B2E74A46A0EB0905082A05F1A9
:109BA000FF35A8BF0822032DA8BF0325B1E700BFDA
:109BB000202020002DE9F04F0D46BA4F85B001213D
:109BC000043500201646994609F060FE2C1FB9F1B5
:109BD000000F07D14846494609F058FE484605B0EF
:109BE000BDE8F08FD7F87022B24200F2B780A6EB42
:109BF0000208D7F880A24FEAD803DAF8302008F03C
:109C000007080233934203D3DAF83820934218D975
:109C100051461846039353F0B7F9039B824670B937
:109C2000A5F1080305F5FC729F4943F8041F934210
:109C3000FAD109F1FF39013605F50075C6E7C7F815
:109C400080029AF80420002A6DD04FF4007200219F
:109C500020465CF0E5FFDAF84030B8F1000F47D15C
:109C600005F11C0BCDE9008843BB43462046082282
:109C7000D7F85C12FFF725FF5C464FF4F073DAF873
:109C8000448004EB030AB8F1000FD2D05445D0D081
:109C900098F8042004F1200BD8F8001008F11C00FB
:109CA000D8F83030B2B30022CDE9000211222046AC
:109CB0005C46FFF706FFD8F84880E4E7DAF8303072
:109CC000112220467949FFF7FCFEDAF8403005F111
:109CD0003C041A6CCDE9008842B94346112274490C
:109CE0005846FFF7EEFE4FF4E073C8E71B6BF5E74D
:109CF000002B0CBF01220222C2EB0812DAF84480CA
:109D0000B8F1000F03D0013AD8F84880F8D14FF4E9
:109D10000073B6E798F805C0D8F81020CDE9000226
:109D20004CF02102C3E7DAF828B0BBF1000F06D1EE
:109D30004FF40072002120465CF072FF79E7DAF8F8
:109D400030204FF4007120469B1ADAF80C2008EB03
:109D5000C308534602EB4822D8476AE7002E64D175
:109D60004FF40072314620465CF05AFF802351497F
:109D700085F8BA310C2385F8BE31D7F86022D7F8C0
:109D800058328A42C4F8C621C4F8CA3118DDFF220D
:109D900085F8BB2185F8BD2185F8BC21013B454AEA
:109DA000934228DDFF2385F8BF3185F8C13185F85E
:109DB000C031552385F8FA31AA2385F8FB3138E7FD
:109DC0003F2143F6C16492FBF1F192FBF4F4C1EB45
:109DD000811C85F8BD41A010A2EB0C0220F03F00D1
:109DE0000132024385F8BC21FF2291FBF2F21144BB
:109DF00085F8BB11D2E73F2243F6C16093FBF2F234
:109E000093FBF0F0C2EB821485F8C10181101B1B9B
:109E100021F03F0101330B4385F8C031FF2392FB52
:109E2000F3F31A4485F8BF21C3E7D7F864329E42A2
:109E300042D152234FF0000841227221237028465C
:109E400063706123E270A37084F8E731D7F8783249
:109E500084F8E411C4F8E8314FF0FF3384F8E511D9
:109E6000414684F8E6214FF4F07284F8EC3184F82E
:109E7000ED3184F8EE3184F8EF315CF0D1FE5523FA
:109E8000C5F8EC81C5F8F081C5F8F48184F8FE319D
:109E90006FF0550384F8FC8184F8FD8184F8FF316C
:109EA000C7E600BF40220120DEADBEEF65530708C4
:109EB00064530708FF03FB00D7F860329E426BD162
:109EC0004FF40072002120465CF0AAFEEB233A4AD0
:109ED0004FF0080C05F8043C5823F82105F8033C22
:109EE000902305F8023C136845F8013C53680222B0
:109EF000C5F8033000232273E37285F809C0A2730A
:109F0000E37369743F212A7321764FF0FF31D7F84C
:109F10006002A1763E2184F82C2001222177D7F817
:109F200058126376091AE37663772162A377E377A1
:109F300084F82D3084F82E3084F82F30D7E99A0138
:109F4000091A616284F8302084F83130802385F862
:109F500042C085F83C30292385F83E30942385F8AB
:109F60003F300E2385F840300D2385F84130134BE8
:109F70001A68C5F843205A68C5F847201A899B7AA1
:109F8000A5F84B200E4A85F84D301368C5F84E30C1
:109F90005368C5F852300CE7D7E99A138E4206D3BE
:109FA0009E4207D2711A204653F012F841E69E42B3
:109FB000FFF4BEAEF11AF6E7900C0708990C0708FB
:109FC000A50C070813460A460146184635F02CBA78
:109FD00082B0054A01901068136801991B1A8B42E0
:109FE000FAD302B0704700BF40220120002808DBEE
:109FF0004209012300F01F0003FA00F0014B43F86F
:10A000002200704700E100E02DE9F04F002385B009
:10A01000DFF8B8816B4ADFF8B89101270C689F40E0
:10A0200007EA040537EA040440F0B6804C6824F0DF
:10A03000100ABAF1020F16D14FEAD30E03F0070B44
:10A040004FF00F0C00EB8E0E4FEA8B0BDEF820600A
:10A050000CFA0BFC26EA0C0C0E6906FA0BF646EA23
:10A060000C06CEF820604FEA430E4FF0030CD0F8F8
:10A0700000B00AF1FF3A0CFA0EFCBAF1010F6FEAD8
:10A080000C062BEA0C0B04F0030C01960CFA0EFCE8
:10A090004CEA0B0CC0F800C015D8D0F808C006EA8E
:10A0A0000C0CCE6806FA0EFA4AEA0C0CC0F808C08E
:10A0B000D0F804C02CEA0707C4F3001C0CFA03FC18
:10A0C0004CEA07074760C768019E37408E6806FA6A
:10A0D0000EF63E43C660E6005ED5D8F8446023F035
:10A0E000030703F0030C4FF00F0E46F4804607F110
:10A0F00080474FEA8C0CC8F8446007F59C37D8F8C5
:10A10000446006F480460396039E0EFA0CF6D7F8D8
:10A1100008A02AEA060E2C4EB04244D006F580660E
:10A12000B04242D006F58066B04240D006F5806667
:10A13000B0423ED006F58066B0423CD048453CD0A7
:10A1400006F50066B0423AD006F58066B0420CBF14
:10A150000726082606FA0CF614F4803F46EA0E0697
:10A16000BE606FEA050716680CBF3E402E4314F42C
:10A17000003F166056680CBF3E402E4314F4801F0B
:10A18000566096680CBF3E402E43A4029660D66887
:10A1900054BF3E402E43D6600133102B7FF43DAFB9
:10A1A00005B0BDE8F08F0026D4E70126D2E70226ED
:10A1B000D0E70326CEE70426CCE70526CAE7062625
:10A1C000C8E700BF003C01400000024000380240E8
:10A1D0000014024003689A69910701D500229A622F
:10A1E0009A69D20703D49A6942F001029A617047D2
:10A1F00070B590F8403004460D461646012B00F02D
:10A200001881012380F84030CB0640F19780D006BA
:10A2100040F19480638D9BB2002B40F08780E36A0D
:10A22000B3F1007F03D0E36AB3F1007F6AD194F801
:10A230004130282B66D129462046FEF7C5F9AB06EA
:10A240005CD5B6065AD52368202207212046DA615C
:10A250000822DA6155F0F8FF236820465A6842F474
:10A2600000425A605A6822F0FF7222F48B3222F4C4
:10A27000FF7222F001025A60FFF7ACFF22681368F8
:10A28000580402D41368190409D594F84130212BDD
:10A290000CBFA36BE36B1B685B689BB26385638D2C
:10A2A0009BB21BB1636C43F0040363646B0710D56E
:10A2B000636A526A591C61621A70238D4BB1013B6B
:10A2C0002385638D013B9BB26385636C43F004037C
:10A2D000636400232363636384F84230636C002B60
:10A2E00000F09A80616C2046FEF79CF994F84130AA
:10A2F000282B03D129462046FEF766F9002084F872
:10A30000400070BDE26A236812F5803F0BD094F8DC
:10A310004120292A07D110222046DA61FFF75AFF8F
:10A32000FEF733F98BE71022DA6188E72368102201
:10A33000DA61636C43F00403636480E769071DD549
:10A3400072071BD5638D9BB263B123685A6A636A37
:10A35000591C61621A70238D013B2385638D013B7B
:10A360009BB26385638D9BB2002B7FF468AFE36A79
:10A3700013F5803F3FF463AF2046D1E72B072CD580
:10A3800030072AD594F84130226803F02803282B9F
:10A3900020D1936991699368D068E068022813D14D
:10A3A000C3F3C21383EA114313F006030CD1A16C6B
:10A3B0000131A164A16C02297FF441AF0821A3649B
:10A3C000D16184F840303AE70421204655F03CFF43
:10A3D0000023F6E70823D361FAE7A9077FF52FAF3B
:10A3E000B2077FF52CAF638D9BB26BB1636A5A1CC9
:10A3F000626222681B789362638D013B9BB2638526
:10A40000238D013B23851AE7E36AB3F1807FB3D044
:10A41000E36A002BB0D012E7E36A13F5803F05D062
:10A42000054BE362202384F8413067E794F841301C
:10A43000F8E7022065E700BF0000FFFF194B9A68AC
:10A4400002F00C02042A28D0082A28D15A68596838
:10A4500002F03F02586811F4800F47F6C07191FA7C
:10A46000A1F3B3FA83F300EA010020FA03F014BF6A
:10A470000D4B0E4BB3FBF2F20A4B50434FF44032FC
:10A480005B6892FAA2F2B2FA82F203F44033D3404C
:10A4900001335B00B0FBF3F070470348704703489B
:10A4A000704700BF0038024000127A000024F40018
:10A4B000094B4FF4E0529B6892FAA2F2B2FA82F290
:10A4C00003F4E053D340054A1344054A93F8473058
:10A4D000D2F8BC01D840704700380240686F0608C7
:10A4E00000000120094B4FF460429B6892FAA2F2EF
:10A4F000B2FA82F203F46043D340054A1344054A9A
:10A5000093F84730D2F8BC01D84070470038024079
:10A51000686F06080000012038B5C2690446036868
:10A52000816800691D68014360690143A1481143C6
:10A530002840256A0143E0681960596821F44051B8
:10A5400001435960A1699868294320F430600143B0
:10A55000996099498B421FD101F59431D1F890103F
:10A5600001F003010139022900F2058193480144F9
:10A5700091F84F10B2F5004F40F0AE80082900F27C
:10A58000A880DFE811F0E600FB000101A6000D0144
:10A59000A600A600A600350089498B420AD101F524
:10A5A000FA31D1F89000854900F00C00014491F88F
:10A5B0005210DFE783498B421FD101F5F831D1F802
:10A5C000901001F03001202900F0DB800AD800292A
:10A5D00000F0BC80102900F0E080B2F5004F78D088
:10A5E0000120C7E03029F8D1B2F5004F40F0A98032
:10A5F0006268530803F58033CCE073498B4210D175
:10A6000001F5F631D1F8901001F0C001802900F079
:10A61000B88004D8002900F099804029DBE7C029E0
:10A62000E1E76A498B4213D101F5F431D1F890107A
:10A6300001F44071B1F5007F00F0A38005D8002936
:10A6400000F08480B1F5807FC5E7B1F5407FCAE7AF
:10A650005F498B4213D101F59231D1F8901001F48A
:10A660004061B1F5006F00F08C8005D8002900F042
:10A670008280B1F5806FAEE7B1F5406FB3E7554921
:10A680008B4211D101F5E031D1F8901001F4405125
:10A69000B1F5005F75D004D8002957D0B1F5805FBF
:10A6A00099E7B1F5405F9EE74B498B4295D101F5A3
:10A6B000DE31D1F8901001F44041B1F5004F60D087
:10A6C00004D8002942D0B1F5804F84E7B1F5404F5E
:10A6D00089E70120002346E0082981D801A252F829
:10A6E00021F000BF09A7000821A7000827A700083C
:10A6F000E1A500083DA70008E1A50008E1A50008C4
:10A70000E1A5000843A70008FFF7D2FED4E9002323
:10A7100000EB5300B0FBF3F080B2D060002029E0E2
:10A72000FFF7E0FEF2E761684A0802F5740202F5FD
:10A730001052B2FBF1F292B2DA60EFE7FFF77EFE61
:10A74000E4E761684A0802F50042F2E7B2F5004F1B
:10A75000DAD1FFF7ADFE63685A0802EB4000B0FBA8
:10A76000F3F39BB2002023F00F02C3F342032168EE
:10A770001343CB6038BDB2F5004FD1D1FFF7B2FE25
:10A78000E9E7B2F5004FCED16268530803F1F473E4
:10A7900003F59043B3FBF2F3E3E7B2F5004FCDD1FD
:10A7A000FFF74CFE61684A0802EB4003B3FBF1F38C
:10A7B000D7E700BFF369FFEF00100140686F06089C
:10A7C0000044004000480040004C00400050004061
:10A7D0000014014000780040007C0040A348A44AD7
:10A7E000A449121A70B5A4B05BF0D0FFA24A0020B1
:10A7F000D2F8883043F47003C2F888309F4B196850
:10A8000041F0010119609860196821F0847121F408
:10A81000803119609A495960196821F480211960C2
:10A820009849D8609160BFF34F8FBFF36F8FC2F824
:10A830005002BFF34F8FBFF36F8F516941F4003166
:10A840005161BFF34F8FBFF36F8F1A6C42F080528C
:10A850001A641A6C02F080520292029A8A4A1168B3
:10A8600041F440411160126802F440420192019AA1
:10A870009A6802F00C02042A07D09A6802F00C02CF
:10A88000082A65D15A68520262D57C4B1B687B4A04
:10A89000936803F00C03082B68D013687B4C23F0FB
:10A8A00080731360216813689D0160D447F6C073FC
:10A8B00093FAA3F3B3FA83F04FF4403393FAA3F37C
:10A8C0004FF0706191FAA1F14FF4D873B1FA81F1B0
:10A8D0008340092000FA01F10B4343F0015343F098
:10A8E00008035360136843F080731360634B21685F
:10A8F0001A68900140D51A6C42F080521A641B6CA1
:10A9000003F080530393039B5F4B1A6842F4803239
:10A910001A6021685A68D20333D51A6842F40032AB
:10A920001A60594A216853689B0330D54FF40013CD
:10A930004FF4C07C04A804934FF0006321930723D5
:10A94000CDE908C303230A93FDF704FF28B3FEE70C
:10A950001A684A4942F480321A604C4A10680B68FF
:10A960009E0394D413681B1A642BF8D9FEE723685E
:10A970005B1A022B97D9F9E72268521A022AB7D933
:10A98000F4E72268521AB2F57A7FC3D9FEE723684A
:10A990005B1AB3F57A7FC6D9F8E73D4A136803F02E
:10A9A0000F03062B08D9354B9A6822F0F0029A6003
:10A9B0001A6890010CD4FEE7136823F00F0343F0EC
:10A9C00007031360136803F00F03072BF3D1EAE7C3
:10A9D0009A6841F2883022F0030242F002029A6043
:10A9E00021689A6802F00C02082A39D1284A1368B3
:10A9F000190755D4214CA36823F4E05343F4A05322
:10AA0000A360A36823F4604343F40043A360FFF70B
:10AA100015FDA368F02292FAA2F2B2FA82F203F0D4
:10AA2000F0031C4ED3401C4D334493F85F30D840A4
:10AA3000C5F8BC0152F09EFE184B04A804930023F5
:10AA4000CDE91333CDE91533CDE91733CDE919330A
:10AA5000CDE91B33CDE91D33FDF77CFE60B3FEE786
:10AA60002268521A8242BCD9A5E700BF000000004C
:10AA7000381A0000046C070800ED00E000380240BE
:10AA80001030002400000008007000404022012027
:10AA9000003C0240686F060800000120C0FF030070
:10AAA000136823F00F0343F007031360136803F0E8
:10AAB0000F03072B9ED07EE7D4F88C3023F08073F1
:10AAC000C4F88C30D4F88C3043F08073C4F88C30E8
:10AAD000A36803F00C03042B14D0082B14D0184BDC
:10AAE000C5F8BC31174B9B68C3F303131E44D5F85C
:10AAF000BC3196F85F20D340134A9342C5F8BC316D
:10AB00001BD0FEE7114BEBE76368626813F4800F1C
:10AB1000636802F03F0218BF0C49C3F3881308BFF3
:10AB20000749B1FBF2F25343064A5268C2F30142AD
:10AB300001325200B3FBF2F3D2E724B070BD00BF84
:10AB40000024F4000038024000E6DF0C00127A0016
:10AB500003682DE9F041C3F30D04054688464D4FC7
:10AB6000002C62D14C4A93421ED302F5804293429C
:10AB700019D302F5804293421ED3484A93421DD90D
:10AB800002F5803293421BD902F50032934219D963
:10AB900002F50032934217D902F50032934215D9DB
:10ABA00005200AF0B3FF012497F8E433012B0FD1FD
:10ABB0004FF0FF30BDE8F0810224F5E70324F3E70E
:10ABC0000424F1E70524EFE70624EDE70724EBE78B
:10ABD000012387F8E43352F04BFD68BB304E3369F4
:10ABE00023F440733361336943F400733361336991
:10ABF00023F0F8033361782393FAA3F3B3FA83F3D2
:10AC000032699C40144344F002043461336943F4D4
:10AC100080333361BFF34F8F52F02AFD336923F045
:10AC20007A03336140B987F8E40397F8E433012BE2
:10AC300006D16FF00100BDE7002387F8E433B7E7E2
:10AC400001232E68D8F8008087F8E43352F010FD15
:10AC5000B0B9134C236923F440732361236943F48F
:10AC600000732361236943F001032361C6F8008068
:10AC7000BFF34F8F52F0FCFC236923F001032361E3
:10AC8000002387F8E4330028D3D12B6804332B60EA
:10AC900090E700BF4022012000400008FFFF0008AD
:10ACA000003C02400148FDF725BD00BF30260120D1
:10ACB0000148FDF7EBB900BF302601200148FDF740
:10ACC00019BD00BF802601200148FDF7DFB900BF94
:10ACD000802601200148FDF70DBD00BFD0260120D0
:10ACE0000148FDF7D3B900BFD02601202DE9F84374
:10ACF0008F4F0C26054606FB0076D6F8E831002B70
:10AD000000F0108196F8EE0152F010FC96F8EC017C
:10AD100008F086FD044696F8ED0108F081FD6B1CF5
:10AD20000646DBB21CB140F60B122372E2801EB164
:10AD300040F60B223372F28020464FF0090908F0EA
:10AD400023FD304608F020FD1121204608F027FDA4
:10AD50001121304608F023FD4FF0650803E005207F
:10AD600000210AF075FE204608F0FDFC10B9B8F18C
:10AD70000108F4D1204608F00CFD002105200AF05E
:10AD800067FE204608F000FD052000210AF060FE65
:10AD9000B9F10109E0D120464FF00C0808F0F9FCA8
:10ADA0000021052008FB05780AF052FE304608F025
:10ADB000F0FC002105200AF04BFE204608F0E4FCE0
:10ADC000002105200AF044FE304608F0DDFC204654
:10ADD00098F8F2213E2108F003FD50243046554EEC
:10ADE00098F8F2213E2108F0FBFC04FB0564D8F83A
:10ADF000E831C4F8F033FFF75BFB98F8EF31022B32
:10AE000000F09280032B00F09180012B14BF4FF4CF
:10AE1000C8714FF4487152F001FB50220021C4F870
:10AE2000F40302FB05630120C3F80014C3F8041403
:10AE3000C3F80C14C3F81014C3E9FE1093F83114CE
:10AE400001F0FF0009B983F8300402FB05622424F5
:10AE5000D2F8F03382F83144196821F00101196009
:10AE6000D2F8F41321F070611961996821F400415E
:10AE700099604FF400419960596841F0007141F4C4
:10AE800000415960D96821F40041D960D2F8081412
:10AE90000902D96000211960186840F001001860AB
:10AEA0002020C2F8341482F83104C2F8201482F849
:10AEB000321492F8310420285FFA80FC17D192F8FE
:10AEC0003004012813D082F83144186820F00100C2
:10AED0001860186820F480501860186818601868A6
:10AEE00040F00100186082F831C482F830140C245C
:10AEF000022104FB057494F9F10152F00FFC94F95E
:10AF0000F101FFF773F8022194F9F00152F006FC09
:10AF100094F9F001FFF76AF85020012300FB056562
:10AF200085F8EC33BDE8F883642174E7C82172E743
:10AF300000000120402201202DE9F04F984685B005
:10AF4000431C064689469DF83C50039200F0208140
:10AF5000AA4F502303FB007393F8ECB3BBF1000F2F
:10AF60006ED0FF2A03D0B8F1000F40F0BE80002D54
:10AF700000F0BB805024744307EB040A9AF8313484
:10AF8000202B40F0FC809AF83034012B00F0F78041
:10AF90009B4B0122D7F800B04FF400411C448AF8C3
:10AFA00030241923CDF800B02046FDF789F8002899
:10AFB00040F0E58021231FFA88F809FA02F9CAF85F
:10AFC00024048AF8313410238AF832340E9BCAF8EC
:10AFD0003404CAF81434AAF81A84BAF81A349BB2A2
:10AFE000FF2B31D94FF40053FF22AAF81824009305
:10AFF0004FF080734FF050084946204608FB067812
:10B00000FDF77CF8B8F81A34594620469BB23BBB92
:10B0100052F0E6FA38BBD8F8F0332021AB46D961BC
:10B020005A6822F0FF7222F48B3222F4FF7222F06F
:10B0300001025A6088F8311488F8300488F8320424
:10B04000584605B0BDE8F08FBAF81A244FF4005303
:10B0500092B2AAF81824D2B200934FF00073C9E755
:10B0600052F0E2FA10B1D8F8343488E0D8F8143449
:10B070005A1CC8F81424D8F8F0231B789362B8F847
:10B080001824B8F81A34013A013B92B29BB2A8F8DE
:10B090001824A8F81A34002AB4D1B8F81A349BB28C
:10B0A000002BAFD00A2380212046CDF800B0FDF759
:10B0B00007F8002863D1B8F81A349BB2FF2B0AD9DD
:10B0C000FF224FF08073A8F81824009049462046CC
:10B0D000FDF714F896E7B8F81A244FF0007392B20F
:10B0E000A8F81824D2B20090F0E7502474433D1918
:10B0F00095F83134202B42D1B8F1000F3FD095F8AC
:10B100003034012B3BD03E4B0122D7F800A04FF446
:10B1100000411C4485F830241923CDF800A02046B6
:10B12000FCF7CEFF58BB212309FA02F91FFA88F871
:10B13000C5F8240485F831344023494685F8323473
:10B140000E9BC5F834042046C5F814344FF4005360
:10B15000A5F81A8400934FF08073FCF7CFFF514697
:10B16000204652F061FA0246A8B1D5F83434502393
:10B1700003FB0673D3F83424002283F83024B7F895
:10B18000DC34304601339BB2A7F8DC34FFF7AEFD68
:10B190004FF0000B54E7D5F8F0332046039999623D
:10B1A0000A238021CDF800A0FCF78AFF0028DED119
:10B1B000B5F81A349BB2FF2B09D8B5F81A244FF012
:10B1C000007392B2A5F81824D2B2009005E0FF22D5
:10B1D0004FF08073A5F8182400904FF050084946AE
:10B1E000204608FB0675FCF789FF5146204652F0C1
:10B1F0001BFA38B108FB067835E700BF4022012072
:10B2000030260120D5F814345A1CC5F81424D5F87A
:10B21000F0231B789362B5F81824B5F81A34013A74
:10B22000013B92B29BB2A5F81824A5F81A34DAB9FA
:10B23000B5F81A349BB2BBB10A2380212046CDF861
:10B2400000A0FCF73DFF002899D1B5F81A349BB255
:10B25000FF2B16D9FF224FF08073A5F81824009019
:10B2600049462046FCF74AFFB5F81A349BB2002B3A
:10B27000BBD15146204652F0B3F960B1D5F8343411
:10B280007DE7B5F81A244FF0007392B2A5F81824A0
:10B29000D2B20090E4E7D5F8F0332021D9615A68A2
:10B2A00022F0FF7222F48B3222F4FF7222F00102AC
:10B2B0005A6085F8311485F8300485F83204BFE609
:10B2C0002DE9F04FB0F1FF3F85B0804693469DF8E1
:10B2D0003C9000F09A805024B74F44433D1995F8B4
:10B2E000ECA3BAF1000F00F0FB809BB2FF2A05F53A
:10B2F0007C744FEA4106039340F0F680B9F1000FE9
:10B3000000F0F28095F83134202B75D195F8303467
:10B31000012B71D00122D7F800A019234FF400416E
:10B3200085F830242046CDF800A0FCF7C9FE00289F
:10B3300062D12223C5F8240485F83134102385F81E
:10B3400032340E9BC5F83404C5F81434039BA5F8B9
:10B350001A34B5F81A349BB2FF2B1DD94FF4105391
:10B36000A5F818B45A4600934FF080735025314623
:10B37000204605FB0875FCF7C1FEB5F81A349BB2F0
:10B38000002B56D15146204652F02AF9002800F0F1
:10B390009280D5F834342FE0B5F81A244FF41053C6
:10B3A00092B2A5F81824D2B200934FF00073DDE7F3
:10B3B0005146204652F0DCF8C8B9D5F8F0339A6906
:10B3C00012F0200224D02021D9615A6822F0FF72A5
:10B3D00022F48B3222F4FF7222F001025A60C5F887
:10B3E000340485F8300485F8311485F8320450238C
:10B3F00003FB0873D3F83434B7F8DC344046013328
:10B400009BB2A7F8DC34FFF771FC4FF0000A67E04D
:10B410003B68A3EB0A030A2B0BD9D5F8343485F823
:10B42000302443F02003C5F83434202385F8313428
:10B43000DDE7D5F8F0339A695207B9D55A6AD5F8DD
:10B440001434591CC5F814141A70B5F81824B5F83A
:10B450001A34013A013B92B29BB2A5F81824A5F820
:10B460001A34002A89D1B5F81A349BB2002B84D043
:10B470000A2380212046CDF800A0FCF721FE0028F9
:10B48000BAD1B5F81A349BB2FF2B0AD9FF224FF07C
:10B490008073A5F81824009031462046FCF72EFE54
:10B4A0006BE7B5F81A244FF0007392B2A5F8182490
:10B4B000D2B20090F0E7D5F8F0332021CA46D96126
:10B4C0005A6822F0FF7222F48B3222F4FF7222F0CB
:10B4D00001025A6085F8311485F8300485F8320489
:10B4E000504605B0BDE8F08F502505FB087595F86E
:10B4F0003134202B80D10E9B002B3FF47DAF95F88B
:10B500003034012B3FF478AF0122D7F80090192393
:10B510004FF4004185F830242046CDF80090FCF728
:10B52000CFFD00287FF468AF2223C5F824043146FC
:10B5300085F831344FF0400385F832340E9BC5F85E
:10B540003404C5F81434039BA5F81A344FF400539F
:10B55000009303462046FCF7D1FD4946204652F0B1
:10B5600063F8024650B1D5F83434502303FB087316
:10B57000D3F83424002283F830243DE7D5F8F033A3
:10B5800040212046C3F828B00A23CDF80090FCF7EC
:10B5900097FD0028E9D1B5F81A349BB2FF2B0DD8DE
:10B5A000B5F81A244FF4105392B2A5F81824D2B269
:10B5B00000934FF0007309E0402201204FF4105334
:10B5C000FF22A5F8182400934FF0807350253146D0
:10B5D000204605FB0875FCF791FD0A230022042193
:10B5E0002046CDF80090FCF76BFD00287FF404AFF7
:10B5F000D5F8F033596AD5F81434581CC5F814043A
:10B600001970B5F81834B5F81A14013B01399BB21A
:10B6100089B2A5F81834A5F81A14E3B9B5F81A34A4
:10B620009BB2C3B10A2380212046CDF80090FCF7DD
:10B6300047FD00287FF4E0AEB5F81A349BB2FF2B2B
:10B640002AD9FF224FF08073A5F8182400903146C4
:10B650002046FCF753FDB5F81A349BB2002BBCD141
:10B660004946204651F0BCFF00287FF492AED5F841
:10B67000F0332021D9615A6822F0FF7222F48B3214
:10B6800022F4FF7222F001025A6085F8311485F825
:10B69000300485F8320423E7B5F81A244FF000731C
:10B6A00092B2A5F81824D2B20090D0E70348D0F89F
:10B6B000183213B100F503701847704700000120DD
:10B6C0000348D0F8383213B100F50B7018477047B3
:10B6D000000001200348D0F8583213B100F5137070
:10B6E00018477047000001200348D0F8783213B1A2
:10B6F00000F51B7018477047000001200348D0F880
:10B70000983213B100F523701847704700000120EC
:10B710000348D0F8B83213B100F52B7018477047C2
:10B72000000001200348D0F8D83213B100F533707F
:10B7300018477047000001200348D0F8F83213B1D1
:10B7400000F53B7018477047000001200348D0F80F
:10B75000183313B100F543701847704700000120FB
:10B760000348D0F8383313B100F54B7018477047D1
:10B77000000001200348D0F8583313B100F553708E
:10B7800018477047000001200348D0F8783313B100
:10B7900000F55B7018477047000001200348D0F89F
:10B7A000983313B100F5637018477047000001200B
:10B7B0000348D0F8B83313B100F56B7018477047E1
:10B7C000000001200348D0F8D83313B100F573709E
:10B7D00018477047000001200348D0F8F83313B130
:10B7E00000F57B70184770470000012038B54468A9
:10B7F00044F4805444603BB9012004E0013C05D18D
:10B80000FCF7EBFC002038BD40F2E9348568AD0759
:10B81000F4D56AB112F8014B047340F2E93485683B
:10B82000ED0707D5C46809B101F8014B013BE2E718
:10B83000FF24F1E7013CF2D1E2E70023054A52F888
:10B840003310814201D1D8B2704701330E2BF6D1AB
:10B85000FE207047D86F06082DE9F04707460068BC
:10B86000FFF7EBFF0D28054608DD0024274A0021DD
:10B87000052004F067F92046BDE8F087DFF89890CE
:10B880004FEA800809EB800ADAF8E0645EBB072122
:10B89000682004F025FA0446CAF8E00428B90146F5
:10B8A0001B4A052004F04EF9E5E7314668225BF0BB
:10B8B000B7F918482AB2DAF8E04400F1700300EB57
:10B8C000C500A46003EBC203006F24622360A4637D
:10B8D0002465FFF7B2FF0D289EBF09F5A36600B2ED
:10B8E00006EB80166660C844787918210023D8F8E2
:10B8F000E04401FB0042D760C2E9043300FB0112BF
:10B90000A35401FB00440834B5E700BFAE0C0708A0
:10B91000D30C0708686F06084022012070B5002884
:10B9200029D04C6854B9036842685B685679022292
:10B930001D68B240EB6823EA0203EB608A6832B903
:10B9400003685B681D68EB6823F00103EB608160AE
:10B950004CB103685B6819684368CC685D79022361
:10B96000AB402343CB6032B103685B681A68D3688D
:10B9700043F00103D36070BD0A4B30B51A46002472
:10B980001D79854208D1DD68294203D0142000FBCF
:10B99000042030BD0029F9D0013414330B2CEFD131
:10B9A0000020F6E70C040120036807EE902A70B52A
:10B9B000D3E900340E461D682368AB4279D03D4B75
:10B9C000F8EE677A2560013E93ED6F7AB6B2B8EE75
:10B9D000477A87EE270ADFED387A30EE270A58F0EB
:10B9E00001F800230138E660A36060602046C4E9E6
:10B9F00004338023A36154F097FB304B9D4216D053
:10BA0000B5F1804F13D0A3F57C439D420FD003F5D1
:10BA100080639D420BD003F580639D4207D003F500
:10BA200078439D4203D003F570539D4241D194F871
:10BA30003C30012B3DD00223214A84F83D3023685D
:10BA400099680A409A609A6822F4803222F00702CC
:10BA50009A60012284F83D20002284F83C20174A95
:10BA6000954212D0B5F1804F0FD0A2F57C4295429D
:10BA70000BD002F58062954207D002F580629542B4
:10BA800003D002F57842954213D10C485A6883429C
:10BA9000996803D000F58060834201D122F47002DE
:10BAA00022F0700221F080015A609960002384F82E
:10BAB0003C3070BD000001200AD7233C000001404B
:10BAC0008800FEFF43680068F0B540685C799A79A9
:10BAD000974B12F00202234490F83C400EBF1546EB
:10BAE00002220825012C93F8E03017D001240C2BFA
:10BAF00080F83C404FF0020480F83D4000F0C680E2
:10BB00000DD8042B65D0082B00F09080002B32D08C
:10BB1000012380F83D30002380F83C30F0BD102B2D
:10BB200000F0DB80142BF3D103681C6A24F480142A
:10BB30001C621D6A5E6825F400155C6D45EA0252C0
:10BB400024F080747B4D24F4E044AB4244F4C044C0
:10BB500003D005F58065AB4201D146F480265E60D6
:10BB60005C65D9651A625A6D42F400625A655A6D75
:10BB700022F48062D7E003681C6A24F001041C628E
:10BB80001C6A5F6824F002049E69224326F4803612
:10BB9000684C26F07306A34246F0600603D004F515
:10BBA0008064A34206D122F0080247F440772A437A
:10BBB00022F004025F609E6159631A629A6942F042
:10BBC00008029A619A6922F004029A619A699A615C
:10BBD0009EE703681C6A24F010041C621C6A5F68FC
:10BBE00024F020049E6944EA021226F08076514C2B
:10BBF00026F4E646A34246F4C04603D004F580642A
:10BC0000A34207D122F0800247F4406742EA0512BE
:10BC100022F040025F609E6199631A629A6942F461
:10BC200000629A619A6922F48062CEE703681C6A16
:10BC300024F480741C621C6A5F6824F40074DE695A
:10BC400044EA022226F480363A4C26F07306A342D8
:10BC500046F0600603D004F58064A34207D122F4C5
:10BC6000006247F4405742EA052222F480625F6096
:10BC7000DE61D9631A62DA6942F00802DA61DA69D0
:10BC800022F00402DA61DA69DA6141E703681C6ACA
:10BC900024F480541C621D6A5E6825F40055DC693A
:10BCA00045EA023224F08074224D24F4E644AB428B
:10BCB00044F4C04403D005F58065AB4201D146F49D
:10BCC00080465E60DC6119641A62DA6942F40062DF
:10BCD000DA61DA6922F48062D4E703681C6A24F42A
:10BCE00080341C621D6A5E6825F400355C6D45EA8F
:10BCF000024224F480340F4D24F07004AB4244F02F
:10BD0000600403D005F58065AB4201D146F480366E
:10BD10005E605C6599651A625A6D42F008025A6568
:10BD20005A6D22F004025A655A6D5A65F0E600BF5A
:10BD3000686F06080000014043685A79032A0FD84B
:10BD4000DFE802F00205080B186834307047186805
:10BD50003830704718683C3070471868403070477A
:10BD600000207047D0E9003251795868054B0B44E8
:10BD700093F8E01093795B0701D554F04AB854F07A
:10BD80005CB800BF686F060842681269F8B5C2F374
:10BD90000322264B044603EB82029668C26855686C
:10BDA000EFF31187102282F312884068D0F800C0A8
:10BDB0004079DCF80C2003EB4000008D00F4F050DB
:10BDC00022EA0002985DCCF80C202A5822F00102E9
:10BDD0002A50E2681069D2F804C020221F2821D915
:10BDE00020388240CCF80C20FAB282F31188985D9A
:10BDF0006769284443681B0C1B040B4343602046BF
:10BE0000FFF79AFF0A4B9B5DEA18D7609060EA58EB
:10BE100042F01002EA50EA5842F00102EA500123CF
:10BE20002374F8BD8240CCF80820DDE7686F06086F
:10BE3000686F06080268137E012B26D10223137651
:10BE40004FF4007392F83010012904D1022143F419
:10BE5000806382F8301092F84810012904D1022141
:10BE600043F4006382F8481092F8601001290ED163
:10BE7000022143F4805382F8601012680021126896
:10BE80005162D1680B43D36003E00023DAE7002B53
:10BE9000F3D17047024B0348D3F8E014FCF73CBFE2
:10BEA000402201200000014010B5064C0648D4F89D
:10BEB000E014FCF731FFD4F804150448BDE8104045
:10BEC000FCF72ABF4022012000000140004401404D
:10BED000034B4FF08040D3F8E414FCF71DBF00BFC4
:10BEE00040220120024B0348D3F8E814FCF714BFAA
:10BEF0004022012000040040024B0348D3F8EC1418
:10BF0000FCF70ABF4022012000080040024B034812
:10BF1000D3F8F014FCF700BF40220120000C0040D1
:10BF2000024B0348D3F8FC14FCF7F6BE4022012074
:10BF30000004014010B5064C0648D4F8FC14FCF788
:10BF4000EBFED4F810150448BDE81040FCF7E4BE41
:10BF50004022012000040140001C004010B5064CA6
:10BF60000648D4F8FC14FCF7D7FED4F8141504489E
:10BF7000BDE81040FCF7D0BE402201200004014083
:10BF800000200040024B0348D3F80015FCF7C4BE64
:10BF90004022012000400140024B0348D3F808151D
:10BFA000FCF7BABE4022012000480140024B034882
:10BFB000D3F80C15FCF7B0BE402201200018004059
:10BFC000704710B501208EB008F03EFB012809D162
:10BFD000002108F03FFB614B1A6882F308885B6818
:10BFE0009847FEE75E4A00245E4BD1685E4821F424
:10BFF000E0610904090C0B43D3605C4B596F196B6A
:10C0000041F480211963196B01F480210D910D9980
:10C01000196B41F480111963196B01F480110C91B3
:10C020000C99196B41F480011963196B01F48001BB
:10C030000B910B99196B41F000511963196B01F0C9
:10C0400000510A910A99196B41F080411963196BEB
:10C0500001F0804109910999196C41F4003119648A
:10C06000196C01F4003108910899196C41F4802190
:10C070001964196C01F4802107910799196C41F436
:10C0800000211964196C01F4002106910699196CBC
:10C0900041F480111964196C01F48011059105991E
:10C0A000196C41F080411964196C01F080410491D0
:10C0B0000499196C41F000411964196C01F00041B8
:10C0C00003910399596C41F010015964596C01F0C6
:10C0D000100102910299596C41F020015964596C88
:10C0E00001F0200101910199596C41F400615964FA
:10C0F0005B6C1F4903F400630093009B1D4BD3F856
:10C10000BC31B3FBF1F1C0F89818D2F8FC101A4812
:10C1100041F08071C2F8FC101849C1F8B00F4C60B2
:10C12000086840F0010008604FF47A71B3FBF1F346
:10C13000013BB3F1807F08D24FF0E0214B61F02347
:10C1400082F8233007238C610B614FF0E0221369E2
:10C1500043F0040313610EB010BD00BF0000F01FD8
:10C1600000ED00E00003FA05402201200038024003
:10C1700040420F000000012055CEACC5001000E089
:10C18000074B03EB8000D0F8E43033B193F8AD20D7
:10C190004A7093F8AC300B7070474B70FBE700BFF0
:10C1A000686F06082DE9F04117462C4A9846054667
:10C1B00002EB8003D3F8E44084B304F1AE0302F54C
:10C1C000827294F8AD00261DA36104F5D7736260F6
:10C1D000E3614FF48073E160C4E904332368C4F879
:10C1E000A830A36307F01CFB18F0080F19D0013525
:10C1F000EDB218B140F20673C380057294F8B6220E
:10C20000022107F0EDFA94F9B702D4F8B81251F010
:10C2100085FA94F9B7023446FDF7E8FE2046BDE8FA
:10C22000F081BA0794F8AC800BD56B1CDBB218B167
:10C2300040F206520372C28094F8B622022107F03F
:10C24000CFFAFB07DFD50135404607F0E9FAEDB23A
:10C250000028D3D040F20663CEE700BF686F06081F
:10C260000148FCF733BE00BFEC0401200148FCF795
:10C270002DBE00BFA80701200148FCF727BE00BF64
:10C28000640A01200148FCF721BE00BF200D0120F7
:10C290000148FCF71BBE00BFDC0F0120426B2423CA
:10C2A000816870B580F89D300446136800F134054C
:10C2B00023F00103136000231360536093608163D4
:10C2C0008179C0F8A03080F89C3080F89D3080F8EB
:10C2D0009E308802A36400F48050E3646365E063E9
:10C2E0000803637900F4005013F0010620644FEA5C
:10C2F000012000F4806060641CBF0420A06413F07F
:10C3000002031EBFA06C40F00800A064C8070FD550
:10C3100036B1A06D40F00200A0654FF48030206679
:10C3200033B1A36D43F00103A3654FF40033E3651C
:10C33000242311F0080F94F89D10284684F89D30AE
:10C34000136823F00103136036D0FEF7E5F80128E7
:10C3500018D0A36D13B12846FBF7EAFE636B5A6849
:10C3600022F490425A609A6822F022029A609A68F7
:10C3700042F008029A6028461A6842F001021A60E8
:10C3800053F0E6FC6179CA070DD5D4F8A4301A68D9
:10C3900042F480721A609A6842F001029A601A6848
:10C3A00042F020021A608B0705D5D4F8A420136848
:10C3B00043F08003136070BDFEF7AEF80128E1D0B2
:10C3C000A36D13B12846FBF7B3FE636B5A6822F4E2
:10C3D00090425A609A6822F02A02CBE781605DE7BA
:10C3E00041715BE710B51C2007F01AFA04461121D1
:10C3F00007F0D5F9204607F0CCF9C82009F039FB41
:10C400002046BDE8104007F0BFB9934B2DE9F04F2F
:10C41000D3F89C5887B06B6913F00103029340F086
:10C42000A9816A69AB691A4200F0A4816B69AA69A3
:10C4300013409C0701D502236B616B69AA69134005
:10C44000180300F19A81844CD4F89C385A69996990
:10C450000A40510311D5D3F8182803F5006304F6F8
:10C460009C0705F5106ADB694FF0000913409BB289
:10C470000193019B002B40F02A84D4F89C08426968
:10C4800083691A4216D5D5F8043823F00103C5F89C
:10C49000043894F8883C012B15BFD4F8983C00234D
:10C4A00093F8FD2184F8883C18BF83F8FC214FF0F5
:10C4B000004343614369826913401B050FD5D5F8DA
:10C4C0000838DF0708D5D4F8983C93F8FC2183F8A6
:10C4D000FD21042283F8FC214FF40063436143698A
:10C4E000826913401E010FD54FF00063436194F839
:10C4F000883C002B40F0FB84012384F8883C436D8A
:10C50000C3F38303C4F88C3C436982691340D904A4
:10C510003AD5D5F80438102105F5006623F001035B
:10C52000736053F03BFAD4F8A00805F510630022BD
:10C53000FF21824240F0E6844FF0FF33B361F3699C
:10C5400043F00113F361D4F8CC38002B00F0E18400
:10C55000D6F8843043F00B03C6F88430736C43F094
:10C560000B037364D5F800383C4A23F4FE6394F857
:10C57000AC18D4F89C08C5F8003853F0A7F9D4F8E3
:10C580009C384FF480525A61D4F89C385A699969A2
:10C590000A40920472D5D3F8002922F4FF6222F0F7
:10C5A0000702C3F8002903F50062916801F0060153
:10C5B000042905D1D3F8001941F00301C3F800198B
:10C5C000516841F480715160D96821F47051D9608B
:10C5D000916811F0060F11D0916801F0060102294F
:10C5E00000F0A184916801F00601062900F09B8407
:10C5F000926802F00602042A00F095844FF400725B
:10C600000027C4F8B028DA68C4F8A87842F41052B9
:10C61000DA60D4F8986C00224FF0400840231146AD
:10C62000D6F8300253F0B6F8434600228021D6F8FF
:10C630003002C6F8108153F0ADF80123C6F820800F
:10C6400086F8FC31D6F8183253B9D6F820323BB907
:10C65000D6F8283253B103E040220120982E012061
:10C66000D6F81432304631795B689847D4F8983C54
:10C670004FF400521F74D4F89C385A61D4F89C28A7
:10C68000536991690B40DB062FD5936923F01003A2
:10C6900093612B6AC3F3434003F00F07022840F075
:10C6A000AF8447F6F0710B421BD01C20C3F30A1372
:10C6B00005F5805500FB0740DE1CD0F8A0CAB61077
:10C6C00002998E4240F094841C2101FB0741D1F86D
:10C6D000A05AD1F8AC0A1D441844C1F8A05AC1F8B8
:10C6E000AC0A936943F01003936153699269134054
:10C6F0001F070ED5D4F8980C90F8FC31032B04D109
:10C70000D0F81432DB6903B19847D4F89C3808227A
:10C710005A61D4F89C28536991690B40DE0202D516
:10C720004FF480135361536991690B409D0202D508
:10C730004FF400135361536991690B40580002D5BF
:10C740004FF080435361536991690B40590711D5EC
:10C7500055686B0709D5D4F8980C012380F8FC3193
:10C76000D0F8143201795B689847D4F89C385A683D
:10C7700015435D6007B0BDE8F08FD5F8183805F5B2
:10C780003067D5F81C284FF0000ADFF85C831340AF
:10C79000A8F69C061B0C0193019B002B3FF453AEA3
:10C7A000019BDA0740F14D81D6F89C385FFA8AF197
:10C7B00003F5306203F5006302EB411292685B6996
:10C7C00002EA030919F0010F39D00123BB60D6F842
:10C7D000AC38012B0CD13B69D8F80022C3F312030B
:10C7E000D31AC8F81032D8F804321344C8F8043207
:10C7F000D6F8984C00297AD1D4F8F431032B10D113
:10C80000D4E94303984264D9C01AD6F8A02A8342D7
:10C81000C4F80C0128BF0346D4F830029BB252F092
:10C8200022FFD6F8AC18012909D1D6F8A83A5AEA5D
:10C83000030304D1AB4AD6F89C0853F047F819F02B
:10C84000080F00F0F480D6F8984C96F8580C04F5D0
:10C85000027B84F8080296F859EC84F809E296F80D
:10C860005B1C96F85A3C03EB01239BB2A4F80A32F6
:10C8700096F85D2C96F85CCC0CEB022C1FFA8CFC25
:10C88000A4F80CC296F85F1C96F85E2C02EB01220D
:10C89000012192B2C4E97D1200F01F01A4F80E221A
:10C8A000012900F04881022900F05A81002940F056
:10C8B0000B82BEF1090F00F2D480DFE81EF01701F1
:10C8C0003201D2002701D2008A002400D2000301E5
:10C8D000CD00D4F814321B692BB194F8FC21032A43
:10C8E00001D120469847204652F0AAFF99E7D4F894
:10C8F00014329B69002B94D094F8FC21032A90D128
:10C90000204698478DE71A0A013A062A00F2A980C4
:10C91000DFE802F0041D2AA7A74A5400D4F8103219
:10C920001B680DF11601207C9847BDF81620002ADF
:10C930007BD0B4F80E32002B77D09A42014628BF44
:10C940001A46ADF81620204652F083FF6DE0227C97
:10C95000D4F8143232B99B6A0DF1160098470223BD
:10C960004370E2E7DB6AF7E7DBB2052B79D8DFE853
:10C9700003F003070B0F1317D4F810325B68D0E7EE
:10C98000D4F810329B68CCE7D4F81032DB68C8E7E3
:10C99000D4F810321B69C4E7D4F810325B69C0E7E1
:10C9A000D4F810329B69BCE7237C002B59D1D4F812
:10C9B00014320DF116005B6B9847B6E7237C002B11
:10C9C0004FD1D4F814320DF116001B6B9847072392
:10C9D000C6E75CEA0202D4F8300203D194F8FC11F5
:10C9E000032902D152F0D0FF1FE003F07F0B84F83F
:10C9F000FEB190F8B833012B0ED00368D3F80018BD
:10CA000021F4FE61C3F80018D3F8001841EA0B11B5
:10CA1000C3F8001880F8B823204652F011FFBBF18C
:10CA2000000F17D0022384F8FC310823BB6019F0F3
:10CA3000100F01D01023BB6019F0200F01D020236C
:10CA4000BB60019B0AF1010A203708F11C085B0852
:10CA50000193A1E60123E6E7D9B2012986F89C1CDF
:10CA600002D9D4F83002BDE794F8FC31022B0FD084
:10CA7000032BF6D1C9B902232046616084F8FC314A
:10CA8000D4F814325A689047204652F0D9FECCE7C9
:10CA90000029F9D001210323616084F8FC3120468C
:10CAA000FBF750FC0228EFD1DBE761680129EBD0EE
:10CAB000D4F81432C9B220465B68984796F89C1C9B
:10CAC0006160ECE7012ACCD194F8FC31022B03D051
:10CAD000032BC6D1211D36E72146002341F8083F2C
:10CAE00031E700BF982E0120DC2A012094F8FC31A8
:10CAF000023B012BB5D80123E360D4F804320BB11B
:10CB00000323E360022204F10C011CE7012B8CD10A
:10CB1000C4F80432D4F81432594620469B6898472A
:10CB2000B2E794F8FC21023A012A9AD8012B7FF44B
:10CB30007CAF0023ECE794F8FC31032B91D15FFA32
:10CB40008CFCBCF1030F8CD8D4F814325946204623
:10CB50009B689847B4F80E32002B7FF466AF93E7DA
:10CB600000F060005FFA8CF1202806D1D4F814326E
:10CB7000594620469B68984757E7BEF1010F46D0BB
:10CB8000BEF1030F33D0BEF1000F7FF44EAF94F827
:10CB9000FC31022B00F09080032B7FF462AF4FFA40
:10CBA0008CFC01F07F0210234FF0040EBCF1000F4B
:10CBB000B4BF501C02F11000BCF1000F4FF01C0C70
:10CBC00013FB00E3D4F83002A8BF0CFB010123449F
:10CBD000B4BF0CFB020291F8FA211946B8BF92F8D3
:10CBE0003A20003A18BF01221A600222ABE694F8FC
:10CBF000FC21022A60D0032A7FF433AF002B89D1B5
:10CC00004B0687D0D4F8300252F07FFE82E794F8CA
:10CC1000FC21022A50D0032A7FF423AF002B7FF49B
:10CC200004AF11F07F003FF42FAF4FFA8CFCD4F823
:10CC300030221C23BCF1000F4FEADC7CB4BF03FBA5
:10CC4000002103FB01214FF00003B4BF383101F58F
:10CC5000FC718B70087081F801C092F8B833012B19
:10CC60003FF458AF01234FF0200E82F8B833136819
:10CC7000BCF1000F14D0C87803F5106309780238AE
:10CC80001EFB01330128196821F40011196003D833
:10CC9000196841F080511960002382F8B83339E7F0
:10CCA00003F530631EFB0033186820F40010186091
:10CCB000C97802390129EAE748063FF4B6AED4F84C
:10CCC000300252F022FEB0E600F08001F7E7019B4F
:10CCD000DA0740F1A980D4F89C285FFA89FBD2F8E2
:10CCE000101802F5106252F8CC3C02EB4B1223FAFA
:10CCF0000BF892684FEAC8185FFA88F848EA01080A
:10CD000008EA020818F0010F4AD00121D5F834389A
:10CD100001FA09F123EA0103C5F834380123CAF8FE
:10CD20000830D4F8AC38012B02BFD7E910239B1888
:10CD30007B6419F0FF01D4F8986C40F0A780D6F816
:10CD4000F431022B17D1D6E90730834276D91C2261
:10CD50001B1AD6F8300202FB0B420391D2F8E028EE
:10CD6000F3619BB252F0B4FC03990B460A46D6F825
:10CD7000300252F078FC96F80032012B02D10023E9
:10CD800086F80032D4F8AC18012909D1D4F8E83873
:10CD900059EA030304D1A64AD4F89C0852F096FD40
:10CDA00018F0080F02D00823CAF8083018F0100F46
:10CDB00002D01023CAF8083018F0400F02D04023E8
:10CDC000CAF8083018F0020F02D00223CAF808305F
:10CDD00018F0800F28D0D4F89C08D7E9133200F55A
:10CDE000106600F580519B1A3A6C06EB4918934285
:10CDF00001EB0B3BA8BF1346DA1C48BF9A1D9210EB
:10CE0000D8F8181089B2914203D9D7E913218A4280
:10CE10004AD8002B08DC0122D0F8343802FA09F293
:10CE200023EA0203C0F83438019B09F101091C37D9
:10CE30000AF1200A5B080193FFF71BBBB269B2FB42
:10CE4000F0F300FB132393B9904210D8D6F8F811F1
:10CE50008A420CD21A461946D6F83002039352F091
:10CE600037FC039BC6F8F8311A4619467FE7D6F817
:10CE70001432DB682BB196F8FC21032A01D130462D
:10CE800098470523C6F8F4310023EDE7D6F81432AD
:10CE90005B69002B3FF476AF96F8FC21032A7FF400
:10CEA00071AF304698476DE7521A3B6C94F8AC1856
:10CEB0009342A8BF1346DA1C48BF9A1D921031B1A5
:10CEC000796C19447964396D1944396598E71FFA0A
:10CED00083FCD7F844E00CF1030C4FEAAC0C8C4512
:10CEE000EED05EF821600131CBF80060F7E7D4F8AE
:10CEF000983C93F8FC2183F8FD21042283F8FC215F
:10CF0000FFF702BB99600132C3F808122033FFF724
:10CF100010BB736943F02B037361336943F00B0358
:10CF20003361FFF71FBB032242494348C4F8A828D6
:10CF30004022C4F8B028414AD2F8BC2111448142B1
:10CF400006D8DA6842F470520127DA60FFF761BB55
:10CF50003B493C481144814203D8DA6842F46052AC
:10CF6000F2E7A2F574013848A1F51051814203D8C7
:10CF7000DA6842F45052E7E7A2F183713348A1F531
:10CF8000E741814203D2DA6842F44052DCE730499B
:10CF900030481144814203D8DA6842F43052D3E772
:10CFA0002D492E481144814203D2DA6842F42052BE
:10CFB000CAE72B492B481144814203D2DA6842F474
:10CFC0001052C1E7A2F1B7712748A1F5585181422B
:10CFD00003D2DA6842F40052B6E724491144244AE5
:10CFE0009142DA6834BF42F4E05242F4C052ABE7F7
:10CFF000029928684CF8210001310291FFF760BBCB
:10D0000006287FF46EAB05F58055C3F30A13296833
:10D01000C4F8581C2968C4F85C1C1C2101FB07419A
:10D02000D1F8AC0A0344C1F8AC3AFFF75ABB00BFD1
:10D03000982E0120405327FFFF340C0000000120F0
:10D04000401E1BFF3F420F007F4F120020D61300EF
:10D0500060B6E5FE5FE3160000D3CEFE40771B000E
:10D06000C05BB3FEC091210020753800E05459FE2A
:10D07000E09C410070B5484CD4F888321A69910799
:10D0800009D5DA68920706D56FF002021A619A692B
:10D09000002284F8A4221A69560709D5DA685507D0
:10D0A00006D56FF004021A619A69002284F8A4225E
:10D0B0001A69100709D5DA68110706D56FF008025A
:10D0C0001A61DA69002284F8A4221A69D20609D505
:10D0D000DA68D60606D56FF010021A61DA69002206
:10D0E00084F8A4221A69D5072ED5DA68D0072BD583
:10D0F0006FF001021A61294A934225D1D4E99125A2
:10D10000AA4221D0264B8CBFC2F58055AD1A1A44D5
:10D11000D4F82032A9B2D3F81462C3F80822C3F8B5
:10D1200010128EB90121D4F83802C3F81412ABB230
:10D13000812152F0CDFAD4F844321D44B5F5805F18
:10D1400018BF2E46C4F84462D4F888321A69110612
:10D1500005D5DA68120602D56FF080021A611A69E5
:10D16000D60505D5DA68150602D56FF080021A617A
:10D170001A69540605D5DA68500602D56FF04002E8
:10D180001A611A69910605D5DA68920602D56FF020
:10D1900020021A6170BD00BF40220120001400402F
:10D1A0000C6301202DE9F041114E0D46D6F82022E6
:10D1B000D2F81432002BFBD104464719DFF8348033
:10D1C000BC4202D12846BDE8F081D6F8483214F8B6
:10D1D000012B08F803200133C3F30B03C6F84832D0
:10D1E000FBF79EF90028EBD1012008F042FCF7E79D
:10D1F000402201200C630120F8B50D461446FBF7D0
:10D2000093F878B1084ED6F8A07C002C0ADD2146B0
:10D210002846FFF7C7FFD6F8A03C241A0544DB1BBD
:10D22000322BF2D9F8BD00BF4022012070472DE912
:10D23000F04F4FF00008DFF834932DED028B8FB0E4
:10D24000444632F031F9474632F008F94546064681
:10D25000BE4200F3A380642C40F04B816825DFF8C8
:10D26000E4824C22B44B0021D8F84C71554305346C
:10D27000C3F89C7108EB0503184659F0D1FC4C2209
:10D28000002159F0CDFCAD4A48F805200122476243
:10D290008260AB4AC0E904668262C0E90777A64BA8
:10D2A000A84DD3F89C717300B3F1805F18DA4C225B
:10D2B0000021C6F1006654432B19184659F0B0FC02
:10D2C0004C22002159F0ACFC9F4A2A5102224762AD
:10D2D0004271012296408260C0E90466C0E9077786
:10D2E0004FF498729949974859F050FA954A042199
:10D2F000134601395F62C3E9077703F14C03F8D1A4
:10D30000AE68002E45D12B79002B42D02B68002B24
:10D310003FD00C468B488C462964E963C5E911115E
:10D32000C76C00F14C03002F40F0228102231068EB
:10D33000002840F04D8186489C1E864B3E22C0F856
:10D340008462C0F85C323F23C0E998234023C0E9DF
:10D350009D41C0F86832A100A30F002C00F0658148
:10D3600040F2FF128A1843F10003520A42EAC35204
:10D3700002F14003C0F86C321344C0F8703203EB82
:10D38000C403DA0DC0F858325B02C0E99F55C0E90A
:10D3900094320FB0BDEC028BBDE8F08F202206A9BD
:10D3A000384632F041F812226B4906A859F03CFD8C
:10D3B0000090002840F08B80AF421DD067490C20C0
:10D3C000621CCA4600FB041465490192A7EB050BD9
:10D3D000204602F0A1FB01214AF84C4B019AC9E911
:10D3E000021557491446C9F82810D9F81C10C9E984
:10D3F00004BBC9E90811D1464F4B3D46D3F89C21E7
:10D40000C9F81C2012220EAB501C1A44554B12F8BE
:10D41000201C18F8032091425CD108F10108B8F1F2
:10D42000150F59D1202206A92844002531F0FCFF10
:10D4300005AA4D4906A859F088FB05AAAA46AB469D
:10D4400008EE102A0195CDE9025538B30BF1FF32F1
:10D45000042A04D8DFE802F00F13171B1F0003F0A3
:10D460004FF8824618EE102A3F4900200BF1010BBD
:10D4700059F06BFBE9E703F043F80190F2E703F0A2
:10D480003FF80290EEE703F03BF80390EAE703F081
:10D4900037F80546E6E703F033F80090BAF1000FDD
:10D4A00012D0AAF2BC7ADDE9012343EA4210039BC1
:10D4B00040EA4A2A680140EAC320009B40EA630030
:10D4C00040EA0A40C9F81C00642C2ED03D4607F5FE
:10D4D0000067BDE64FF00008202808D12035AE4295
:10D4E000F2DB024606A9284631F09EFF00200246E4
:10D4F00089E7AF4219D0A7EB0508184A0C2718494D
:10D5000007FB042701343846224602F005FB0122BE
:10D51000C9F80070C9E90225094AC9F82820D9F8D4
:10D520001C20C9E90488C9E90822251D002C7FF4C4
:10D5300096AE0424B3E600BFF8100120290D0708B9
:10D54000C59F000894330120360D07089C7006081B
:10D5500040220120430D0708ED0C0708E42E0120AE
:10D56000000D07080E0D0708240D0708C43401201C
:10D570009F6804F1FF3EC3F840C07745C3F83CC044
:10D58000C3E911CC05D1002C3FF403AF53F80C0CC8
:10D590003C4604F1010E774508D10479002C3FF494
:10D5A000F8AE4364186474461846B9E6A7427FF49F
:10D5B000F0AE002F3FF4EDAED0F840E0DEF83C4096
:10D5C0000134CEF83C40C3F840E0BE468364EAE74D
:10D5D000107903F1FF3CA0B11363D36B5B0116BF5D
:10D5E00003F6FF7301231B0B6344C2E90477C2E90E
:10D5F0000D33D2E90D0301364C32181A01330144C0
:10D6000095E61469136364B104F6FF74240B644453
:10D610005069546338B100F6FF70000B60449063AA
:10D62000E7E70124F3E70120F8E70122A0E600BFC5
:10D630002DE9F74FCDE900124F4AD38911681B023B
:10D640005689178AC91A93896EEB0E0EA3FB010443
:10D6500003FB0E44C009138940EA44601B04E41133
:10D66000C018A6FB013506FB0E554FEA1323D688DA
:10D6700044F1000443EA0563F6032D129B19A7FB4E
:10D68000012607FB0E664FEAD25245F1000542EA39
:10D690004622F61512F5FA6C46F1000BBCF5FA6F4E
:10D6A0007BF100074CDAA2FB02784FF0050A02FB7F
:10D6B00006F908EB4909A7FB0A780AFB09884FEA33
:10D6C0005709BF0849EAC87947EA8877B0EB0900EB
:10D6D00064EB6804DB1B294F65EBA805BC454FF0E4
:10D6E000FF377BEB070720DA40F6AC57D21946F13B
:10D6F00000065643A2FB027202EB4606FA004FEA0E
:10D70000C608BA1A48EA577866EB0808101844EBBE
:10D7100008044FF00B08A7FB087208FB06267F08D9
:10D7200047EAC677DB1B65EB660501FB0EFEA1FB36
:10D73000011202EB4E0EC90F41EA4E01BCEB010C87
:10D74000009A8AB10C4A5169A1FB032301FB0535FC
:10D75000520D009B42EAC5226D15121A65EB0404B6
:10D76000D20B42EA44421A60019B0BB1C3F800C0DD
:10D77000012003B0BDE8F08F1073012024FAFFFFF1
:10D7800031B10A4BD3ED0C7AFDEEE77AC1ED007AA8
:10D7900052B1064B9FED067AD3ED0D7A67EE877A8C
:10D7A000FDEEE77AC2ED007A012070471073012088
:10D7B0000000C842007970470079C0F340107047FC
:10D7C00000794009704700BF704700BF704700BF35
:10D7D0009FED047AC7EE007A77EEA07A80EEA70A72
:10D7E000704700BF72C7D13D002380ED020A03607D
:10D7F0004360704703685A1C02601970704700BF8D
:10D8000003690133012B03611CD0D0ED005A07EEF0
:10D81000903AD0ED026A30EE656AF8EEE77A86EE6D
:10D82000277A77EE257A30EE670AC0ED017AC0EDEF
:10D83000007AF0EE667AE6EE007AC0ED037AC0ED8B
:10D84000027A7047002380ED010A80ED000A8360B0
:10D85000704703685A1C02601970704790F83020B6
:10D86000034602F0FF0012B1002283F83020704717
:10D870004FF40063838170474FF4006383817047E6
:10D88000064A002352F8041B814204D00133042BC2
:10D89000F8D1002070470120704700BF4873012075
:10D8A00001207047012070472DE9F8435F4F15466E
:10D8B0000E46BC6CB7F84C20B7F85290C2EB24135C
:10D8C0005200C2EBE402B7F94E40624303FB03F49B
:10D8D000B7F9503024135C43B7F95630A4134FEA1C
:10D8E000E37804EBE224A4F5FA317C6681FB01CEF7
:10D8F00003FB0EF20CFB0822A3FB0C389044B7F993
:10D9000054201B0A82FB010243EA0863120342EA25
:10D91000105200031B184FF0000042EB2822A3FB1B
:10D92000093802F5004209FB02884FEAE8734FEA22
:10D93000680253EA68086CD0B7F95C904FEAE9785E
:10D9400009FB0EFE0CFB08EEA9FB0C9CE644B7F9A4
:10D950005AC08CFB01814FEA414C4FEA48414CEAE6
:10D96000D83C11EB0909B96E4EEB0C0CC1F5801EC9
:10D9700010EB0900B7F958100EF000480CEBC1018C
:10D9800048EA5E084FEACE7EBEEB000068EB010C71
:10D9900040F63548A0FB080108FB0C1153F024FBAE
:10D9A000B7F962304FEA613E80464FEA503C03FBD4
:10D9B0000EF24FEAE3794CEAC14C0CFB0929A3FBB8
:10D9C0000C324A4403FB0EFE0CFB02EEB7F960205A
:10D9D000A3FB0C3C4FEAE279E6445B0E43EACE132C
:10D9E00013EB000C02FB01F3A2FB082841EB6E6E67
:10D9F00009FB0031D00CB7F95E30414440EA4130B8
:10DA00001CEB00004EEBE141000A40EA016000EB34
:10DA100003100EB1000A306025B104EB8404803499
:10DA200024122C600120BDE8F88300BF1073012090
:10DA300001207047084B1868084B10B5DC6E001BBE
:10DA4000FA2807D809B1186F08600AB15B6F136034
:10DA5000012000E0002010BDE02E01201073012005
:10DA6000034B00220120C3E91E22C3E92022704794
:10DA700010730120094B1A68094BD3F88410521A0D
:10DA8000FA2A9FBF9A6FC286DA6FD3F880309DBFA3
:10DA90000287438701200020704700BFE02E01204D
:10DAA0001073012012B10B0E00F8013B0B0C8170BA
:10DAB00003700B0A437070470048704798120120AA
:10DAC0002DE9F0410C4D0127DFF830802C686B699F
:10DAD0001C400CB9BDE8F081B4FA84F3C3F11F0314
:10DAE00007FA03F608EB8303D3F8880024EA060458
:10DAF000036898476E61ECE7003C01401073012019
:10DB000008B5006851F04BFC014B1860012008BDBE
:10DB10001073012008B5006851F041FC014B5861B9
:10DB2000012008BD1073012038B514460D460029A8
:10DB300043D0344B9FED346AD3ED327AB3F9E02011
:10DB4000F8EEE77AC7EE866A07EE902AB3F9DC2092
:10DB500007EE102AB3F9DE20F8EEE77AB8EEC77ABE
:10DB6000A6EEA77AD3ED357AF8EEE77AE6EE877A75
:10DB700093ED347AB8EEC70AA6EEA70A07EE902A0C
:10DB8000B3F9DA20F8EEE77A07EE102AB3F9D820D5
:10DB9000B8EEC77AA6EEA77A07EE902AF8EEE77AF3
:10DBA000E6EE877A93ED397AB8EEC77AC7EE066A61
:10DBB000A6EEA70A55F016FF28600CB3114BDFED57
:10DBC000126AD3ED397AB3F9CC20F8EEE77AB3F9DB
:10DBD000CE3007EE102A87EEA60A07EE903AF8EE4E
:10DBE000E77AB8EEC77AF6EE006A60EE277A9FED24
:10DBF000070AE7EE267A27EE800A55F0F3FE20604A
:10DC0000012038BD107301200000F04A0000C84216
:10DC10002DE9F04F04463C2200218BB0654858F0B6
:10DC2000FFFF621E6449033412F8013F581E0328A7
:10DC300088BF0023944241F8043BF5D10120FFF74F
:10DC40001FFE40B15D4B322283F8F42093F824216B
:10DC5000013283F824210220FFF712FE40B1574B16
:10DC6000312283F8002193F82421013283F8242102
:10DC70000320FFF705FE40B1504B302283F80C2102
:10DC800093F82421013283F824210420FFF7F8FDC2
:10DC900040B14A4B142283F8182193F82421013211
:10DCA00083F82421434C4FF00F084FF00009444EF5
:10DCB000444F207B38B394F90D5005F0B1FD28B1E5
:10DCC000052380F80780837100230372032105F088
:10DCD00066FD227B002316F83310914265D106EBD6
:10DCE000C3035B682361C02303FB0575D5F8CC3003
:10DCF0005A1C23750723C5F8CC20A375012399442A
:10DD0000637585F8C83008F101080C345FFA88F8AB
:10DD1000B8F1130FCDD1B9F1000F43D02A4B002534
:10DD20002A4C2B4E049394F8B830002B33D06079F2
:10DD30004FF0FCFB20794FF0F9FB0122D4F8BC1026
:10DD40004FF440331F4FC020914263614FF00003F6
:10DD5000A2622264D8BF4FF0000CA361C8BF4FF08D
:10DD6000010CE361636200FB05720191E162C4F89A
:10DD700020C0C4E90E33C4E90C3323682361116E5B
:10DD800001B9516600FB0570016E11F0100121D040
:10DD9000002384F84C30049B0135C034C833032D74
:10DDA0000493C0D10BB0BDE8F08F0133102B92D19A
:10DDB000002397E7F87301204873012010730120B6
:10DDC000DC7C06089812012038740120A81201207A
:10DDD00000230140026E4FF4005822F4885222F0D2
:10DDE000020242F002020266726822F4403272605D
:10DDF000726842F4403272605A6822F480725A604B
:10DE00005A6842EA0C225A605A6822F040725A60FC
:10DE10005A685A609A6822F400629A609A689A6016
:10DE20009A6822F070629A609A689A609A6822F002
:10DE300040529A609A689A609A6822F002029A6048
:10DE40009A6842F002029A605A6822F400625A60AC
:10DE5000DA6A22F47002DA62019AD3F82CE002F155
:10DE6000FF3C4EEA0C524FF4806EDA629A6822F45C
:10DE700000729A609A6842F400729A609A6822F47A
:10DE800080629A609A689A604166026E22F003028C
:10DE900042F0010202664FF40062D4F80CC084F82C
:10DEA0004C106166C4F88810C4E91AE24FF480721D
:10DEB000DFF898E3C4E91C824FF40032C4E91E2164
:10DEC0000322C4E92021A268C4E917C1A265DEF8D3
:10DED000008084F88C10022180F89D10116821F0D8
:10DEE000010111601168C90700F130811168182023
:10DEF00022F47F7EDFF8589321F0FF512EF0030EBD
:10DF000021F4772121F47C6141EA0C0C4CF40B31B3
:10DF100041F480711160516921F007015161D1B262
:10DF20001039B1FBF0FCC0485F294FF03F0160445D
:10DF300088BF0EF1040E90F88000C4F8B0E0814074
:10DF4000C4F8B40004F15800CEF808100591C021BF
:10DF500001FB05770021C7F8BC10012187F89D104F
:10DF6000A06404F110000391C4F8900068B2079017
:10DF700099F8150000285CD099F90D00079FB84268
:10DF800057D101F1010C94F84CA0D9F810005FFAB8
:10DF90008CF7BAF1010F99F8168006974FF0000739
:10DFA00008973FF4F8AE4FF00107092884F84C7049
:10DFB00087B2029740F2E28007EB470C4FF0070B65
:10DFC000D3F80CA0ACF11E0C984F0BFA0CFBB84226
:10DFD0002AEA0B0AC3F80CA040F0C980D3F80CC0A1
:10DFE0004CEA086CC3F80CC0062901EB810C00F266
:10DFF000DA80ACF1050C4FF01F08596B08FA0CF8E9
:10E00000029F21EA080107FA0CFC5963596B4CEA9C
:10E010000101596386498B4206D1122840F01A81CA
:10E02000716841F4800171604FF0000184F84C1078
:10E030000699039809F10C0901300528039097D13E
:10E040000021099194F84C1001293FF4A4AE01215C
:10E0500084F84C109968CF0740F1CB809968C807C5
:10E060007FF599AE734FC02000FB0570016E21F45F
:10E07000E06121F0010141F48071016659684905B0
:10E0800005D5016E21F4405141F480510166C02153
:10E0900001FB0571086E10F4805002D0486E20F02C
:10E0A000060048660021644884F84C10C4F89400C7
:10E0B0006248C4F898006248C4F8A4006FF02200D7
:10E0C0001860586840F080605860986840F480702C
:10E0D0009860012084F88C00C02000FB057797F839
:10E0E0009D00012840F09880022087F89D00C7F825
:10E0F000BC101168019821F480211160142148435B
:10E1000003F14C01506091600499D1600599CEF8FB
:10E110000810116841F016011160516941F0800149
:10E120005161116841F008011160116841F001016D
:10E1300011607268D20672D19A6812F0405F7FF463
:10E140002AAE9A6842F080429A6024E6DEF8001017
:10E15000A1EB080105297FF6C5AEC02303FB0577B7
:10E160002023C7F8BC30032387F89D3013E6D3F88B
:10E170000CA008FA0CFC4CEA0A0C33E700EB400B4D
:10E180004FF0070AD3F810C00AFA0BFA08FA0BF896
:10E190002CEA0A0CC3F810C0D3F810C048EA0C08E7
:10E1A000C3F8108020E70C294FF01F0110D8ACF104
:10E1B000230CD3F83080029F01FA0CF107FA0CFC13
:10E1C00028EA01011963196B4CEA0101196321E77F
:10E1D000ACF1410CD3F82C80029F01FA0CF107FA44
:10E1E0000CFC28EA0101D962D96A4CEA0101D96222
:10E1F00010E79968134841F00101996012490968D4
:10E20000B1FBF0F101EB41010991099900293FF4BB
:10E2100025AF09990139F7E784F88C1089E7044A9A
:10E2200093427FF4B8AD87E7DC7C0608120000104B
:10E23000002001409812012001800008578000084A
:10E240005980000840420F00BC01012040220120FB
:10E25000F87301200E49884202D011287FF4E4AE01
:10E26000716841F400017160094988427FF4DCAEB5
:10E27000084909480968B1FBF0F10A2041430891B7
:10E28000089900293FF4D0AE08990139F7E700BF9B
:10E2900012000010BC01012040420F00024BD3F8D5
:10E2A000800307F077BA00BF1073012007B58DF81F
:10E2B0000700012305480DF107020021D0F884036F
:10E2C00051F038F803B05DF804FB00BF1073012073
:10E2D00013B50C4C94F8880368B10523D4F8840373
:10E2E0006A4601A9ADF80030022351F023F89DF8E9
:10E2F000050000F0010084F8880380F0010002B0FE
:10E3000010BD00BF1073012038B558B9094BD3F8C0
:10E310008C43094DFFF7DCFF40B1064B0022C3F8E8
:10E320008C2306E0044B1C680444F2E72B689C42F3
:10E33000F0D838BD10730120E02E012010B5002068
:10E34000FFF7E2FF80B10620084CFFF7AFFF012383
:10E35000C72084F88833FFF7A9FF054B1B6803F536
:10E36000A4430833C4F88C3310BD00BF10730120E0
:10E37000E02E012073B5154CD8230025014694F8F2
:10E3800090630DF10100009332468DF80450FFF7C1
:10E3900089FB2846FFF7B8FFB0B10620FFF786FFDC
:10E3A0000123AE426A4684F88833294614BF052308
:10E3B0000423D4F8840350F0BDFF054B1B6803F51C
:10E3C0009C530833C4F88C3302B070BD1073012025
:10E3D000E02E0120F0B5194E0027154689B096F8B9
:10E3E0009023022304468DF80470BA4200930297EA
:10E3F00014BF05230423CDF80CD0CDE90615014642
:10E400000DF10100CDE90437FFF74CFB3846FFF76B
:10E410007BFF80B106202C44FFF748FF012302A9AF
:10E42000D6F8840386F8883350F05AFF044B1B68F3
:10E430000633C6F88C33204609B0F0BD10730120B6
:10E44000E02E012070B5144E0025144688B096F8D1
:10E45000902303238DF80450AA420093029514BF21
:10E4600005230423CDF80CD0CDE9043101460DF18C
:10E470000100CDE90654FFF715FB2846FFF744FFDE
:10E4800038B102A9D6F8840350F02AFF204608B01C
:10E4900070BD0446FAE700BF107301204A0901234A
:10E4A00001F01F0103FA01F150F822300B4340F84C
:10E4B000223070474A09012301F01F0103FA01F1DC
:10E4C00050F82230194214BF01200020704780EA22
:10E4D0000120082341F2210210F4004F4FEA4000CE
:10E4E00018BF5040013B80B2F6D1704738B50C469A
:10E4F0008D18AC4200D138BD14F8011BFFF7E7FFBF
:10E50000F7E74840082310F0800F4FEA400018BF9B
:10E5100080F0D500013BC0B2F5D1704710B50A4478
:10E520000C46944200D110BD14F8011BFFF7E9FF1F
:10E53000F7E738B50A46044605680020AA4203D327
:10E540006B1C2360287038BD12F8011BFFF7D9FF40
:10E55000F4E700BF82B08DED010A019802B0704768
:10E56000C31783EA400070479FED087A0023C0ED8F
:10E57000020AC7EE007A036030EEA77AC0ED017A96
:10E58000C0EE877AC0ED037A704700BF83F9223E60
:10E5900080ED010A704700BFD0ED016AD0ED007A2E
:10E5A00070EEA66AC0ED020A30EE677A80EEA66AC7
:10E5B000E6EE077AB0EE670AC0ED007A704700BF5A
:10E5C00080ED000A704700BF9FED047AC7EE007A25
:10E5D00077EEA07A80EEA70A704700BF4E2DA63DC9
:10E5E000002380ED030A036043608360704700BF2F
:10E5F00080ED030A704700BFF5EEC00AF1EE10FA95
:10E6000006DCF0EE407A80ED000AB0EE670A704753
:10E6100060EE810A90ED007A77EE607AF4EEC07ACF
:10E62000F1EE10FA03DC77EE200AC0FEC07AB0EEFD
:10E63000670AC0ED007A7047B4EEE00AF1EE10FA16
:10E6400002D480FE410A7047B0EE600A704700BFF6
:10E65000874BB3FBF2F399420DD300234FF07E5268
:10E66000436083600260C360036100238361436190
:10E670000362C361704707EE902ADFED7E6AB8EE51
:10E68000677A07EE901AF8EE677A27EE267A27EE79
:10E69000277AFDEEC77A17EE903A2033402B00F22E
:10E6A000D880DFED757AB4EEE77AF0EE477AF1EED6
:10E6B00010FA0CDDDFED715A9FED716AF0EE676ABA
:10E6C00077EEE57AF4EEC66AF1EE10FAF6DCDFEDED
:10E6D0006D6AF4EEE67AF1EE10FA0CD5DFED675ACA
:10E6E0009FED696AF0EE676A77EEA57AF4EEC66A86
:10E6F000F1EE10FAF6D4DFED656AF4EEE67AF1EEAB
:10E7000010FA00F39C80DFED626AF4EEE67AF1EE37
:10E7100010FA03D5DFED5B6A76EEE77A27EEA76A9B
:10E720009FED5C4ADFED5C4AF7EE006A9FED5B5AB5
:10E73000E6EE044ADFED5A5A67EE863A9FED594AF3
:10E74000A6EE245AE6EE055AE3EEA57AF0EE665AF6
:10E75000E7EEC46AE7EE845AC6EEA53ADFED4B6AEF
:10E7600077EE267ABDEEE76A16EE103A2033402B9C
:10E7700068D8B4EEE67AF1EE10FA0CDD9FED3F6A50
:10E78000DFED3F6AB0EE677A77EEC67AB4EEE67AEE
:10E79000F1EE10FAF6DC9FED3B7AF4EEC77AF1EE7B
:10E7A00010FA0CD59FED356ADFED376AB0EE677A67
:10E7B00077EE867AB4EEE67AF1EE10FAF6D49FEDB3
:10E7C000337AF4EEC77AF1EE10FA47DD9FED2A7A3C
:10E7D00077EE677A67EEA76A9FED2E7A9FED2E4A55
:10E7E000B7EE006ADFED2D4AB8EE003AA6EE874A92
:10E7F0009FED2B5A67EEA62AB6EE007AE6EE844A23
:10E80000A6EEA45AE2EE857A36EE676A67EE837A60
:10E8100026EE077AB7EE005AC0ED043AC5EE256A37
:10E8200026EE877A26EE866A66EEA77A80ED007A73
:10E8300080ED016A80ED027AC0ED037A15E7DFED25
:10E840000E6A69E7B6EE007ADFED177AB7EE006A76
:10E85000E0E7F7EE003AF0EE635A7FE79FED0C7ABF
:10E86000F4EEC77AF1EE10FAB4D59FED067AAFE771
:10E8700020A1070027D4D236DB0F4940DB0FC94067
:10E88000E4CB1641DB0F49C0E4CB16C1DB0FC93F17
:10E89000DB0FC9BF9A7C2E36FAAF4FB93587083CDB
:10E8A000A4AA2ABEF304353F00000000FDEEC07AA2
:10E8B00017EE903A2033402B51D8DFED2A7AB4EE90
:10E8C000E70AF1EE10FA0CDDDFED276A9FED277AFB
:10E8D000F0EE407A30EE660AF4EEC77AF1EE10FA06
:10E8E000F6DCDFED237AB4EEE70AF1EE10FA0CD590
:10E8F000DFED1D6A9FED1F7AF0EE407A30EE260ABA
:10E90000F4EEC77AF1EE10FAF6D4DFED1B7AB4EE2E
:10E91000E70AF1EE10FA18DDDFED127A37EEC00AE1
:10E9200060EE007ADFED155A9FED156ADFED156A8E
:10E93000A7EEA56A9FED147A60EE275AE7EE866A85
:10E94000A7EEA67AA5EE870A7047DFED107AB4EE3F
:10E95000E70AF1EE10FAE3D5DFED057ADEE79FED89
:10E960000C0A7047DB0F4940DB0FC940E4CB16416E
:10E97000DB0F49C0E4CB16C1DB0FC93F9A7C2E36B2
:10E98000FAAF4FB93587083CA4AA2ABEDB0FC9BF2E
:10E99000000000009FED2F7A70EE077AFDEEE76A27
:10E9A00016EE903A2033402B51D8B4EEC70AF1EE60
:10E9B00010FA0CDD9FED286ADFED286AB0EE677A69
:10E9C00077EEC67AB4EEE67AF1EE10FAF6DC9FED59
:10E9D000247AF4EEC77AF1EE10FA0CD59FED1E6A98
:10E9E000DFED206AB0EE677A77EE867AB4EEE67AEB
:10E9F000F1EE10FAF6D49FED177AF4EEC77AF1EE45
:10EA000010FA1ADD9FED187A77EE677A27EEA77A6B
:10EA10009FED165ADFED165A9FED166AE7EE055A7E
:10EA2000DFED156A27EE875AA7EE256AE7EE066A3C
:10EA3000E5EE267AB0EE670A70479FED107AF4EEA5
:10EA4000C77AF1EE10FAE1D59FED057ADCE79FED8C
:10EA50000C0A7047DB0FC93FDB0FC940E4CB1641FE
:10EA6000DB0F49C0E4CB16C1DB0F49409A7C2E3640
:10EA7000FAAF4FB93587083CA4AA2ABEDB0FC9BF3D
:10EA800000000000B5EE400AF1EE10FA25D007EEC6
:10EA9000902AF0EE406AF8EE670ADFED107A08B5CA
:10EAA000034660EEA70A08464BB9FFF75DFDFCEE92
:10EAB000E66A16EE903A99B2BDE80840C8E5022B26
:10EAC00006D0032BF3D1FFF77FFDBDE8084087E5B3
:10EAD000FEF77EFEFEF788FEE9E77047BD37863514
:10EAE000B5EE400AF1EE10FA02D1044B0B6070470C
:10EAF00003280CBF024B034BF8E700BFC9D700083F
:10EB000065000000F1000000D0ED0E7AF0EE405AF2
:10EB1000B0EE605AF5EEC07AF0EE414AF1EE10FA2E
:10EB200008B503467DDC30EE604AD3ED013A1A7831
:10EB300064EE233A002A5DD101F00102D3ED117A8F
:10EB4000002A60D074EE677AB0EE445AD3ED0F0A13
:10EB500087EEA40A83ED115AF5EEC00AF1EE10FA21
:10EB600054DCD3ED036A60EE266A93ED057A93EDEB
:10EB7000106A25EE877A77EE067A77EEA37A77EE3B
:10EB8000A67AF4EEE71AF1EE10FA54DC82FE670A78
:10EB900070EE677A93ED045AD3ED025A480783ED7D
:10EBA000157AB0EE467A67EE857AC3ED133A83EDB7
:10EBB000126AC3ED146AE4EE257A83ED160AA4EE18
:10EBC000A77A08D5F0EEC77AF0EEC66AF4EEE67AD8
:10EBD000F1EE10FA32D583ED107A0A0700D408BDA1
:10EBE000F4EEC71AF1EE10FA01DCC2FE471AC3EDCB
:10EBF000101A08BD11F001024FF0000045FE047A22
:10EC00001870002A9ED177EEC57A9FE793ED035ADC
:10EC1000B0EE641A03F1280058F082F965EE006A3C
:10EC2000A3E730EE600A1830F0EE670A58F078F982
:10EC3000B0EE404A79E7B0EE610AA9E7B0EE467A55
:10EC4000CBE700BF00230122C36402708364036525
:10EC5000036443644365836283657047DFED1D7A17
:10EC600080ED010AF4EE670AC0ED020A80ED031A96
:10EC7000C0ED051AF1EE10FA20DDB4EE670AF1EEF0
:10EC800010FA1BDD81EE007AC0EE207AF0EE006A09
:10EC900077EE877A86EEA77A80ED047A0023012248
:10ECA00080ED0F2AC0ED0E2A0270C36483640365F1
:10ECB000036443644365836283657047DFED057ACF
:10ECC0000023F4EEE70A0361F1EE10FAD8BF836087
:10ECD000E4E700BFBD378635B0EEC07AF0EEE06AFB
:10ECE00086FE876AB5EE406AF1EE10FA3DD0C6FEA8
:10ECF000C75AC5EE867ADFED1E2ADFED1E3ADFED3C
:10ED00001E4A9FED1E5A9FED1E3AB7EE006A9FED18
:10ED10001D4ADFED1D5AE7EEE23AA7EE834AE7EE21
:10ED2000A34AA7EE846AA7EEA45AE7EE855AC5EE79
:10ED3000867AF4EEC76AF1EE10FAF5EEC00A44BF27
:10ED40009FED127A77EE677AF1EE10FAB5EEC00A0F
:10ED500044BF9FED0F7A77EE677AF1EE10FA48BF65
:10ED6000F1EE677AB0EE670A7047DFED077AE0E709
:10ED700039094E3DE3B59E3E88FA163E45FE7F3F7B
:10ED800099FB243F69A2163EA7DFA834DB0FC93FD9
:10ED9000DB0F4940B7EE007AF0EEC07AF4EEC77AA6
:10EDA00077EE676AF1EE10FA1DD89FED105AB1EEBA
:10EDB000E67ADFED0F5A9FED0F6ADFED0F6AE7EE9F
:10EDC000855AA7EEA56AE7EE866A67EE266AB5EE73
:10EDD000C00AF1EE10FA44BF9FED087A77EE666A3A
:10EDE000B0EE660A7047DFED066AF0E7306E99BC58
:10EDF0002716983D843459BEA40DC93FDB0F494006
:10EE000000000000B0FBF1F301FB130308463BB127
:10EE10001946B0FBF1F301FB13030846002BF7D1B1
:10EE2000704700BF44F25063984203DD054B034432
:10EE300018467047044B984202DA48F6A043F6E7BA
:10EE40000346F5E76073FFFFB0B9FFFF48F69F4345
:10EE5000984203DD054B034418467047002802DA48
:10EE600048F6A043F7E70346F6E700BF6073FFFFED
:10EE700080EAE073A3EBE0738B4203DB002803DD41
:10EE8000401A704700207047FDD00844704700BF0B
:10EE9000884203DB9042A8BF10467047084670477F
:10EEA00000230361704770B503780446012B32D10B
:10EEB00003691F4D1BB942680AB92A684260D4ED44
:10EEC000067A013304F11C0677EE807A236130461E
:10EED000C4ED067AFEF794FC62682B689B1AA26860
:10EEE000934218D9E06A94ED0A0A50F089FBD4EDF8
:10EEF000057AB4EEE70AF1EE10FA0DDD237B43B993
:10EF00002A683046236100236260A361BDE8704037
:10EF1000C6E70323237070BDD4ED047A0223D4ED39
:10EF2000066AF8EE677A86EEA77A84ED067AF1E74C
:10EF3000E02E01202DE9F04104461C30254604F165
:10EF40006402064650ED017AB1EC010A77EE807A50
:10EF500040ED017AFEF754FC18309042F2D123695B
:10EF6000274F0133626823613B689B1AA268934272
:10EF700044D904F13008E86A95ED0A0A50F040FBE4
:10EF8000A845D4ED057A1AD0B4EEE70A1835F1EEAB
:10EF900010FAF0DD237B7BBB3A6830462361626068
:10EFA0000022A261FFF77CFF04F134002263FFF727
:10EFB00077FF04F14C00A264BDE8F04170E7B4EEC5
:10EFC000E70AF1EE10FAE5DCD4ED047A0223D4ED81
:10EFD000066AF8EE677A86EEA77AD4ED0C6A84EDBD
:10EFE000067A86EEA77AD4ED126A84ED0C7A86EE64
:10EFF000A77A84ED127A00E003232370BDE8F08144
:10F00000E02E012010B4019C401A511AA4EB030C0D
:10F010005DF8044B00FB0CFC9CFBF1FC0CEB0300CB
:10F02000704700BF30EE600A32EE612A71EE600A6E
:10F0300022EE002A82EE200A30EE210A704700BF3D
:10F04000DFEDE26AD1ED007A37EEA67ABDEEC76A4F
:10F0500016EE103A2033402B00F25882F4EEE67A96
:10F06000F1EE10FA0CDDDFEDDB5A9FEDD96AF0EE20
:10F07000476A37EE657AF4EEC66AF1EE10FAF6DC0E
:10F08000DFEDDE6AB4EEE67AF1EE10FA0CD5DFEDD4
:10F09000D15A9FEDD16AF0EE476A37EE257AF4EE49
:10F0A000C66AF1EE10FAF6D4DFEDC86AB4EEE67A7D
:10F0B000F1EE10FA40F30282DFEDC96A36EEC77A4C
:10F0C00067EE076ADFEDC74A9FEDC75ADFEDC75A03
:10F0D000A6EEA45A9FEDC66A27EE264AE6EE855AAA
:10F0E000A6EEA56AA4EE067AF0EE474ABDEEE77AF0
:10F0F00017EE103A2033402B00F205829FEDB87ACC
:10F10000F4EEC77AF1EE10FA0CDD9FEDB26A9FEDD6
:10F11000B07AF0EE676A77EEC67AF4EEC76AF1EE7F
:10F1200010FAF6DC9FEDB57AF4EEC77AF1EE10FA3C
:10F130000CD59FEDA86A9FEDA87AF0EE676A77EE8E
:10F14000867AF4EEC76AF1EE10FAF6D49FED9F7A54
:10F15000F4EEC77AF1EE10FA40F3DB819FEDA07A6E
:10F1600077EE677A27EEA77A9FED9E5ADFED9E5ADB
:10F170009FED9E6AE7EE055ADFED9D6A27EE874A0E
:10F18000A7EE256AE7EE066AE4EE267AB0EE675A45
:10F1900091ED017ADFED8D7A77EE276ABDEEE66AB2
:10F1A00016EE103A2033402B00F2A681B4EEE77A37
:10F1B000F1EE10FA0CDDDFED875ADFED857AB0EE67
:10F1C000666A76EEE56AB4EEE76AF1EE10FAF6DC0E
:10F1D000DFED8A7AF4EEE76AF1EE10FA0CD5DFED96
:10F1E0007D5ADFED7D7AB0EE666A76EEA56AB4EE02
:10F1F000E76AF1EE10FAF6D4DFED747AF4EEE76A1E
:10F20000F1EE10FA40F39B81DFED757A77EEE66A56
:10F2100066EEA67ADFED733A9FED734A9FED736A4F
:10F22000A7EEA34ADFED725A66EEA73AA7EE846A0C
:10F23000E7EE865AE3EEA56AB0EE666A66EEC52A88
:10F2400024EEA63AFDEEC77A17EE903A2033402B13
:10F2500000F24F81DFED627AB4EEE77AF1EE10FA58
:10F260000CDDDFED5C5ADFED5A7AF0EE476A37EEDF
:10F27000657AF4EEE76AF1EE10FAF6DCDFED5F7A1C
:10F28000B4EEE77AF1EE10FA0CD5DFED525ADFED6D
:10F29000527AF0EE476A37EE257AF4EEE76AF1EE3D
:10F2A00010FAF6D4DFED497AB4EEE77AF1EE10FA0F
:10F2B00040F33A81DFED4A7A37EEC77A67EE077A94
:10F2C000DFED483A9FED484ADFED486AA7EEA34AD2
:10F2D000DFED475A67EE273AE7EE846AE7EEA65A73
:10F2E000A3EEA57AF0EE476AD1ED027ADFED375A48
:10F2F00037EEA57ABDEEC74A14EE103A2033402B04
:10F3000000F2EC80F4EEE57AF1EE10FA0CDDDFEDC0
:10F31000313A9FED2F4AF0EE475A37EE637AF4EE1A
:10F32000C45AF1EE10FAF6DCDFED345AB4EEE57AA9
:10F33000F1EE10FA0CD5DFED273A9FED274AF0EEFB
:10F34000475A37EE237AF4EEC45AF1EE10FAF6D4A7
:10F35000DFED1E5AB4EEE57AF1EE10FA40F3FA80D2
:10F36000DFED1F5A35EEC77A67EE075ADFED1D1A3B
:10F370009FED1D2ADFED1D3AA5EEA12A9FED1C4A47
:10F3800067EE251AE5EE823AA5EEA34AA1EE847A4D
:10F3900025EE072A64EE871A26EE077A26EE821AF1
:10F3A00026EEA10AFDEEE75A15EE903A2033402BE7
:10F3B00000F28F80DFED0A5AF4EEE57AF1EE10FAF2
:10F3C00027DDDFED043A9FED024A19E0DB0FC93F6C
:10F3D000E4CB1641DB0FC940E4CB16C1DB0FC93FBC
:10F3E000DB0F49409A7C2E36FAAF4FB93587083C7F
:10F3F000A4AA2ABE00000000DB0FC9BFDB0F49C072
:10F40000F0EE675A77EEE37AF4EEC45AF1EE10FAB2
:10F41000F6DC5FED065AF4EEE57AF1EE10FA0CD563
:10F420005FED143A1FED144AF0EE675A77EEA37AB7
:10F43000F4EEC45AF1EE10FAF6D45FED185AF4EE79
:10F44000E57AF1EE10FA40F390805FED1B5A75EE0D
:10F45000E77A27EEA74A5FED1D5A5FED1D3A5FED93
:10F460001D0AE4EE253A67EE845AE4EE230A5FEDC6
:10F47000203AE4EE203AE5EEA37A64EEA74A65EE80
:10F48000275A67EEC67AA6EEA42AE6EEE51A31EE12
:10F49000241A75EEC05A80ED007AC0ED017AC0EDF5
:10F4A000026A80ED031AC0ED041AC0ED052AC0ED12
:10F4B000065A80ED072A80ED083A70475FED326A00
:10F4C000B4EEE67AF1EE10FA7FF5FAAD5FED356A4B
:10F4D000F4E55FED385AF0EE657ADAE71FED3B2A86
:10F4E000F0EE421AB0EE420AB0EE421AB0EE427AA4
:10F4F00058E75FED406AF7E61FED423AF0EE432A27
:10F50000B0EE436A9EE61FED455A41E65FED474A7D
:10F51000ECE51FED477AF4EEC77AF1EE10FA7FF5CD
:10F5200021AE1FED4A7A1BE65FED4D7AB4EEE77A25
:10F53000F1EE10FA7FF5C2AE5FED507ABCE65FEDFA
:10F54000527AF4EEE76AF1EE10FA7FF561AE5FED04
:10F55000557A5BE65FED585AB4EEE57AF1EE10FAB3
:10F560007FF502AF5FED5B5AFCE65FED5D5AF4EEAE
:10F57000E57AF1EE10FA7FF56CAF5FED605A66E761
:10F580000023036143618361C361036003624362DB
:10F590008362C3624360036343638363C3638360C3
:10F5A000036443648364C364C3607047D1ED016A3C
:10F5B000F7EE000A91ED007AF8EEE66AD1ED027AF4
:10F5C000B8EEC77A90ED044AF8EEE77AD0ED054A36
:10F5D00026EEA62A90ED065AE7EE264AD0ED075A07
:10F5E000A7EE275A90ED080AB0EE426AD0ED0A1A4B
:10F5F000A7EE074AD0ED0C2A75EE875A90ED0D3A2A
:10F60000A7EE076AD0ED0E3A90ED091AA7EE260A8A
:10F61000E6EEA71AC0ED054AE7EE272AD0ED104A1C
:10F62000A6EEA73A80ED044AE7EEA73A90ED0F4A1E
:10F6300031EE021A80ED065A90ED0B2AA7EEA76A6A
:10F6400090ED115A34EE274AC0ED075A74EE874AFE
:10F65000D0ED125A35EE265A32EE262A80ED0F4AA8
:10F6600075EEA75AC0ED104A80ED115A80ED080AD8
:10F6700080ED091AC0ED0A1A80ED0B2AC0ED0C2AA4
:10F6800080ED0D3AC0ED0E3AC0ED125AD0ED004AB1
:10F69000D0ED025AE7EE064A90ED015AB0EE657AD7
:10F6A00090ED134AA6EE865A74EE206AA7EE867A8B
:10F6B000D0ED037A37EE866AC0ED136AC0ED004ADA
:10F6C00080ED015A80ED036A80ED027A704700BF39
:10F6D00010B50024034684468646002C00F00D81B8
:10F6E000DEED006A012C9CED007AD3ED007AE6EEA7
:10F6F000C77AC3ED007A00F00F81DEED016A032CBA
:10F700009CED047AE6EEC77AC3ED007A6CD1DEEDAB
:10F71000026A9CED087AE6EEC77AC3ED007AD2ED74
:10F72000007AD0ED044A90ED085AD0ED0C5A92EDD3
:10F73000017AD2ED026A92ED036AA7EEE47AE7EE6F
:10F74000C56AD0ED094AA7EEE56A90ED0D5AD0EDF5
:10F750000E5AE7EE646AA5EE476AA5EEE66A81ED09
:10F76000036A90ED0F5AC1ED026AC6EE055AC1ED6B
:10F77000035A90ED0B6AE5EEC66AC1ED026A90EDA0
:10F780000A5A81ED017A86EE856A81ED026AD0ED32
:10F79000066AA6EE667A81ED017AD0ED076AA5EEDB
:10F7A000E67A81ED017A90ED055AC1ED007AC7EE57
:10F7B000056AC1ED016A90ED017AE7EE667AC1ED66
:10F7C000007A90ED027AE7EE467AC1ED007A90ED8C
:10F7D000037AE7EE657AC1ED007AD0ED006A87EE34
:10F7E000A67A81ED007A10BD9EED007A022CDCED48
:10F7F000016AD3ED017AB1EE476AE7EE667AC3EDAE
:10F80000017ADEED016A9CED057AE6EEC77AC3ED7A
:10F81000017A40F0AC80DEED046A012C9CED007AA8
:10F82000D3ED047AE6EEC77AC3ED047A40F287801E
:10F83000DEED056A032C9CED047AE6EEC77AC3ED93
:10F84000047A7FD19EED066ADCED086A93ED007ABA
:10F85000E6EE667AC7EE876AC3ED046A9EED086A33
:10F86000012CDCED006AD3ED087AE6EE667AC3ED92
:10F87000087A70D99EED096A032CDCED046AE6EE85
:10F88000667AC3ED087A07D19EED0A6ADCED086A54
:10F89000E6EE667AC3ED087A93ED086A032CD3EDA1
:10F8A0000C7AC6EE076AC3ED086A9CED006ADEEDCD
:10F8B0000C6AE6EE667AC3ED0C7A9CED046ADEED26
:10F8C0000D6AE6EE667AC3ED0C7A07D19EED0E6AFC
:10F8D000DCED086AE6EE667AC3ED0C7AD3ED0C6ACD
:10F8E000C6EE877AC3ED0C7A013414330EF1100E94
:10F8F0000CF1040C002C7FF4F3AED3ED047A93EDFD
:10F90000007A93ED086AC7EE876AC6EE077AC3ED00
:10F91000046AC3ED087AE1E7DEED006A9CED016A56
:10F9200093ED017AD3ED027AA6EEC67A83ED017AE1
:10F930009CED027AE7EE667AC3ED027A6BE793ED0F
:10F94000007A87E793ED007A022CC7EE876AC3ED51
:10F95000046AC9D082E7C7EE876AC3ED086AC3D0DC
:10F960009CED006ADEED0C6AD3ED0C7AB2E79CEDFB
:10F97000027A032CD3ED027AE6EE077AC3ED027A1F
:10F98000DCED066A9EED017AE6EEC77AC3ED027AF7
:10F990007FF441AFDEED026A9CED0A7AE6EEC77AAB
:10F9A000C3ED027ABBE600BF10B584B00C46024638
:10F9B00010306946FFF78CFEB6EE006ADDED006A96
:10F9C00001209DED017ADDED027A66EE866A27EE72
:10F9D000067A67EE867AC4ED006A84ED017AC4ED9A
:10F9E000027A04B010BD00BFF0EE407A9FED060A27
:10F9F000BEEE007A60EEA00A67EEA77A67EE877A1D
:10FA0000C7EEA00A54F04CB954F82D4008B551F097
:10FA10008DF907EE900AF5EEC07AF1EE10FAACBF60
:10FA2000B1EEE70A9FED010A08BD00BF000000002B
:10FA300060EEA00AE0EE000AB1EEE00A704700BFF7
:10FA400021EE011AA0EEA01AA0EE001AB1EEC10A32
:10FA500070472DE9F74F90469DF8302005460F4638
:10FA6000002A0D9A14BF4FF030094FF020091C1ED8
:10FA7000BABF64420123002312F8011B01B12CB963
:10FA8000A24663B100240D9EA41B12E0013CF3E7E3
:10FA9000BD4204D2494628460193C047019BBAF1B2
:10FAA000010AF5D2EFE7BD4203D228460193C047D1
:10FAB000019B06EB040B16F8011B0029F3D133B1AF
:10FAC0005446002C07DCBAF1000FA8BFD3445846B7
:10FAD00003B0BDE8F08FBD4202D249462846C04778
:10FAE000013CEEE70FB437B506AB0A4D53F8042BD3
:10FAF000D5E9E50101934DF091FB0446D5F880036B
:10FB000005F0B7FE0028F9D0204603B0BDE830402C
:10FB100004B07047107301200EB403B503AB08495D
:10FB200053F8042BCDE9003001A84DF077FB019B81
:10FB300000221A7002B05DF804EB03B0704700BFFA
:10FB400053D800080CB430B52C4CA5B0D4F89C3375
:10FB50001BB9D4F8A033002B39D094F8A4339942C0
:10FB600006D9012303FA00F0D4F8A83318422ED0A6
:10FB7000234B04A819684FF47A73B1FBF3F203FB2B
:10FB800012132049FFF7C8FF04AB289A0546034427
:10FB90001D4903A8039329AB02934DF03FFB039B40
:10FBA0000246D4F89C03591C03910A211970039B47
:10FBB000591C03910021197090B103681B6A03B1AD
:10FBC0009847D4F89C5304AC14F8011B21B925B014
:10FBD000BDE8304002B07047284605F0DBFDF3E792
:10FBE000D4F8A033002BF2D002212A44FD200A448D
:10FBF000009104A923F0FEFAE9E700BF1073012089
:10FC0000E02E01206B0D0708F5D7000830B54FF442
:10FC1000004087B021F0A8FC0446A0B34FF4004197
:10FC200021F004FE02281CD1226848F201039A4206
:10FC300029D1234C00254FF4004084F840564CF065
:10FC4000B3FF00B3D4F8AC3383421ED0D4F8883469
:10FC500083422FD0D4F8643598422ED0C4F8A053F4
:10FC600011E00023022294F904004FF40041CDE991
:10FC700001234FF4612200921A4621F03EFE104B00
:10FC8000C3F89C0328B907B030BD04F56B73C4F802
:10FC9000A0330C4B02210C4A002004930B4B03931E
:10FCA0000B4B02930B4B01930B4B00930B4BFFF74A
:10FCB00049FFE8E704F59163E9E704F26453E6E7F6
:10FCC00010730120770D0708821A0708800D0708B6
:10FCD000890D0708950D07089B0D0708720C07088A
:10FCE000174A033038B5D2F8444604EB9003B3F515
:10FCF000007F18D802F5C965C2F8443602EB8102CC
:10FD000020F00300C3F5007305EB8404D2F8481E0D
:10FD10009B0008440421C2F8480E0020094AFFF75E
:10FD200011FF204638BD0021074A00240846FFF78E
:10FD300009FF064A136843F000731360F1E700BF40
:10FD400010730120A90D0708CC0D07080000002042
:10FD500003685A1C02601970090A03685A1C026081
:10FD60001970704703685A1C0260197003685A1CA6
:10FD700002600A0A1A7003685A1C02600A0C090E13
:10FD80001A7003685A1C02601970704703685A1C85
:10FD900002600A0A1A7003685A1C026019707047E0
:10FDA00038B504460068154656F0F0FC23682B442D
:10FDB000236038BD03685A1C0260187870470368D6
:10FDC0005A1C02601A4612F8021B0260587841EA77
:10FDD0000020704702681146531C10B50360D31C05
:10FDE00011F8024B01605178036093781B0443EAD9
:10FDF0000123111D23430160D07843EA006010BD48
:10FE0000D1E900329A4206D05A1C0A6008B11B7828
:10FE100003700120704700207047D1E9002310B51E
:10FE20009B1A04460846012B04DDFFF7C8FF20801B
:10FE3000012010BD0020FCE730B50A440446914281
:10FE400001D1002011E014F8013BA3F14100192871
:10FE500011F8010BA0F1410598BF2033192D98BF6F
:10FE600020301B1A02D10028E9D130BD1846FCE72A
:10FE7000028810B5A2F5FA62C37840F2B554910831
:10FE8000013B02F0030204FB013381780C240139A9
:10FE900004FB02120C49847901EB42021821B2F8EA
:10FEA00088201344027901FB03223C214379008915
:10FEB00001FB0233054A224401FB03224FF47A730B
:10FEC0000021C2FB030110BDDC7C060880436D38B5
:10FED0002DE9F04190461F4605464FF47A72002303
:10FEE0004046394651F080F8274B3C21034493FBB0
:10FEF000F1F201FB1233AB7192FBF1F301FB132220
:10FF000040F2B5516A71182293FBF2F402FB1433EC
:10FF100094FBF1F201FB12442B719300B4F5896F4D
:10FF20002EDA40F2DA2294422CDCB4F5B77FB4BF6B
:10FF300000210121154A18200B2600FB012232F86E
:10FF40001600A04201DD013EF9D103F5FA63013448
:10FF50004FF47A7240460B442B80731CAB700C2319
:10FF600003FB01660A4B394603EB4606B6F88830B8
:10FF7000E41A0023EC7051F037F82A81BDE8F081D3
:10FF80000321D7E70221D5E780BC92C7647D06082C
:10FF9000DC7C0608F0B5274D8DB006460F466C4652
:10FFA0000FCD0FC40FCD0FC495E80F0084E80F00EC
:10FFB00016F0030339D1642196FBF1F201FB1262C2
:10FFC00042B94FF4C87296FBF2F302FB1363003B95
:10FFD00018BF0123721EC3F11D0369460024002AC5
:10FFE000019340F26D131046B8BFB01C0725734350
:10FFF000013F03EBA0006FF0630392FBF3F318449F
:020000040801F1
:100000004FF4C87392FBF3F21044063051F8042BFE
:10001000A74202EB000393FBF5F0C0EBC000A3EB9B
:10002000000004D1101A0DB0F0BD0123D2E7013455
:10003000ECE700BFC47D0608094BD3F8D01ED3F807
:10004000D42E51EA020308D0064B1B685B1842F11C
:100050000002C0E90032012070470020704700BF55
:1000600010730120E02E012037B505466846FFF7E2
:10007000E3FF044638B12846DDE90023FFF728FFF7
:10008000204603B030BD40F201132880A8806B8069
:10009000A8712881F4E700BF884270B54FF00104D1
:1000A0005AD301FB04F4B0FBF4FC8C45F9D2002CCC
:1000B0004ED0BAB10025BCF1000F1A4604FB1C005B
:1000C000D4BF00260126B4FBF1FE85BB7EBBA14256
:1000D000354639D91A460CF1300C02F801CB002311
:1000E000137070BD154605E0A1427546F2D834463E
:1000F000B0FBF6FCBCF1000F1A4604FB1C00B4FB7D
:10010000F1F606DCB5F1000E18BF4FF0010E002D20
:10011000EAD0BCF1090F05F10105CCBF572330230C
:10012000A1429C4402F801CB1346E0D9D7E7BCF1C9
:10013000090F05F10105CCBF37233023A1429C44B0
:1001400002F801CB1346CAD87446B0FBFEFCB2E7F6
:100150001A460023137070BD8446002AAAD1C1E755
:100160000028BCBF2D23404270B5B8BF01F8013B49
:10017000092884464FF0010307DD03EB83035B008E
:10018000B0FBF3F2092AF8D843B30024164EA6FBBD
:1001900003508E46BCFBF3F2002A4FEAD00003FB6B
:1001A00012CCD4BF0025012554B94DB9092B2C46DA
:1001B00012D830320EF8012B00238EF8003070BDBB
:1001C000092A04F101048CBF57213021092B0A446C
:1001D0000EF8012B7146EFD90346D8E78E4600236F
:1001E0008EF8003070BD00BFCDCCCCCC90420B4619
:1001F0002DE9F041B0FBF2F60446154608D2124A4A
:1002000005FB16441846135D00F8013BBDE8F0817C
:100210009642B6FBF2F706D20B4A05FB1767D15D93
:1002200003F8011BECE7BA42B7FBF2F807D905FB6C
:100230001878054A12F8081003F8011BEDE740464C
:10024000FFF7D4FF0346F2E7080E0708B5EEC00A31
:10025000DFED317A0023F1EE10FA70B5C8BF30EE51
:10026000270A86B0D8BF30EE670ADFED2C7A054644
:1002700003A902936E4620EE270ACDE90033FDEE76
:10028000C07A17EE904A84EAE470A0EBE4704DF077
:100290008FFA002C03A8ACBF20232D238DF800304B
:1002A00050F0B0F8012827D002282ED003281DD006
:1002B00003A9304656F072FD304650F0A3F80446CC
:1002C00031462846033CE4B2224656F05FFA00234A
:1002D00028462B5550F096F82E22431C31192A54EB
:1002E000E81856F077FD284606B070BD302303A904
:1002F00030468DF80130DDE743F23002302303A9A8
:10030000ADF801208DF80330D3E743F2300303A9A1
:100310003046ADF80130CDE76F12033A00007A4461
:100320000378092B01D0202B05D110F8013F202B99
:10033000FBD0092BF9D02D2B00F0AC802B2B78D0E3
:10034000A3F13002B7EE000AD1B209297AD8F2EE51
:10035000046ADFED5C7A07EE102A10F8013FB8EE70
:10036000C77AA3F13002D1B2A7EEA67A0929F0EE3E
:10037000477AF0D92E2B69D003F0DF03452B40F0EC
:10038000868010B442782D2A00F091802B2A0DBF70
:100390008278A2F130030130023008BFA2F13003AD
:1003A000092B7BD80024002303EB830302EB4303D8
:1003B00010F8012FA2F13001303B0929F4D9B3F52F
:1003C0009A7F1A46B7EE007A28BF4FF49A72072B2D
:1003D00009D91346DFED3C6A083B27EE267A072B46
:1003E000FAD802F00702DAB1F2EE046A012A27EE27
:1003F000267A15D0022A27EE267A11D0032A27EE74
:10040000267A0DD0042A27EE267A09D0053A27EE5F
:10041000267A05D027EE267A012A18BF27EE267AFB
:10042000002C3DD0C7EE877A5DF8044B20EE270AFA
:100430007047B7EE000A4378A3F130020130D1B221
:10044000092984D92E2BDFED1F7A95D1437801300D
:10045000A3F13002D1B209298ED8B2EE047AF0EEBF
:10046000475A06EE902A10F8013FB8EEE66AA3F16B
:100470003002D1B2C6EE076A092927EE257A77EE57
:10048000A67AEED903F0DF03452B3FF47AAF20EED6
:10049000270A7047BFEE000A4378CDE7B7EE007A2F
:1004A00067EE877A5DF8044B20EE270A7047827862
:1004B0000230A2F13003092B01D8012473E7B7EE13
:1004C000007AAFE70000000020BCBE4C0246037873
:1004D00001E012F8013F202BFBD0092BF9D0303B73
:1004E0000020DBB2092B0AD812F8011F00EB8000B4
:1004F000303903EB4000CBB2092BF5D97047704778
:10050000037801E010F8013F202BFBD0092BF9D034
:100510002D2B06BF01304FF0FF3C4FF0010C01784E
:10052000A1F13002D3B2092B4FF0000302D903FB33
:100530000CF0704710F8011F03EB830302EB430339
:10054000A1F13002D1B20929F0E7002310B58028CB
:1005500004D893420AD2C854581C10BD934205D007
:1005600060F07F04C009CC540133F0E74FF0FF3056
:10057000F3E770B5124C0122124E00201249FDF72C
:10058000B5FF228862B1A31DB34217D2A518B542A8
:1005900014D2052A12D921462C46FDF7A7FFF0E711
:1005A00021460222FDF7A2FF63880849C31A084AC0
:1005B000641A5842A2F8D84E584170BD0020FCE79A
:1005C000014000080080000800400008FC3F0008CF
:1005D0001073012003682DE9F0411344044640687C
:1005E00083421AD80D468E18002704F10C08B54234
:1005F000606901D1BDE8F08123695A1C234422615E
:10060000042A15F8011B1973F1D118B94146204687
:10061000FAF79EFAC4E90470E9E74FF0FF30E9E722
:10062000034AD2F8DC3E1843C2F8DC0E704700BF24
:1006300010730120034AD2F8DC3E23EA0000C2F81E
:10064000DC0E7047107301200346064906488842B5
:1006500001D3002070470288C2F30B029342F9D005
:100660001430F4E7148B07083C86070842880B46D1
:1006700013B5C2F30B02044600211846019256F04E
:10068000CFFA216903460A48814209D30948019AF1
:10069000814205D2184602B0BDE8104056F076B847
:1006A00021B1184602B0BDE81040084702B010BDA5
:1006B000148B0708BA8F070810B4B0F902400B4634
:1006C0004288002C41685DF8044BBEBFC2F30B02A8
:1006D000DBB203FB0211C9E730B5094B094CA34259
:1006E00000D330BDB3F902205988002A06DA5A68CF
:1006F000C1F30B01DD6800FB01222A601433EEE731
:100700003C860708148B070802460144002030B5D8
:1007100012F8015B082480EA050340086D0813F015
:10072000010F1CBF80F08C03D8B2631E13F0FF04CE
:10073000F1D18A42ECD130BD144901EB8000806BCD
:1007400070B500B30C2202FB001292F9E930581C7C
:100750001AD092F8F100B0B1C818642592F8F040B0
:10076000142290F824616B4300201D19013A34448F
:1007700001EB4505B5F8285110FA85F0F5D11423A1
:10078000B0FBF3F080B270BD0020FCE710730120D5
:1007900010B5427A044632B10146406851F80A3B2E
:1007A00098470023637210BD10B4447A621C04445D
:1007B000D2B24272A172037A934202D85DF8044B1E
:1007C000E6E75DF8044B7047036810B51A790446F4
:1007D000022A02D1987A4EF0D3FD002323602371C0
:1007E00010BD2DE9F0471F46AB4DAC4B9D4221D2C9
:1007F0006C798C4240F06E812C79844202D00028C2
:1008000040F06881EC79944240F064812C68DCB15E
:100810001C220021201D56F003FA25602B7923713C
:10082000012B95F80680C4F808802A7AE26003D08C
:10083000022B0CD0002407E0E87A02F0F1FF6B7A7B
:10084000A0612374AB7A63742046BDE8F087E87A30
:1008500002F0E6FF95F90960A0612674A87A02F01B
:10086000DFFF6061002800F0318114238C4D734359
:1008700005EB0309EB58002B00F0288199F81230A2
:10088000002B40F0EE8099F808004CF04FFE99F8EC
:100890000830012103F01F025B09023B01FA02F25A
:1008A000032B08D8DFE803F0827C02767D490B69D0
:1008B00023EA02020A61142306F1010A03FB06532C
:1008C0005FFA8AFA587902F0ABFF814620B140F610
:1008D0000A3380F808A0C380142303FB0653D87999
:1008E00002F09EFF20B140F60A5380F808A0C380B2
:1008F000142303FB0653987902F092FF20B140F6CF
:100900000A4380F808A0C380142348464FF0140916
:1009100018F0040803FB065309FB065918BF4E21C3
:100920005A7A08BF2E2102F05BFF99F8070002F007
:1009300077FF99F80A202E2102F052FF99F806005D
:1009400002F06EFF99F80B200E2102F049FF99F892
:10095000040050B102F064FF20B140F60A6380F851
:1009600008A0C3800D2102F01AFF14237343EA5834
:10097000136823F0400313604B4B9A421CD103F5DC
:100980008433596A41F480515962596A21F4805183
:1009900059622AE043494B6923EA02024A618AE725
:1009A00040490B6A23EA02020A6284E73D494B6A26
:1009B00023EA02024A627EE73C4B9A420CD003F5DE
:1009C00080639A425BD1374B196A41F40041196246
:1009D000196A21F4004107E0324B196A41F4804161
:1009E0001962196A21F4804119625368B8F1000F45
:1009F00043F4805314BF00200220536013685B0649
:100A000015D4116821F47F4121F0BF01B8F1000F26
:100A100008BF41F00101014341F445711160536881
:100A200023F4706323F0040343F4E0635360D36959
:100A300023F40063D361136843F0400313605368E9
:100A400043F480535360142303FB0653187918B101
:100A500002F0E6FE02F098FE142303FB0655012384
:100A6000AB74606920B10E238771C37100230372D8
:100A70000D2102F094FE606902F086FEE4E60C4B64
:100A80009A4217D1074B596A41F400515962596A89
:100A900021F400517CE700BFE8010008680300086A
:100AA00000000120003802400030014000380040C2
:100AB00000340140084B9A4297D1084B596A41F4DF
:100AC00080115962596A21F4801161E72046FFF7CD
:100AD0007BFEAFE60C3589E600500140003802404D
:100AE00073B50279022A38D190F910301426032008
:100AF0000025734302AE8DF80300012431441A48E7
:100B00008DF80050C3588DF801408DF8022011F87F
:100B1000086C16498B4222D0A1F578418B4220D037
:100B200001F580618B4205D0114A934214BF4FF00A
:100B3000FF3203221968142421F0400104FB020251
:100B40001960D068196821F0380250F826100A435D
:100B50001A601A6842F040021A6002B070BD2A465C
:100B6000E8E72246E6E700BF000001200030014030
:100B70000034014013B5474CC2B20D232F2102208F
:100B8000FFF72FFEC4F88403B0B30321FFF7A8FFDB
:100B90009F233220009304F06CFF00236A46D4F8B0
:100BA00084038DF8053004230DEB03014EF0C2FBE6
:100BB0009DF806209DF80530120242EA03429DF896
:100BC00007301A43344B9A42344B5ED047DC3449E9
:100BD0008A4255D024DC33498A4227D001F5D61108
:100BE00001F6FF718A4252D02F498A4248D0002034
:100BF00018809881C3E9010002B010BD2B4911444F
:100C00000429F4D801A252F821F000BF810C010898
:100C1000EF0B01088F0C01082D0C0108770C01085F
:100C200023498A4233D001318A42E0D14FF48072A5
:100C30001A809A8100229A735A8811021A884A43AC
:100C40005960B2F1807F9A6005D90123B72084F8FA
:100C50009033FDF72BFB012084F88803CCE715497E
:100C60008A420BDC05398A42C8DC13498A420ED01D
:100C700002318A42BBD14FF4007202E00F49D3E740
:100C800020221A804FF48072D3E74022F9E78022B5
:100C9000F7E700BF107301201620C2009812012050
:100CA000152020001860010015400100EBBF10FF67
:100CB00017BA20001940EF001720C2001870EF008B
:100CC000C36910B5044623B909211420FFF708F8B9
:100CD000E061E06910BD10B504460068FFF7F0FF61
:100CE000837853B183885BBAE381C3885BBA23827C
:100CF000038901205BBA638210BD1846FCE710B57A
:100D000000680C46FFF7DCFF83784BB14389222251
:100D10000120DBBA93FBF2F303F26D13238010BDC5
:100D20001846FCE710B504464FF4FA7004F022FEB2
:100D30006069BDE8104002F027BDF7B515461E46B4
:100D4000142290F91030044653430E4AD758836852
:100D50009A0704D4406901914EF0BAFA01993846D5
:100D60004EF0A4FD33462A4600213846FAF73EFDF0
:100D7000A3689B0702D42046FFF7D4FF012003B0ED
:100D8000F0BD00BF00000120F7B507791646012F1E
:100D90000AD0022F15D18468E40758BF41F08001C2
:100DA00003B0BDE8F040C8E7826802F00102CDE977
:100DB00000620A46417C90F91000FAF7BDF803B0D2
:100DC000F0BD0020FBE7F7B515461E46142290F94A
:100DD0001030044653430E4AD75883689A0704D408
:100DE000406901914EF074FA019938464EF05EFD6B
:100DF0003346002229463846FAF7F8FCA3689B07D9
:100E000002D42046FFF78EFF012003B0F0BD00BFE3
:100E100000000120F7B507791646012F0AD0022FEE
:100E200015D18468E40758BF41F0800103B0BDE8E4
:100E3000F040C8E7826802F00102CDE900620A468C
:100E4000417C90F91000FAF73BFA03B0F0BD0020A6
:100E5000FBE713B506236A46F7210068FFF7DAFFC0
:100E6000134BE8B19DF801109DF8002009019DF891
:100E7000034041EA02319DF8022041EA12119DF837
:100E8000042012019966C3F8E01E42EA04329DF87C
:100E9000054042EA14129A64C3F8E42E02B010BD71
:100EA000D3F8E02E9A66D3F8E42E9A64F6E700BFF2
:100EB00010730120032307B5194601AA0068FFF744
:100EC000A9FFA0B19DF804309DF904209DF80510FC
:100ED0001B04002A43EA01239DF80610B4BF4FF01B
:100EE0007F4200220B431343024AC2F8E43003B0AE
:100EF0005DF804FB1073012007B5032301AA00214C
:100F00000068FFF787FFA0B19DF804309DF9042029
:100F10009DF805101B04002A43EA01239DF80610E2
:100F2000B4BF4FF07F4200220B431343024AC2F882
:100F3000C83003B05DF804FB1073012070B506687B
:100F400005463046FFF7BCFE0446021D0E233B213A
:100F50003046FFF75FFFA07040B1A3895BBAAB8357
:100F6000E3895BBAEB83238A5BBA2B8470BD13B52C
:100F7000044600686A460379022B4FF006030CBF53
:100F800043210321FFF746FF18B9E086A06302B0B2
:100F900010BDBDF800305BBAE386BDF802305BBA25
:100FA0006387BDF804305BBA2387F0E713B50623E7
:100FB00004466A4611210068FFF72CFF18B9E08645
:100FC000A06302B010BDBDF90030F7EE086A07EE6D
:100FD000103AB8EEC77A27EE267ABDEEC77A17EE3A
:100FE000103AE386BDF9023007EE103AB8EEC77A40
:100FF00027EE267ABDEEC77A17EE103A2387BDF9A1
:10100000043007EE903AF8EEE77A67EEA67AFDEE46
:10101000E77A17EE903A6387D3E7002313B5C386C8
:10102000044683636A46062303210068FFF7F2FE45
:1010300078B1BDF8003003EB4303E386BDF902301D
:101040005B4203EB43032387BDF8043003EB430308
:10105000638702B010BD73B590F9103015461422A5
:10106000044653430C4AD65883689A0704D440690F
:1010700001914EF02DF9019930464EF017FC2946AA
:1010800030464EF013FCA3689B0702D42046FFF7BE
:1010900049FE012002B070BD000001207FB5037938
:1010A0000D46012B0AD0022B19D18368DB0758BFEC
:1010B00001F07F0104B0BDE87040CCE781688DF895
:1010C0000F200DF10F0201F0010100922A4601915B
:1010D000417C90F91000F9F72FFF04B070BD00209B
:1010E000FBE7012258210068D8E701224821006867
:1010F000D4E73122F421006808B5FFF7CFFF0120C3
:1011000008BD022208210068C8E701220821006802
:10111000C4E7F022FF210068C0E7B422FF21006885
:10112000BCE7CA43006841EA0212D221D2B2B5E755
:101130000A460068A521B1E75521F9E79622FF216B
:101140000068ABE70A4600688721A7E7C901006885
:1011500001F080027821A1E7F7B5C16A0446424F49
:10116000056890F82900B7FBF1F189B24BF048F916
:101170004388064600212846B7FBF3F76763FFF76D
:10118000AFFC80226B212846FFF788FF962004F0F1
:1011900070FC032268212846FFF780FF962004F0A8
:1011A00068FC03226B212846FFF778FF0F200021FF
:1011B00004F04EFC10226A212846FFF76FFF0F2033
:1011C000002104F045FC00226C212846FFF766FF51
:1011D0000F20002104F03CFC727919212846FFF70A
:1011E0005DFF0F20002104F033FC18221B2128464C
:1011F000FFF754FF0F20002104F02AFC18221C21C5
:101200002846FFF74BFF0F20002104F021FC327924
:101210001A212846FFF742FF0120002104F018FCA4
:1012200003212846FFF75CFC06236A464321206819
:10123000FFF7F0FD58B1BDF800305BBAA383BDF8ED
:1012400002305BBAE383BDF804305BBA238494F9BF
:101250001E30013306D194F91C30013302D106202F
:1012600004F054FC03B0F0BD40420F00F8B5C16A71
:1012700005462C4F046890F82900B7FBF1F189B2BC
:101280004BF0BEF84388064600212046B7FBF3F733
:101290006F63FFF725FC80226B212046FFF7FEFEDF
:1012A000642004F0E6FB072268212046FFF7F6FEE3
:1012B000642004F0DEFB00226B212046FFF7EEFEE7
:1012C000642004F0D6FB01226B212046FFF7E6FEE6
:1012D0000F2004F0CEFB18221B212046FFF7DEFE74
:1012E0000F2004F0C6FB18221C212046FFF7D6FE73
:1012F0000F2004F0BEFB32791A212046FFF7CEFE04
:101300000F2004F0B6FB727919212046FFF7C6FEC4
:10131000642004F0AEFB20460321BDE8F840FFF74F
:10132000DFBB00BF40420F0010B578220446002109
:101330000068FFF7B3FE052004F09BFB202201218B
:101340002068FFF7ABFE052004F093FB002202218A
:101350002068FFF7A3FE642004F08BFB012010BD82
:1013600010B52422044641210068FFF797FE80B1A2
:10137000202230212068FFF791FE50B10622312152
:101380002068FFF78BFE20B1002234212068FFF790
:1013900085FE052004F06DFB012010BD10B507226D
:1013A00004460A210068FFF779FE052004F061FB7E
:1013B000242241212068FFF771FE052004F059FB2B
:1013C000C02242212068FFF769FE052004F051FB8E
:1013D000012010BD10B50446002221210068FFF74E
:1013E0005DFEFC2220212068FFF758FE40222421C8
:1013F0002068FFF753FE0C2223212068FFF74EFEE2
:10140000002222212068FFF749FE012010BD10B5FF
:101410000122044610210068FFF740FE40B114206D
:1014200004F027FB2068A0221121BDE8104035E61A
:1014300010BD10B5012204460B210068FFF72EFEF7
:1014400020B11D2209212068FFF728FE00F00100CD
:1014500010BD044B0246D3F8E80E08B180211DE60A
:10146000704700BF1073012073B590F91030154616
:101470001422044653430E4AD65883689A0704D46C
:10148000406901914DF024FF019930464EF00EFA6B
:101490000123002229463046FAF7A8F9A3689B07E2
:1014A00002D42046FFF73EFC012002B070BD00BF11
:1014B0000000012073B503791646012B0AD0022BD8
:1014C00015D18368DB0758BF41F0800102B0BDE849
:1014D0007040C9E7826802F00102CDE900620A4665
:1014E000417C90F91000F9F7EBFE02B070BD0020CE
:1014F000FBE7F8B504460E461546071D3A46FF21A0
:101500002068FFF7D7FF30B116B12379DB07F5D498
:101510000DB123792B70F8BD00220121E9E710B548
:101520000446FFF7FAFD18B12046BDE81040F3E786
:1015300010BD10B50446FFF7FBFD18B12046BDE80D
:101540001040E9E710BD73B50546CDE90023FFF76C
:10155000E6FFA8B12846FFF7EFFD88B12846FFF760
:10156000DBFF68B16E46082416F8011B2846FFF71A
:10157000E0FF28B1013C14F0FF04F5D102B070BDCA
:101580000020FBE7CC21D4E770B506460C468D1849
:10159000AC4201D1012006E014F8011B3046FFF7F0
:1015A000C8FF0028F4D170BD38B505461446FFF7D2
:1015B000C9FD2846FFF7B0FF20B11CB12B79C3F35A
:1015C0004013237038BD10B50446FFF7A8FF38B1AB
:1015D0002046FFF7D7FF18B12046BDE810409BE733
:1015E000002010BD2DE9F04F002587B08046049300
:1015F0000195CDE90212039B4046EC0003EBC50ABE
:10160000FFF78DFF024600286CD0002201214046E2
:10161000FFF76FFF0246002864D098F8043099075E
:1016200060D5F0214046FFF784FF0246002859D0DC
:10163000A4F108024FF0000B0127039B5E46134400
:101640003C460593029B002B54D0082C52D804F141
:10165000FF3943FA09F909F0010949464046FFF705
:1016600075FD024600283DD0002201214046FFF7CB
:1016700040FF0246002835D098F8041001F0600CB5
:10168000C809BCF1600F16D0029B1BB1082C01D811
:10169000814527D1002841D01AF8061039437F0030
:1016A00001340AF8061017F0FF07E4B2CAD1013678
:1016B000F6B2082E1CD1402C10D9072150460592B5
:1016C000FFF722F89AF80710059A814206D10135F2
:1016D000EDB2BBF1000F05D0CDF804B0049B1B7830
:1016E000AB4288D8049B10461D7007B0BDE8F08F50
:1016F0000127A7E75DB1019BA34208D9059B9A5D2D
:10170000174214BF4FF001094FF00009A5E7019BF4
:101710001B1BD3F1000949EB03099EE7880940EA46
:10172000511111F0010F1AF8061008BFA34621EA63
:101730000701B4E7C90138B501F080010446154638
:10174000FFF704FD08B9002038BD00220121204622
:10175000FFF7CFFE0028F6D023795B092B70F3E763
:1017600010B5021D0446FF210068FFF7A3FE18B163
:101770002079C04300F0010010BD38B5044615467D
:1017800000680A46E121FFF789FC28B12A46206853
:10179000FF21BDE838408DE638BD0A46C321ECE79D
:1017A00038B5021D0D46F0210446FFF7E6FF08B1EB
:1017B00023792B7038BD0A46E121DEE738B50446AF
:1017C0000D46FFF7BBFC40B12046FFF7A5FE20B158
:1017D00029462046BDE83840EDE7002038BD70B509
:1017E00006460C468D18AC4201D1012006E0214688
:1017F00030460134FFF7E2FF0028F4D170BDF7B5A1
:1018000015460DF107021C4606460F46FFF752FE2D
:101810009DF8073005EA0302A24208D023EA050238
:1018200039463046224303B0BDE8F04036E403B009
:10183000F0BD09230C211A4630B5044687B0FFF7E6
:10184000DEFF282004F015F901AA08212046FFF741
:1018500031FE9DF904209DF80430002A03DB0025A9
:10186000284607B030BD5D06F9D5122301AA102124
:101870002046FFF7CFFA05460028F0D09DF8052056
:101880009DF804301109120241EA0311DB09544B9F
:1018900002F4706218BFA1F5805110059DF8070091
:1018A00019839DF8061041EA02019DF8082048BFFF
:1018B000A1F580511201598342EA00329DF80910C6
:1018C00042EA11101203BDF80A204FEA014148BF55
:1018D000A0F5801052BA01F47021D86192B20A4387
:1018E000090348BFA2F580121A62BDF80C2052BA53
:1018F00091B21204BDF80E2048BFA1F5803152BA52
:101900009984100491B2BDF8102048BFA1F5803130
:1019100052BAD98491B21204BDF8122048BFA1F581
:10192000803152BA1985100491B2BDF814202046B6
:1019300048BFA1F5803152BA598591B212044FF0D7
:10194000070248BFA1F58031998500230821FFF7E0
:1019500056FFA5220E212046FFF7A0FB96220F215D
:101960002046FFF79BFB022262212046FFF796FBF1
:1019700000220E212046FFF791FB00220F21204676
:10198000FFF78CFB0223072208212046FFF737FFD1
:10199000282004F06EF85423204606211A46FFF74B
:1019A0002EFF0DF1030228212046FFF783FD9DF84D
:1019B00003302046072123F07F0343F054031A46E7
:1019C000FFF71DFF0C23204609211A46FFF717FFDA
:1019D0000723082120461A46FFF711FF40E700BF02
:1019E0001073012013B504466A4608210068FFF70A
:1019F00061FD9DF8003013F010037ED006236A4687
:101A000000212068FFF706FA002874D09DF8013005
:101A10009DF800201B029DF804109FED396A03EB2E
:101A200002439DF8022009021A441C029DF803306B
:101A300048BF02F17F4201EB03419DF8053007EEFC
:101A4000902A0B440902F8EEE77A48BF03F17F437E
:101A5000C7EE866A07EE903A2A4BB3F92C20B8EE0F
:101A6000E77A07EE902AB3F92820F8EEE77AC7EE76
:101A7000065A06EE102AB3F92420B8EEC66AA6EE7E
:101A8000A76AD3ED087AB8EEE77AD3ED077AF8EED5
:101A9000E77AA6EE867A26EEA55AE6EE877A07EE74
:101AA000102AB3F92A20B8EEC77A06EE102AB3F945
:101AB0002620B8EEC66AE5EE877A07EE102AB3F95B
:101AC0001820B8EEC77AA6EE867AF6EE006AE5EE42
:101AD000077A07EE102AB3F91A20B8EEC77AC3EDD9
:101AE0000C7A07EE902AF8EEE77A67EEA57AE7EE31
:101AF000267AC3ED0D7A02B010BD1846FBE700BF91
:101B0000000078481073012013B5002204460A2112
:101B10000068FFF7C3FA142003F0ABFF0F220A217D
:101B20002068FFF7BBFA0A2003F0A3FF032301AAF2
:101B300010212068FFF76EF90A2003F09AFF0022B7
:101B40000A212068FFF7AAFA0A2003F092FF0DF19C
:101B5000030202212068FFF7ADFC0DF10302092109
:101B60002068FFF7A7FC01220A212068FFF796FAF8
:101B7000012002B010BD30B5002385B0044602211B
:101B8000C3860DF1070283630068FFF793FC18B961
:101B90000025284605B030BD9DF80730DB07F7D596
:101BA000062302AA03212068FFF734F90DF107028A
:101BB00009212068FFF77EFC05460028E8D09DF843
:101BC000073013F00C0FE3D1BDF8083001220A21D1
:101BD0002068C3EB83339B00E386BDF80A309B008B
:101BE0002387BDF80C30C3EB83339B006387FFF77B
:101BF00055FACEE71FB5002304460DF10702272151
:101C000000688DF80730FFF755FC68B19DF8073084
:101C100013F0080320D0062302AA28212068FFF72A
:101C2000F9F818B9E086A06304B010BDBDF908301A
:101C3000002BB8BF03339B10E386BDF90A30002B9D
:101C4000B8BF03339B102387BDF90C30002BB8BFFE
:101C500003339B106387E7E71846E5E71FB50021CC
:101C600004460DF10702C18681630068FFF722FC7C
:101C7000C0B19DF8073013F0080315D0062302AA5F
:101C800001212068FFF7C6F860B1BDF808305BBAE3
:101C9000E386BDF80A305BBA2387BDF80C305BBA27
:101CA0005B42638704B010BD1846FBE730B50025E2
:101CB00085B004460621C5860DF1070285630068DC
:101CC000FFF7F8FBA0B19DF8073013F0040311D023
:101CD000062302AA29462068FFF79CF840B1BDF808
:101CE0000830E386BDF80A302387BDF80C306387DF
:101CF00005B030BD1846FBE70368DB6B13B504463F
:101D00002BB923685B6B3BB9FF23E38202E0984762
:101D10000028F6D102B010BD214601A8984700283E
:101D2000F2D0BDF80630013B9BB2EEE7036810B578
:101D30009B680446984701236374FF23A37410BD76
:101D4000036810B504461B689847236820469B68C3
:101D50009847E37C0133E37410BD036810B5044673
:101D60005B689847236820469B689847E37C013B63
:101D7000E37410BDF0B5044685B00D46184616460E
:101D800003934EF03FFB226828440021E673A073C2
:101D900020460091294657693246039BB84705B053
:101DA000F0BD30B5046885B0E469089D34B10DB963
:101DB0000DF10F050095A04705B030BD2046FBE7AB
:101DC00003689B6A184738B58B68044601600D4666
:101DD00098470B4B2361002323752B6B13B12046CF
:101DE00098472075074B93F8EC3E1BB1237D23F0F9
:101DF0000103237500232046E382BDE838407BE7DA
:101E00000001FF001073012003681B6803B118472D
:101E1000704703685B6803B11847704703681B6A23
:101E200003B11847704703685B6A03B118477047EE
:101E300030B40468A46A14B1A44630BC604730BC16
:101E4000704730B40468E46A14B1A44630BC6047FB
:101E500030BC704703685B6C03B118477047036878
:101E60009B6C03B11847704703689B6F03B1184719
:101E700070470368D3F8803003B118477047036890
:101E8000D3F8843003B1184770470368D3F888301B
:101E900003B11847704721B10B68D3F88C3003B1F8
:101EA00018470020704710B5B0204FF48064FFF74A
:101EB000D0FA4020FFF7CDFA0020FFF7CAFA102031
:101EC000FFF7C7FA013C00204DF084F9A4B2002CC2
:101ED000F8D110BD503910B50446C8B2FFF7B9FAB1
:101EE00004EB440004EB4404400000F00E00FFF754
:101EF000B0FAC4F3C300BDE810401030FFF7A9BA30
:101F0000503808B5C0B2FFF7A4FA0020FFF7A1FAD5
:101F10001020BDE80840FFF79CBA38B50524094BEE
:101F200004FB0030A0F1A005013C15F8010B4DF0B9
:101F300051F914F0FF04F7D12046BDE838404DF0C8
:101F400049B900BFF47D060810B5441E14F8010F0E
:101F500000B910BDFFF7E1FFF8E738B500221E23F6
:101F600031210120FEF73DFC3C4BC3F8E80E10B9CF
:101F70000024204638BDAE20FFF76BFA0446002847
:101F8000F6D0D4204FF48065FFF763FA8020FFF786
:101F900060FAA820FFF75DFA3F20FFF75AFAD32036
:101FA000FFF757FA0020FFF754FA4020FFF751FAE5
:101FB0008D20FFF74EFA1420FFF74BFAA120FFF710
:101FC00048FAC820FFF745FADA20FFF742FA122054
:101FD000FFF73FFA8120FFF73CFACF20FFF739FAED
:101FE000D920FFF736FAF120FFF733FADB20FFF7AD
:101FF00030FA4020FFF72DFAA420FFF72AFAA62096
:10200000FFF727FAAF20FFF724FAA620FFF721FAFF
:10201000AE20FFF71EFA2020FFF71BFA0020FFF783
:1020200018FAB020FFF715FA4020FFF712FA002047
:10203000FFF70FFA1020FFF70CFA013D00204DF0DA
:10204000C9F8ADB2002DF8D18120FFF702FAC820FF
:10205000FFF7FFF9AF20FFF7FCF98AE710730120C3
:10206000FBF72EBDFBF72CBDFBF72ABDFBF728BD08
:10207000FBF726BDFBF724BDFBF722BD034BD3F8CE
:10208000F00E08B143681847704700BF1073012075
:102090000448D0F8F03E0BB11B6A184700F6F46014
:1020A000704700BF1073012030B500220624064B94
:1020B00004FB02F1CD5C854204D00132092AF7D13C
:1020C000002030BD5818FCE71482012038B5194DA6
:1020D0003622194C002105F6047054F0A1FD04F5D8
:1020E0001474236800209847C5F8F04EFFF7D0FF1E
:1020F0008368D3B104880320FFF7D6FFB8B9013C49
:102100000220A4B2FFF7D0FF50B9D5F83C3F082B0E
:102110000BD05A1C0948C5F83C2F062202FB0300CD
:1021200002238480037000234380012038BD44884B
:10213000E5E700BF107301209812012014820120EE
:1021400030B1006800F13F4000F57E00800A704722
:102150004FF0FF30704790F85F3230B53BB990F8E0
:102160005D12012490F85E32DAB2914200D830BD9F
:1021700004FA03F2B0F8665201332A43A0F866224B
:10218000F2E7437913F001031FBFD0E90732C068BB
:102190009B1A00F1FF3014BF18401846704743796E
:1021A00013F002031FBFD0E9093200699B1A00F146
:1021B000FF3014BF98431846704710B54379014665
:1021C00013F001030DD0FFF7DCFF60B10A6A4B6921
:1021D000C8689B5C0132B2FBF0F4DBB200FB142256
:1021E0000A62184610BD0346FBE743799B070AD5F0
:1021F000436A8269D154436A02690133B3FBF2F145
:1022000002FB11334362704741717047D0E90920E6
:10221000131A584258417047014B1B685B681847B6
:102220000C8C0120024B08301B689B68184700BFCC
:102230000C8C01200120704701207047012070475D
:102240000120704731B10C4BD3ED007AF8EEE77AFC
:10225000C1ED007A72B1094BDFED096A1B68A3F585
:10226000D543333B07EE903AF8EEE77A87EEA67A4D
:1022700082ED007A704700BF149401201894012069
:102280000000C8420120704701207047704700BF1E
:1022900040F2FF72034B914203EBC000A8BF11460E
:1022A00081807047E8A90120154B164A9B79032BC2
:1022B00082F860301AD9191F022914D8052B17D0BB
:1022C000062B14BF4FF47A614FF47A510E4B002065
:1022D000B3FBF1F39FED087B0C49D06682ED1C7BCC
:1022E000C2E9191370470A4B53667047094BFBE765
:1022F0004FF4FA51EAE700BF0000000000000000C0
:1023000088870120E8A9012040420F00912201089E
:102310008D220108D1310108034B03EB8000836F4C
:102320000BB19B6819607047E8A90120084AD2F8F0
:10233000B8305BB140B1B2F8BC00064A9968B2FB54
:10234000F0F35B100B6070479B681860704700BF2C
:10235000E8A9012040420F0007B50DF10702FFF781
:10236000A9F8034B18709DF8070003B05DF804FB53
:102370008416012008B5FEF791FE014B187008BDC8
:1023800084160120F8B5144E41F0010200210446E4
:10239000124FFFF7EFFF3568C7F8C05013212046F2
:1023A000FFF7DAFF10F007000BD001220B212046C7
:1023B000FFF7E0FF002220461146FFF7DBFF012078
:1023C00008E0D7F8C420002AE8D033689BB25B1B32
:1023D0009A42E3D2F8BD00BFE02E0120E8A9012017
:1023E0000C4A13787BB10C4B93F8C81059B193F891
:1023F000C91059B150680021FA2883F8C910A8BF44
:102400004FF0FF3070476FF0010070476FF002002F
:10241000704700BF84160120E8A901200B4B93F8F8
:10242000CA206AB193F8CB206AB1002283F8CB208E
:10243000074B9868B0F5967FA8BF4FF0FF30704704
:102440006FF0010070476FF002007047E8A90120AB
:1024500084160120014B1B685B681847008C012023
:10246000014B1B689B681847008C0120014B1B68BF
:10247000DB681847008C0120014BD868704700BF0B
:1024800084160120044B93F8CC3013B1034B186928
:1024900070476FF001007047E8A901208416012001
:1024A00020B10078B0FA80F04009704701207047F1
:1024B0002DE9F04F944D0024A7B04FF00A0E05F11E
:1024C000D00C95F8143120462746664605F5867AE5
:1024D00099E002EBC70205EB4201D7B2B1F818410F
:1024E000C2F30721660701914FEA142BE1B240F1D4
:1024F000BE805C0613D400F1020843F04003B8F13B
:102500008C0F00F2F18026AE441C30444FF00406DC
:1025100000F88C6C26A80444404604F88C3C00F17A
:102520000208019CB8F18C0F44F0020900F2DC8033
:1025300026AC044404F88B9C4FF0050904F88C9CED
:1025400000F10409B9F18C0F00F2CE8026AE8900AB
:10255000B0444FF00606C9B208F88C6C00F10608CA
:1025600004F8897CB8F18C0F00F2BE8026AEB1442D
:102570004FF0070609F88C6C04F8871C00F108017D
:102580008C2900F2B18026AE4FF00509B044019EBF
:1025900008F88C9C04F8856C00F10A068C2E00F279
:1025A000A3800DF198094FF00608494401F88C8C7E
:1025B00000F10C0104F8837C8C2900F295804FF027
:1025C00007044E440B3006F88C4C4C46204400F86F
:1025D0008CBC08465609012102F01F04BEF1010E11
:1025E00001FA04F45CF8261021EA04014CF82610E4
:1025F0007DD0541CB4F5F07F79D262090CEB8206D1
:102600009700564573D24FF0FF3204F01F04316833
:1026100002FA04F404EA010292FAA2F2B2FA82F295
:10262000D2B2202A7FF455AF311D514518D2374A16
:10263000921B083622F00302164401E0B1420FD08B
:102640000C460431226892FAA2F2B2FA82F2D2B2B5
:10265000202AF3D0A4EB0C0412EBC4027FF53BAFAD
:1026600085F81431002844D127B0BDE8F08F5E060C
:1026700003D403F03808884512D023F078032343AD
:10268000841C8C2CDBB22FD826AE411C30444FF07A
:10269000040600F88C6C26A80144204601F88C3C06
:1026A000811C8C2920D826AC019E044404F88B6C34
:1026B0004FF0050604F88C6C061D8C2E14D80DF115
:1026C000980841444FF0060801F88C8C811D04F8ED
:1026D000897C8C2908D826AC053026444FF00704A5
:1026E00006F88C4C26AC71E76FF0004072E785F875
:1026F0001431034603AAD5F80C0100214CF01AFE50
:10270000012027B0BDE8F08FE8A90120EFAA012041
:10271000624B2DE9F04F93F81251C7B005B1FEE7B7
:102720005E4A012304460E4692F8137182F8123174
:1027300007F0F707D2F80C3182F8137103931B7975
:10274000012B00F09A80022B40F0958003983A46C6
:10275000836813F0010118BF294605ADFEF77BFC25
:102760004E4BD3F80C310393FF2C4FF009036C70E0
:102770004FF002008CBFA4084FF000084FF0000C8F
:102780004FF00A0988BF04F0C0080DF1150A4FF098
:102790000B0B2B7011E0BEF5827F05F8009016F848
:1027A0000C700AF8002016D80CF1010C05F804B0E2
:1027B00070466F54BCF1360F16D0841C48EA0C02E8
:1027C000034600F1040EB4F5827FD2B200F103019A
:1027D00003F10603DFD90CF1010C6FF0004E304B12
:1027E000BCF1360F7046E8D1B3F5827F0DF11304CA
:1027F0009DBF08230DF11502A0216FF000439EBF7D
:1028000005F80E30831C11542A46039800214CF021
:1028100091FD224B234DD3F80C010379012B18D0E5
:10282000022B0CD12246A021FEF71EFE18B1237800
:1028300013F0200319D0194BD3F80C010379D5F804
:10284000A810012BB5F8AC204E6982EA06024A6155
:10285000E6D18668A022417C06F0010690F91000BE
:10286000CDE90046F8F72CFDE0E70C4A82F812317A
:1028700047B0BDE8F08F05AD76E703982A4681683A
:1028800001F00105014690F91000497C019505AD64
:102890002F700095F8F750FB62E700BFE8A9012010
:1028A0000100008050820120C36B59680A68487992
:1028B0000349136A51F820100B431362704700BF9D
:1028C0008C830608836837B51C686379DB0727D5D6
:1028D000A57994F85C3205F001010D4613B3E06B65
:1028E00003685B681A68D36A5B08536294F86D32B8
:1028F000012B07D094F8613223B1B4F86832013368
:10290000A4F8683285F001014AF0ECFB2046FFF79D
:10291000CBFF0023A4F866324FF08073C4F85C321A
:1029200003B030BD94F85F3220460191012B04BF03
:1029300094F85D3284F85E32FFF70DFC94F85F3254
:10294000019963B9012385EA030184F85F32E06BE2
:102950004AF0C8FB204603B0BDE83040A4E700239E
:1029600084F85F32F3E738B50D4603201446FDF7CF
:10297000E3FE07EE900A8DB1F8EE677A9FED097AD3
:10298000F0EE006A67EE877AB8EE047AA7EEA67AD0
:10299000DFED057A67EE277AC5ED007A0CB1034BBF
:1029A000236038BD6740533A00007A4433139043A4
:1029B00007B5012301AAFF210068FEF72BFA03B037
:1029C0005DF804FB07B5022301AAFEF723FA044BC6
:1029D0001870BDF8040040BA80B203B05DF804FB83
:1029E0008416012070B53B4C054694F8C830002B86
:1029F00036D094F8D864012E33D0022E4FD07EBB4F
:102A0000012280210068FFF7B5FC0122FF21286820
:102A1000FFF7B0FC324631462868FFF7ABFC94F86C
:102A2000D92491212868FFF7A5FC012231462868A6
:102A3000FFF7A0FC3246FF212868FFF79BFC3246D7
:102A400080212868FFF796FC012231462868FFF7AD
:102A500091FC214B1B68C4F8C030012384F8D834A2
:102A600070BD00210068FFF777FCC20711D5D4F8CC
:102A7000C420002AF4D0184BD4F8C0101B689BB2B5
:102A80005B1A9A42ECD2154B4FF0FF325A6000238A
:102A9000E4E7114B1B68C4F8C0300223DEE71321C2
:102AA0000068FFF759FC4307E1D01E212868FFF7B3
:102AB00089FF012206460B212868FFF75BFC0A20EC
:102AC000064BB6FBF0F6B6B25E60012384F8C9305F
:102AD000DDE700BFE8A90120E02E012084160120D7
:102AE00007B5022301AA00210068FEF793F90F4BF6
:102AF00083F8CC0050B1BDF804300D4A5BBA9BB2EC
:102B0000B3F5FA6F05D34FF0FF33136103B05DF8EF
:102B100004FB0A21B3FBF1F307EE903AF8EEE77AF3
:102B2000FDEEE77AC2ED047AF0E700BFE8A90120E4
:102B30008416012013B502230C4601AA0021006867
:102B4000FEF768F960B15CB19DF805309DF904208D
:102B5000DB0902EB820203EB830303EB42032380D6
:102B600002B010BDF7B505460068FEF7A9F80023CE
:102B70000446FF210370042328680DEB0302FEF7CF
:102B800049F910B9002003B0F0BD04236A46FF21C3
:102B90002868FEF73FF90028F4D09DF804108A0950
:102BA000023A012AEED99DF800209DF805309DF8E3
:102BB000015003EB012305EB0225C3F30D03C5F31D
:102BC0000D055A1B002AB8BF5242FF2ADADC9DF8D5
:102BD00006109DF807209DF8027002EB01229DF877
:102BE000031001EB072156114911C1EB5212002AC3
:102BF000B8BF5242FF2AC5DC01222B4431441341A5
:102C000022701141C4F80530C4F80110BBE738B593
:102C100000680D461446FEF753F8D0F8013007EE71
:102C2000103ACDB1D0F80530DFED166A07EE903AD4
:102C30009FED156AF8EE677A77EEE67A77EEA77A77
:102C4000C7EE866AF7EE007A76EEE77ADFED0F6A76
:102C500067EEE67AC5ED007A9CB1B8EEC77ADFED93
:102C60000C7ADFED0C6A27EE277AC7EE267A9FED05
:102C70000A7A77EEC77A9FED097A77EE877AC4ED04
:102C8000007A38BD9AC9CC449AC94C460E76D745CD
:102C90000000484300E0FF4400004842339388436B
:102CA0003B4BF0B52DED028B1B7E83B00E461546D7
:102CB000022B69D1374B384C1B6894F8DA2403F0A7
:102CC0000203002A45D0002B59D0344F0DF10600E5
:102CD0001EF08CF8BDF80630D7F8E823F0EE408AF5
:102CE0009FED2F7A04F2DC449B1A07EE903AF8EE3F
:102CF000E77A87EE870ADFED2B7A20EE270AFBF7CB
:102D000049FE97EDFF8AA0EE688A3AF0C3FDD4ED44
:102D1000020AD0ED057A70EEA70AB0EE480AFCF779
:102D200087FE7EB120EE000ADFED1F7A9FED1F7A4D
:102D300020EE270AC0EE077A9FED1D7A77EE877A9C
:102D4000C6ED007A0DB11B4B2B6003B0BDEC028BBE
:102D5000F0BDA3B1B4F90A3501EE103AB4F9083563
:102D600000EE903AB4F90635B8EEC11A00EE103A0A
:102D7000F8EEE00AB8EEC00AFCF762FED1E7D4F83C
:102D8000203593ED350ACCE79FED0B0AC9E700BF6C
:102D9000008A012008000020E8A9012050990120A4
:102DA0000000C84235FA8E3CCDCC9C3F00409C468A
:102DB00082E6C54733139043000000002DE9F04F31
:102DC0008DB0CDE90223BDF858309DF85CB001907C
:102DD00005910493F8F740FD0646002800F0AC800A
:102DE0005B4F97F82455072D00F2AB805C234FF022
:102DF000000A05EB45096C1C03FB0573C5EBC90212
:102E000007F5A569C3F828A5E4B283F82CA509EB5A
:102E10008209019B87F824451B794FEA131803F0B8
:102E20000F0308F1FF38B8F1030F40D8494A32F8D0
:102E3000180040FA03F2D20739D5012202FA03F34F
:102E4000013B18404EF038F9434B02219844059B52
:102E500098F810201044414A00EB400002EB800833
:102E600088F8084000FA01F488F8063088F807105E
:102E7000BBF1000F46D1384B4046FFF761F91844CB
:102E8000007D4AF053FBB8F80430344A07A9079391
:102E9000112310590893CDF82CB0CDE909BBF7F7F1
:102EA000B3F8B8F804302D4A1B04A25893615C2390
:102EB0003046012403FB0575DDE90221C5F82865CC
:102EC000F8F772FD0499D5F82805F8F7FBFDD5F859
:102ED0002805F8F747FFD5F82805022203685B6844
:102EE000196883F83D200A6822430A6083F83D4050
:102EF000F8F722FF0023C5F83005036048460DB0FF
:102F0000BDE8F08F019B4046FFF71AF993F808B02F
:102F1000114B1844007D4AF009FB104A0221B8F811
:102F200004301059089107A9CDF82CB00793CDE9CA
:102F300009AAF7F769F8BAE7814648460DB0BDE837
:102F4000F08F0021064A04208946FCF7FBFDD5E7F7
:102F5000E8A90120988006088C8306085082012089
:102F6000300E07082DE9F0437E4D83B00C46134622
:102F700095F860C0BCF1060F00F2EF80DFE80CF0BE
:102F80002DBA629204040400BCF1050F00F0D98050
:102F9000754A7649BCF1060F08BF0A464FF0000992
:102FA000019302211423CDF80090FFF707FF074695
:102FB000002800F0D0808046122258F8140B4146B9
:102FC0004CF058FF0646002840F0BD80012645F829
:102FD0003470304603B0BDE8F083654A00210193A8
:102FE000644B16684FF6FF720091A3FB067102EB6B
:102FF000D1120221120CB6FBF2F6A3FB06233246D5
:10300000C3F3CF13FFF7DAFE98B107EE906A9FED96
:103010005A7ADFED5A6A0123F8EE677A67EE877A0B
:1030200027EE877A0371E7EE667A80ED047AC0EDC9
:10303000037A061E45F8340018BF0126304603B057
:10304000BDE8F0834A4A002101934D4B16684FF6C4
:10305000FF720091A3FB067102EBD1120221120C48
:10306000B6FBF2F6A3FB06233246C3F3CF13FFF7FA
:10307000A5FE0028DDD007EE906ADFED426A9FEDE5
:103080003F7A0123F8EE677A9FED3F6A037167EE9E
:10309000A66A27EE667AC0ED046AA7EE867A80ED0E
:1030A000037AC6E701930026384B4FF6FF71304A8A
:1030B0009B8812680096B2FBF3F63144090CB2FB10
:1030C000F1F2B2FBF3F60221B3B2FFF777FE00286C
:1030D000AFD007EE906ADFED286A9FED287A0123D2
:1030E000F8EE677A037167EEA67A27EE677AC0ED8D
:1030F000047AD4E71E4A00210193214B16684FF64B
:10310000FF720091A3FB067102EB91120221120CD7
:10311000B6FBF2F6A3FB06233246C3F38F13FFF789
:103120004DFE002885D007EE906A9FED196A9FED4D
:10313000127A0123F8EE677ADFED106A67EE867A7D
:103140006EE7144A2AE749464046482253F068FD94
:1031500001233B713BE7064639E700231E4645F84D
:10316000313036E7E8A90120C0C62D00001BB700AA
:10317000BC0101201F85EB516F12833A00007A4495
:10318000D34D621077CCAB32ACC5A736888701200F
:103190006F120339808D5B0010B582B00A4C00932A
:1031A0009DF810300193B4FBF2F322469BB20C461B
:1031B0000321FFF703FE034620B10449012001EB80
:1031C00084018B6702B010BD40420F00E8A90120C6
:1031D0000B4B10B553F8304082B001916CB107EE43
:1031E000901A94ED047A94ED030AF8EEE77AA7EECC
:1031F000870A50F0F7FBA368186002B010BD00BF4B
:10320000E8A9012010B5C04C04EB80039B6F0BB103
:103210009B6819600F2822D8DFE810F022003100E7
:10322000480063007A009100AC00C300D500E400C0
:10323000FB0016012D0144015F011000084623F038
:1032400069FC94F81D3800F00702C0F3C70003F0D2
:103250001F0384F81E0843EA421384F81D3810BD8A
:10326000084623F057FC94F80A38C0F3022284F889
:10327000090823F00703134384F80A3810BD0846F1
:1032800023F048FC94F80A2894F80B3800F01F014A
:1032900002F00702C0F3451023F03F0342EAC102E7
:1032A000184384F80A2884F80B0810BD084623F058
:1032B00031FC94F80B2800F0030194F80D3802F06B
:1032C0003F0223F0010342EA8112C0F38021C0F3E0
:1032D00087000B4384F80B2884F80C0884F80D3819
:1032E00010BD084623F016FC94F80D2894F80E380B
:1032F00000F07F0102F00102C0F3C31023F00F03BE
:1033000042EA4102184384F80D2884F80E0810BDE3
:10331000084623F0FFFB94F80E2894F80F3800F0CD
:103320000F0102F00F02C0F3061023F07F0342EA00
:103330000112184384F80E2884F80F0810BD0846BF
:1033400023F0E8FB94F80F2800F0010194F81138FD
:1033500002F07F0223F0030342EAC112C0F34121CD
:10336000C0F347000B4384F80F2884F8100884F852
:10337000113810BD084623F0CDFB94F8112894F8BD
:10338000123800F03F0102F00302C0F3841023F072
:103390001F0342EA8102184384F8112884F81208B6
:1033A00010BD084623F0B6FB94F8123800F007026F
:1033B000C0F3C70003F01F0384F8130843EA421365
:1033C00084F8123810BD084623F0A4FB94F8153891
:1033D000C0F3022284F8140823F00703134384F88F
:1033E000153810BD084623F095FB94F8152894F87D
:1033F000163800F01F0102F00702C0F3451023F059
:103400003F0342EAC102184384F8152884F81608DD
:1034100010BD084623F07EFB94F8162800F0030147
:1034200094F8183802F03F0223F0010342EA8112B7
:10343000C0F38021C0F387000B4384F8162884F87A
:10344000170884F8183810BD084623F063FB94F879
:10345000182894F8193800F07F0102F00102C0F337
:10346000C31023F00F0342EA4102184384F81828DE
:1034700084F8190810BD084623F04CFB94F819286D
:1034800094F81A3800F00F0102F00F02C0F3061092
:1034900023F07F0342EA0112184384F8192884F8C4
:1034A0001A0810BD084623F035FB94F81A2800F0DE
:1034B000010194F81C3802F07F0223F0030342EA72
:1034C000C112C0F34121C0F347000B4384F81A280E
:1034D00084F81B0884F81C3810BD084623F01AFB3A
:1034E00094F81C2894F81D3800F03F0102F0030204
:1034F000C0F3841023F01F0342EA8102184384F8CA
:103500001C2884F81D0810BDE8A9012010B5094C3D
:1035100094F82C38012B05D0022B07D0064BC4F8A9
:10352000303810BD4BF0ACFB044BF8E74BF0A8FB78
:10353000034BF4E7E8A9012019230108BDD10208D3
:103540000532010810B50023094C84F834380323F0
:1035500084F83518FF2184F8362804F63402FDF784
:1035600013FC00280CBF6FF00C00002010BD00BF42
:10357000E8A90120F8B5124D00241646022305F6ED
:10358000340285F83518FF21074685F83448FDF7E1
:10359000FBFB05F6340210B96FF00C00F8BD0223F6
:1035A000FF213846FDF736FC0028F5D095F8342881
:1035B000204695F8353803EB02233380EEE700BF51
:1035C000E8A901200023024A51210068FDF7DCBB75
:1035D0001CB3012013B5022301AA0446512100683F
:1035E000FDF718FC114AF0B1BDF804305BBA9BB28C
:1035F000D360D368B3F5C87F02DD4FF0FF33D360EB
:103600000B4B0C4A1968D2F8343932338B4208D24A
:10361000C2F83419002302F6341251212068FDF754
:10362000B3FB02B010BD6FF00103E8E78416012080
:10363000E02E0120E8A9012037B5124D044695F887
:10364000CA30E3B10DF1050100684BF028FD9DF88B
:1036500005307BB10DF1060296212068FFF78AFF45
:103660000A22BDF80630B3FBF2F3074A9360012348
:1036700085F8CB30012286212068FFF763FF03B075
:1036800030BD00BFE8A9012084160120FDF78CB8E9
:103690000FB413B504AB094C094953F8042BD4F803
:1036A0003809019349F0BAFDD4F83809FDF770F8EC
:1036B00002B0BDE8104004B0704700BFE8A9012087
:1036C0008D360108202108B553F077FB034618B169
:1036D0001A780130202AF9D0184608BD2DE9F041AA
:1036E0000D461646044600274FF019082046FFF7FE
:1036F000E9FF044690B1FCF703FF40F634024FF4B3
:103700006171FBF7C5FBA0F5617090FBF8F0302804
:1037100004D84FB9287033780133337017B120467D
:10372000BDE8F0810127E1E76870F4E737B50546A9
:10373000084601914CF066FE01990446024628466F
:10374000FCF77AFB68B92B5DA3F13002092A06D990
:1037500023F02003413B192B01D90134281903B070
:1037600030BD0020FBE730B1036882881B691A4234
:1037700014BF01200020704718B10268838809B186
:10378000936170471B04FBE710B1036882889A615C
:10379000704718B1838802681B049361704730B585
:1037A0000C4687B00546B8B10C4BFEF7C9FC18446F
:1037B000007D49F0BBFE002301A928680593AB8872
:1037C000019304F013030293C4F34113C4F381047F
:1037D00003930494F6F718FC07B030BD8C830608F9
:1037E00070B50C4686B016460546A8B10B4BFEF7E1
:1037F000A7FC1844007D49F099FEAB8801A9286810
:10380000019304F0130302936309C4F38104039347
:10381000CDE90446F6F7F8FB06B070BD8C830608C8
:1038200010B5040900F00F02013C032C18D80D4B11
:1038300033F8141041FA02F313F001000FD0012302
:1038400003FA02F2013A02EA01004DF035FC064AA1
:1038500014440C22237C1844044B02FB003010BD9E
:103860000020FCE7988006088C830608508201201F
:10387000054B03EB8000C26922B111689388486947
:1038800043404B61704700BF8C830608034B81F0B7
:10389000010103EB8000C0696EE700BF8C8306085E
:1038A0002DE9F84F6A4FD7F83C09037C03F0FF0C71
:1038B000002B40F0CB8097F8422907F6461E97F878
:1038C0004339E24697F844993C25A7F840C99EF849
:1038D00002109EF80360C1F1FF0189B2002900F0D7
:1038E000B180BEF80040C1F1FF01B4FBF5FB7143AC
:1038F0000912BBF1050F22D8DFE80BF0030E637449
:103900008593731A5FFA81F96343B3FBF5F353FAB6
:1039100081F3DBB2324610E0B4FBF5F205FB124254
:10392000741A5FFA81F992B2C2F13C026243B2FBAF
:10393000F5F252FA81F2D2B233464FF0010A160282
:10394000002146EA034646EA09064FF00108C1F1A4
:10395000170B0CEB010408FA0BFB4144A4B21BEA61
:10396000060F07EB840414BF4FF0020BC34618295F
:10397000C4F8C8B9E9D10CF1180C0EF1040E1FFA05
:103980008CFCBCF5407FA2D13249A1F878C5BAF1D0
:10399000000F05D087F8422987F8433987F8449902
:1039A0002023A7F8403991F87A35002B4ED040F209
:1039B0002A31F8F7E9F9D7F83C09BDE8F84FF8F7EC
:1039C00039BAB4FBF5F305FB1344A6EB0109CAB2FF
:1039D000A4B204FB09F9B9FBF5F959FA81F15FFAD0
:1039E00081F9A9E7B4FBF5F305FB1343741ACAB2D6
:1039F0009BB2C3F13C036343B3FBF5F353FA81F38A
:103A0000DBB2B14699E7B4FBF5F905FB1944721A2C
:103A1000CBB2A4B26243B2FBF5F252FA81F2D2B257
:103A2000EFE7B4FBF5F205FB1242741ACBB292B287
:103A3000C2F13C026243B2FBF5F252FA81F25FFA44
:103A400082F967E7B1463346324676E7BDE8F88F3C
:103A5000E8A90120E0BA0120F8B500211820F7F705
:103A60008BFF054650B31C4FF7F7F6FE0446C7F828
:103A70003C0918B3194E1820FFF7D2FEC6F87C0592
:103A800020B14FF40573C380002303722A7A4E21BC
:103A9000FFF7A6FE124A03212046F7F785FF002113
:103AA000D7F83C09F8F70EF840F22A320D49D7F85A
:103AB0003C094CF0DFF910B986F87A05F8BD40F6FC
:103AC000A8420021074853F0ABF8012386F87A3565
:103AD000BDE8F840E4E600BFE8A90120E0BA012013
:103AE000009F2400B0B30120084B93F811214AB184
:103AF00093F8133113F0400F14BF4FF4F0704FF4EC
:103B0000C37070474FF4F070704700BFE8A9012000
:103B1000054B93F8110130B193F8133113F0400FB6
:103B20000CBF0D2010207047E8A90120F0B5564CBD
:103B30008DB005461023002228210220FCF751FEFB
:103B4000C4F80C01002800F090800221FCF7C8FFA7
:103B500002220021D4F80C01FDF7A0FA002104F59F
:103B60008C7304F59B6284F814114FF0202184F8C3
:103B7000105143F8041B9342FBD1444E444F356827
:103B80003235D4F80C010379012B70D0022B0ED101
:103B9000836880213E4ADB075CBF3D4A8021FDF7F8
:103BA00063FC10B133689D42EBD8D4F80C011024AB
:103BB0001123122113224FF0140E15271626172554
:103BC0008DF80C4018248DF80E3019238DF8101044
:103BD0001A218DF812201B224FF0010C8DF814E0F1
:103BE0008DF816704FF01C0E8DF818601D278DF89B
:103BF0001A501E268DF81C401F254C248DF81E30AF
:103C00008DF8201022238DF82220002103AA8DF8A0
:103C10000DC08DF80FC08DF811C08DF813C08DF850
:103C200015C08DF817C08DF819C08DF81BC08DF820
:103C30001DC08DF81FC08DF821C08DF823C08DF8F0
:103C400024E08DF825C08DF826708DF827C08DF8FA
:103C500028608DF829C08DF82A508DF82BC08DF87A
:103C60002CC08DF82D404BF065FB0DB0F0BD826887
:103C7000417C02F0010C90F910008022CDE9007C1B
:103C8000F7F71EFB8DE700BFE8A90120E02E012019
:103C9000FBAA01200F4A002370B54FF400560124FF
:103CA00002F5707EA2F1460532F8020F4FEA531C6E
:103CB00003F01F010133B0F5005F04FA01F11FBFEB
:103CC00055F82C001680014345F82C107245EBD1B5
:103CD00070BD00BFFEAA01204FF01E0C43EA022374
:103CE000FF2A0CFB01011BB288BF43F00403B1F5AE
:103CF000F07F07DA0C4A9BB202EB4100B0F818C122
:103D00009C4500D170474FEA511CD032A0F81831C1
:103D100001F01F01012052F82C3000FA01F10B4391
:103D200042F82C30704700BFE8A901204FF01E0C6C
:103D30000CFB0101B1F5F07F01DB002070470B485F
:103D400000EB4101B1F81811080AC9B210801970CE
:103D5000490709D51188012041F4807111801A7832
:103D600022F004021A70704701207047E8A9012070
:103D70002DE9F0471E2404FB010114787CB31D28B3
:103D80002DDC184E0FFA83FEC1F10105012706EB69
:103D9000410C483E02E003441D2B20DCB1F5F07FCE
:103DA0004EEA042405EB010311D2BCF800A04FEA4F
:103DB000511901F01F08A24507FA08F81FBFACF817
:103DC000004056F8294044EA080446F8294012F811
:103DD000014F0CF1020CDBB20131002CDBD1BDE84C
:103DE000F08700BF00AB0120F0B54F4C85B0D4F890
:103DF0000C5115B194F812310BB105B0F0BD01238F
:103E000084F812312B79012B78D0022B35D128463A
:103E10000DF10E028421FDF727FBD4F80C5194F824
:103E200014212B7942F00402012B75D18DF80F205B
:103E3000AA6895F9100002F00102697C01920DF167
:103E40000F0200920422F7F777F813E0022B0CD14F
:103E5000AB680DF10E0284212846DB075EBF0DF131
:103E60000E0284212846FDF7FFFA9DF80E3013F06C
:103E7000040616D0D4F80C512B79012BE6D1AA6890
:103E8000697C95F9100002F001020DF10E05CDE9F3
:103E900000528422F7F714FA9DF80E3013F004064E
:103EA000E8D1224D31463C22214884F814310127C3
:103EB00052F0B6FE3146A5F1460E05F5707635F89E
:103EC000023F4FEA511C01F01F0001311A0A03F0B2
:103ED000040307FA00F022F0200213431EBF5EF82D
:103EE0002C3018434EF82C00B542E8D1FEF7E0FA2A
:103EF0000028FBD184F8120105B0F0BDAA68697CE6
:103F000002F0010295F9100001920DF10E020092EB
:103F10008422F7F7D5F980E7022BAED12846042199
:103F2000FDF799F8A6E700BFE8A90120FEAA012045
:103F3000B8AA012010B52D4C84B0D4F80C01E8B11A
:103F400094F81031012B32D0022B19D1082204230E
:103F5000002184F813218DF80D2003AA8DF80E306E
:103F60008DF80F308DF80C104BF0E4F93C22FF2156
:103F70001F4852F055FE94F81131D3B104B010BD72
:103F80000379012B22D0022B1AD09DF80B3003F0BD
:103F90000503012B09D013B9D4F80C01D6E7154A53
:103FA00040F2DC5312689A42E8D9D4F80C01482256
:103FB000CDE7FFF719FF012384F8113104B010BDDC
:103FC0000DF10B02A021FDF74FFADEE78268417C7C
:103FD00002F0010290F910C001920DF10B0260464F
:103FE0000092A022F7F76CF9CFE700BFE8A9012003
:103FF000B8AA0120E02E0120F0B53E4C85B0D4F8DF
:104000000C5195B194F81331180702D594F8123178
:104010006BB194F8113143B9FFF78CFF94F811316B
:10402000002B3BD1002384F8123105B0F0BD0122F2
:1040300094F8113184F81221002BEDD02B79012B4B
:104040002FD0022BE8D10DF10E0280212846FDF77A
:104050000BFA0028E0D094F813219DF80E309A4214
:10406000DAD194F81051002DD8D1234B234E1F687C
:10407000D6F88035FB1AB3F57A7FCFD9A0210DF1A0
:104080000F02D4F80C01FDF715FA9DF80F3059070F
:1040900015D5C6F88455C6F88075BFE7FEF708FA4F
:1040A000C0E7AA68697C02F0010295F9100001924C
:1040B0000DF10E0200928022F7F702F9C9E703F032
:1040C0000503012B0ED0002BE5D194F813315B06CC
:1040D000E1D5D6F8843553B1FB1A642BDBD9FFF751
:1040E00029FFD8E794F813315A06F2D5D3E7C6F87A
:1040F0008475D0E7E8A90120E02E0120E0BA012074
:104100002DE9F0438D4E85B0D6F80C41002C6DD0D2
:1041100096F81291B9F1000F00D0FEE796F813C19E
:10412000012305460F460CF0F70C86F8123186F88D
:1041300013C12379012B00F0DD80022B00F0978062
:104140000DF10F08B5F5807F00F0B2802379012BC7
:1041500000F0B980022B07D1204650220821FCF73D
:104160007AFFD6F80C412379012B754D19D0022B1B
:104170000DD142462046A021FDF776F920B19DF8E9
:104180000F4014F0200450D0D6F80C412379D5F814
:10419000A810012BB5F8AC20486982EA00024A61F8
:1041A000E5D1A268617C02F0010294F91000CDE92A
:1041B0000082A022F7F784F8E0E7B9F1000F12D1EE
:1041C00096F81341D6F80C5104F0F70486F8134121
:1041D0002B79012B00F0A380022B04D12246494603
:1041E0002846FCF738FF002386F8123105B0BDE8F9
:1041F000F083022B16D162460A212846FCF72BFFDA
:10420000D6F80C0107EB040C0379012B28D1856843
:10421000C022417C05F0010590F91000CDE900C5F0
:10422000F7F74EF80134362CC7D0D6F80C515FFAA8
:1042300084FC2B79012BDCD1AA6895F91000697CEC
:1042400002F001050A228DF80FC0CDE90085F6F7CE
:1042500073FED6F80C0107EB040C0379012BD6D0C2
:10426000022BDFD16246C021FDF7FEF8DAE74946AE
:10427000204662460DF10F08FCF7EDFED6F80C4122
:1042800081462379EAB2012B2CD1A16894F9100060
:1042900001F0010C617C8DF80F200922CDE9008C22
:1042A000F6F74AFEB5F5807FD6F80C417FF44EAFA5
:1042B000204640220A21FCF7F1FED6F80C41237972
:1042C000012B7FF447AFA26894F9100002F00102BD
:1042D000617CCDE9008250228DF80F200822F6F78C
:1042E0002BFE3EE7022B7FF42DAF20460921FCF781
:1042F000B2FED7E7A1680DF10F0894F910004A4605
:1043000001F0010E617CCDF80080CDF804E08DF85D
:104310000FC0F6F711FED6F80C418146B1E7A96847
:104320004A4695F9100001F00107697C8DF80F40AD
:10433000CDE90087F6F700FE55E700BFE8A90120A8
:1043400050820120034BD3F80C310BB1FEF7E0B9DA
:10435000704700BFE8A901208379806BDB0748BF65
:1043600081F0010109B1FFF70FBAFFF712BA10B5DA
:104370008379044613F0010F03F02002C36B13D0BE
:10438000002A5B6818BF02211A7A08BF4221606BBD
:10439000FFF726FA0123204684F86032A4F85C3245
:1043A000BDE81040FEF780BA002A5B6818BF022102
:1043B0001A7A08BF2221EAE7036C806B23B15B689D
:1043C00001211A7AFFF70CBA0121FFF7E8B98368D7
:1043D00070B51C6863799A0731D594F86152D5B1EC
:1043E00094F962329BB1B4F8641220464B0801F094
:1043F0000101A4F86432FFF7AFFF94F86232A279AA
:10440000013B50065BB284F8623218D5BBB9002379
:1044100084F8613213E0A36A626A94F860129A42E7
:1044200027D161B9A3791B0709D5236CA06BE3B130
:104430005B681A7AFFF7D4F92046FFF798FF637993
:10444000D90740F1868094F85C32002B40F08180DF
:1044500094F85D320133DBB2092B84F85D323AD136
:104460002046BDE87040FDF776BE1946FFF797F984
:10447000E2E75A1CA0692669A262C35CB24234BF5B
:10448000104628465B00A06243F40073A4F864322F
:104490000A2384F86232012384F86132B9B1A37926
:1044A0001E0714D5E36B2B485B6819685E790A6AAE
:1044B00050F8260022EA0002606B0A6229461A7A46
:1044C000FFF78EF9204684F86052FFF775FFA37955
:1044D0005D0685D4B3E70A2B3BD194F85F322BB944
:1044E000B4F8663243F00103A4F86632B4F8660209
:1044F000820501D4C30719D4B4F86A320133A4F891
:104500006A320123A4F85C3294F85F32012B20D187
:10451000A1790023E06B84F85F3201F0010148F0DB
:10452000E1FD2046BDE87040FEF7BEB9E36AC0F386
:10453000470013B1216B9847E3E7E3696269D05400
:10454000E369E2680133B3FBF2F102FB1133E3618B
:10455000D7E770BD8C8306081D4B1A6810B513464B
:104560000446B3FBF1F0B0F5803F03D3012BFAD939
:104570005B08F6E781B22046F7F716FA23681B6856
:10458000587948B140B2032149F0C8F823681B6844
:1045900093F90500F5F72AFD23681B68987948B15F
:1045A00040B2032149F0BAF823681B6893F906006A
:1045B000F5F71CFD236802225B68196883F83D202B
:1045C0000A6842F001020A60012283F83D2010BD12
:1045D000BC0101208160C06BBEE7002A4FF0200CB7
:1045E000BCBF80185242002BBCBFC9185B420028D8
:1045F000BCBF121A00200029F0B500EB020501EB48
:104600000304B8BF00210F4EA5F11D05B8BF234616
:104610000F3C3C27002DC8BF521B002CC8BF1B1BE2
:1046200002440B4490420CDC06EB40050C4604E0CF
:1046300007FB04FE013425F80EC09C42F8DD013072
:10464000F0E7F0BD00AB0120014B53F820007047AC
:1046500050280040014B43F820107047502800407C
:104660001A4B07B51A6C1A4942F080521A641A6C38
:1046700002F080520192019A0A6842F480720A6044
:10468000FF211A6C42F480621A641A6C02F4806290
:104690000092009A0F4A5162CA215162532151621D
:1046A0005B6FDB0005D50020FFF7CEFF0A4B984279
:1046B00009D000210120FFF7CDFF0749002003B0FA
:1046C0005DF804EBC6E703B05DF804FB0038024078
:1046D000007000400028004076614E692DE9F74FD8
:1046E0000026054688466A4C3746DFF8B0A1C0E987
:1046F000006614F0EFFE81469AF80630022B29D1AD
:10470000E3685A0742BF23F0040343F00803E36061
:10471000E368980604D523F0200343F04003E360E8
:10472000012001A9F7F72CFD01201DF0DDF838B3B9
:1047300023799DF805209A421ED13346554A01211E
:104740000420FBF7FFF9013614340B2ED4D103B04B
:10475000BDE8F08F012BE3D1E368190742BF23F0D6
:10476000080343F00403E360E3685A06D8D523F056
:10477000400343F02003D2E79DF804209A42DCD0A6
:10478000022001A9F7F7FCFC02201DF0ADF840B1B2
:1047900023799DF805209A42CFD09DF804209A42B3
:1047A000CBD0032001A9F7F7EBFC03201DF09CF808
:1047B00040B123799DF805209A42BED09DF804208F
:1047C0009A42BAD0052001A9F7F7DAFC05201DF0BE
:1047D0008BF840B123799DF805209A42ADD09DF821
:1047E00004209A42A9D02C4BD3F800B01BF0400F04
:1047F00008D000211220F7F7BFF818B1026823682B
:104800009A429AD01BF4803F08D000211820F7F775
:10481000B3F818B1226803689A428ED02379A3F1C5
:104820003002022A89D9142B87D09AF80120E36834
:104830000AB1032A1AD1580722D5B94524D923F041
:1048400008030137E360FFB2B8F1000F02D0E3685C
:10485000190710D4E36813F0040F3FF474AF2B680A
:104860005A1C02332A6045F823406CE75A0602D4EA
:1048700013F0200FF1E76B685A1C0A336A60F2E705
:10488000B8F1000FE3D15EE7B8F1000FE7D0DEE743
:104890000C0401206B0E070804000020C0910120C9
:1048A000F7B5054614F016FE0C2804460CDD224B25
:1048B00001221A700C23214A009303460021042090
:1048C000FBF740F903B0F0BDFDF7EEFC1C4B9A7905
:1048D0001C4B03EB420393F828303BB91A4A0221E0
:1048E000042003B0BDE8F040FBF72CB92B68A342CD
:1048F00019DB08350026154FA642E3DA3A68F1B213
:1049000055F8040BC2F30072FEF72CFB014688B980
:10491000094B052204201A7033460D4A03B0BDE846
:10492000F040FBF70FB9044A0321117000932346AE
:10493000084AC3E70136DFE794870120830E0708A2
:10494000888701208C830608AF0E0708040000202A
:10495000060F0708CD0E07082F4B2DE9F3411C78F1
:10496000064634B12D4B93F8884593F889350134C8
:10497000E41A2B4B1B783BB92A4A0221042002B0CF
:10498000BDE8F041FBF7DEB8102C0DDD264B02220E
:10499000002104201A701023244A00932346FBF7B9
:1049A000D1F802B0BDE8F081214FFEF7AFFD97F8D6
:1049B0002C1811F0FD0101D01E4ADEE77368A342F6
:1049C00020DB28360D46DFF87880A542E9DAD8F8F2
:1049D0000030E9B2B7F82628C3F300730093B7F8A4
:1049E000243856F8040BFEF7D7FB014688B90E4B66
:1049F000052204201A702B460F4A02B0BDE8F04190
:104A0000FBF7A0B8084A04201070009323460B4A15
:104A1000C5E70135D9E700BF84870120E0BA01204E
:104A2000868701202B0F070894870120450F070870
:104A3000E8A90120710F0708E30F0708AD0F070869
:104A400004000020014B00221A75704784160120D3
:104A5000014B01221A75704784160120044A054B48
:104A600092F8602003EB420393F82900704700BFDF
:104A7000E8A901208C8306081049114B91F86020A9
:104A800003EB420393F8293003B970470D4B10B480
:104A90001C7884B100234FF0010C51F833203AB157
:104AA00012792AB1984204BF01EBC30282F806C012
:104AB00001339C42F1D15DF8044B7047E8A9012015
:104AC0008C8306081810002010B5154C82B0D4F85D
:104AD0009C25D4F8A035D4F8941502FB03F38DF887
:104AE00007008B421AD0D4F890350DF10701D4F8A5
:104AF0009805184451F04AFED4F89035D4F89C2516
:104B0000D4F894151344D4F8A025B3FBF1F0013286
:104B100001FB1033C4F8A025C4F8903502B010BDD5
:104B2000E0BA01200B4B0022012003F2A45110B483
:104B30000824C3F88C25C3F89C05C3F89445C3F832
:104B400098155DF8044BC3F89025C3F8A025C3F869
:104B5000B0257047E0BA01200F4B93F86030062B68
:104B600017D8DFE803F00416070A0D1013004FF4FE
:104B7000C87070474FF4FA607047084B98887047C8
:104B80004FF47A6070474FF4FA5070474FF47A5000
:104B900070474FF47A707047E8A901208887012098
:104BA000034B53F8300010B103685B681879704705
:104BB000E8A90120034BD3F8302812B10F2800D800
:104BC00010477047E8A90120130A07B58DF8043093
:104BD00002238DF8052001AAFCF7D6F8024B1870C5
:104BE00003B05DF804FB00BF8416012050B101380A
:104BF000002330F0FF019AB203F1010303D140EA30
:104C0000022080B270474008F3E710B50C4601213E
:104C1000FDF7A2FBC0F300132370C0F3C003A37021
:104C2000C0F380036370C0F38013C0F3C010E3705F
:104C3000207110BD2DE9F0478846502114460646E4
:104C4000FDF78AFB01304621304F40004FF47A795E
:104C50004FF4FA6AC0B220803046FDF77DFB23781E
:104C6000013051217B4380B203F5FA73A080B3FB7E
:104C7000F9F2B3FBFAF300FB02333046B3FBF9F36E
:104C8000E360FDF79FFEC0F30F22C3B225783046E4
:104C900003FA02F27D43013293B205F5FA72B2FBD8
:104CA000F9F1B2FBFAF203FB01227021E380B2FBBF
:104CB000F9F22282FDF750FB013071214000C0B2B1
:104CC00060803046FDF77EFE98F80320C3B2C0F343
:104CD0000F20834001339BB2238112B1E2889B1ADB
:104CE0002381A3784FF47A724FF4FA6520897B43CD
:104CF00003F5FA73B3FBF2F1B3FBF5F300FB0133F9
:104D0000B3FBF2F36382BDE8F08700BF002F3A00E7
:104D10002DE9F0474FF4FA730026834F8CB0044618
:104D200089210068C7F8C43087F8C860FDF714FB14
:104D300040F001008921DFF8F481C2B22068FDF75C
:104D400019FB324688212068FDF714FB01228021DF
:104D50002068FDF70FFB0122FF212068FDF70AFB09
:104D6000324631462068FDF705FB91212068FDF7AA
:104D7000F3FA3146012287F8D9042068FDF7FAFAE0
:104D80003246FF212068FDF7F5FA3246802120687F
:104D9000FDF7F0FA60212068FDF7DEFA40F012001E
:104DA0006021C2B22068FDF7E5FA20224421206884
:104DB000FFF70AFFFF2201212068FDF7DBFA2568D3
:104DC000012280212846FDF7D5FA0122FF2128463D
:104DD000FDF7D0FA324631462846FDF7CBFA0622D7
:104DE000FF212846FDF7C6FA83212846FDF7B4FACD
:104DF00040F004008321C2B22846FDF7BBFA072227
:104E0000FF212846FDF7B6FA012281212846FDF749
:104E1000B1FA012280212846FDF7ACFA6B229421D9
:104E20002846FDF7A7FA324683212846FDF7A2FA65
:104E3000D8F80060C7F8C06083212846FDF78CFAD7
:104E4000002800F05583012228468321DFF8E08006
:104E5000FDF790FA92212846FDF77EFA0022C0F372
:104E6000C716814681212846FDF784FA0622284686
:104E7000FF21FDF77FFA8321284609F07F09FDF71E
:104E80006BFA832100F0FB022846FDF773FA2846EF
:104E90000122FF21FDF76EFA284601220021FDF7CD
:104EA00069FA28460022FF21FDF764FA284600220D
:104EB0008021FDF75FFA062305AAB02120680025AE
:104EC000FBF7A8FF0122FF2188F800002068FDF70A
:104ED00051FA00224F212068FDF74CFA2C224E2176
:104EE0002068FDF747FA0022FF212068FDF742FA0B
:104EF000B422B6212068FDF73DFA002E2A464FF075
:104F0000010C18BF0C260CAB5FFA85FEC5F3C4007C
:104F100005F007017645184410F81C3C0AD8914565
:104F200040F0F18206E000BFE8A90120E02E012058
:104F3000841601200CFA01F123EA010300F81C3C5D
:104F40000135302DDFD1062305AAB0212068FBF7FB
:104F50001BFF0122FF2188F800002068FDF70AFAF4
:104F6000002220681146FDF705FA0022FF21206883
:104F7000FDF700FA002209212068FDF7FBF9002265
:104F800010212068FDF7F6F9002211212068FDF7B5
:104F9000F1F9012224212068FDF7ECF9FF222521F7
:104FA0002068FDF7E7F9002275212068FDF7E2F996
:104FB0000122FF212068FDF7DDF92C224E21206817
:104FC000FDF7D8F9002248212068FDF7D3F92946DA
:104FD00020222068FDF7CEF90022FF212068FDF78E
:104FE000C9F9294609222068FDF7C4F90022542195
:104FF0002068FDF7BFF9042231212068FDF7BAF9D6
:10500000032232212068FDF7B5F983224021206870
:10501000FDF7B0F9252246212068FDF7ABF9002203
:1050200060212068FDF7A6F9002227212068FDF7FE
:10503000A1F9062250212068FDF79CF90022512198
:105040002068FDF797F9962252212068FDF792F922
:10505000082256212068FDF78DF92A46572120683D
:10506000FDF788F9002261212068FDF783F900220D
:1050700062212068FDF77EF9002264212068FDF797
:1050800079F9002265212068FDF774F9A0226621D4
:105090002068FDF76FF90122FF212068FDF76AF90A
:1050A000322222212068FDF765F914224721206869
:1050B000FDF760F9FF2249212068FDF75BF9002226
:1050C0004A212068FDF756F90022FF212068FDF7EC
:1050D00051F90A227A212068FDF74CF900227B2140
:1050E0002068FDF747F9212278212068FDF742F971
:1050F0000122FF212068FDF73DF934222321206899
:10510000FDF738F9002242212068FDF733F9FF222C
:1051100044212068FDF72EF9262245212068FDF75D
:1051200029F9052246212068FDF724F9402220684C
:105130001146FDF71FF906220E212068FDF71AF926
:105140001A2220212068FDF715F94022432120680A
:10515000FDF710F90022FF212068FDF70BF903226B
:1051600034212068FDF706F9442235212068FDF737
:1051700001F90122FF212068FDF7FCF8042231210A
:105180002068FDF7F7F809224B212068FDF7F2F8B7
:1051900005224C212068FDF7EDF804224D212068FE
:1051A000FDF7E8F80022FF212068FDF7E3F8002270
:1051B00044212068FDF7DEF8202245212068FDF714
:1051C000D9F8082247212068FDF7D4F82822482181
:1051D0002068FDF7CFF8002267212068FDF7CAF8A4
:1051E000042270212068FDF7C5F801227121206892
:1051F000FDF7C0F8FE2272212068FDF7BBF80022FF
:1052000076212068FDF7B6F8002277212068FDF7A7
:10521000B1F80122FF212068FDF7ACF801220D2131
:105220002068FDF7A7F80022FF212068FDF7A2F80B
:10523000012280212068FDF79DF8F82201212068D5
:10524000FDF798F80122FF212068FDF793F801226D
:105250008E212068FDF78EF8012200212068FDF7DD
:1052600089F80022FF212068FDF784F800228021C0
:105270002068FDF77FF804220A212068FDF77AF8FC
:10528000256884212846FDF767F8842100F0EF02A5
:105290002846FDF76FF801220B212068FDF76AF818
:1052A000206803A90190FFF7B0FC07AA03A90198A1
:1052B000FFF7C0FC9DF80C30002B00F02A810A9DFE
:1052C00005F684559DF80E30002B00F025810A9BD1
:1052D00003F2B22305EB43059DF80F3023B1BDF86F
:1052E0002C3003F525731D449DF8103023B1BDF813
:1052F0002E3003F226231D44DFF83482E8220121F8
:105300002068C8F8B455FDF735F844F61F639D4290
:1053100003D92946206849F0E2FE0122206811469F
:10532000FDF728F840212068FDF72CF8002800F050
:10533000E780012120680222FDF71CF80021206887
:10534000FDF720F8002800F0DB80E822012120682A
:105350004FF47A7AFDF70EF8202244212068FFF7F7
:1053600033FC256803A948F20E662846DFF8C4918D
:10537000FFF74BFC07AA03A92846FFF75BFC502266
:1053800057212846FCF7F6FF082256212846FCF74D
:10539000F1FF082250212846FCF7ECFFBDF82C0055
:1053A0000AFB0060B0FBF9F080B2FFF71FFC51214F
:1053B00002462846FFF708FC0A9A5C4B46210AFB86
:1053C000026628469E429BBFB6FBF9F202F1FF320D
:1053D000FF22D2B2FCF7CEFFD8F8B41544F61F6313
:1053E000994202D9284649F07AFE01212846FCF765
:1053F000B3FF0222064601212846FCF7BBFF00212D
:105400002846FCF7BFFF324601212846FCF7B2FFD1
:10541000246803A92046FFF7F8FB07AA03A9204642
:10542000FFF708FC482220461146FCF7A3FF08229C
:1054300047212046FCF79EFF032232212046FCF73D
:1054400099FF072230212046FCF794FF0122FF211B
:105450002046FCF78FFF202230212046FCF78AFFF0
:105460000022FF212046FCF785FF062220467021FE
:10547000FCF780FFBDF82E304FF47A7246F64400F8
:1054800002FB03004DF28803B0FBF3F09DF80F30F0
:1054900080B21BB1BDF82230184480B2FFF7A6FBE2
:1054A000712102462046FFF78FFBD8F8B41544F669
:1054B0001F63994202D9204649F011FE012120467E
:1054C000FCF74AFF0222054601212046FCF752FF65
:1054D00000212046FCF756FF2A4601212046FCF712
:1054E00049FF6423C7F8C430012387F8C83007E0B8
:1054F000D8F800309BB29B1BB3F5FA7F7FF69CACCB
:105500000CB0BDE8F0870B41DB0744BF0132D2B2DB
:1055100016E540F63635D5E69DF80D30002B3FF404
:10552000DBAE0A9B03F525731D44D5E61B280D0150
:10553000E0BA01201C0C010010B500230A4C84F8CD
:105540003438130A84F83518FF2184F836380423D8
:1055500084F8372804F63402FBF716FC00280CBF49
:105560006FF00C00002010BDE8A901202DE9F341E7
:105570000023744D06460468DFF8D4812D2785F892
:10558000CA30B9B2013718F8012B2046FDF7DAFF0F
:10559000882FF6D1402287212046FDF7D3FF002334
:1055A0008DF806300DF10601204649F078FD9DF892
:1055B0000630002BF6D0012286212046FDF7C2FFDF
:1055C000002287212046FDF7BDFF09220821204641
:1055D000FDF7B8FF00220B212046FDF7B3FF00289E
:1055E00051D137680DF106025E213846FDF7C2FF42
:1055F000BDF80630B3F5D77F00F09F8053D8512B0C
:1056000000F0998047D81D2B6AD01E2B00F09380A4
:105610002121306849F0B2FC34680DF10602DE2128
:105620002046FDF7A7FFBDF8063028229FED467AF9
:10563000C3F30903FF212046ADF80630534300228F
:1056400007EE903A85F834286C22F8EEE77A85F870
:10565000352867EE877AFCEEE77A17EE903A1A0E55
:1056600085F8393885F836281A0C85F837281A0A4B
:10567000062385F83828354AFBF786FB4022872128
:105680003068FDF75FFFB0FA80F0400985F8CA0086
:1056900002B0BDE8F081AD2B4FD0D62B01D0602BEE
:1056A000B6D121241DE040F2E132934247D00CD81C
:1056B00040F2D922934242D040F2E122934202D0FA
:1056C000B3F5E67FA4D164240BE040F28F4293420D
:1056D00003D040F2915293429AD14FF4FA7400E011
:1056E0000F24002894D10A224B213846FDF72AFFC7
:1056F0000F2260213846FDF725FF0D226321384631
:10570000FDF720FFB82269213846FDF71BFF40F660
:105710000D7278213846FFF70FFF40F60E627A21AE
:105720003846FFF709FF00287FF472AF214638465C
:1057300049F024FC6CE71424D3E73224D1E7C824D1
:10574000CFE700BFE8A901209A99893F1CB2012048
:10575000C283060838B50B0A15460D4A044682F87E
:105760003438022382F8351802F63402FF21FBF7A1
:105770000BFB10B96FF00C0038BD01232A46FF2146
:105780002046FBF747FB0028F4D00020F4E700BFD9
:10579000E8A9012003681B68184703685B6818477D
:1057A00003689B6818470368DB6970B506460C46BA
:1057B000154683B1BDE8704018473046FFF7F0FF4B
:1057C0000028FAD014F8011B3046FFF7E3FF2B1B2B
:1057D000002BF2DC70BD0D44F9E7E4E70368DB68F9
:1057E000184708B51F4B204CD3F8B855A0681CF0DB
:1057F000F7F928461CF0F4F9A06841798B0704D426
:10580000036841F002019B69984700210846FEF7B2
:105810003DF800210120FEF739F8A068FFF7BDFF31
:1058200070B101210020FEF731F8A068FFF7D6FF24
:1058300001462846FFF7AEFF00210846FEF726F88E
:105840002846FFF7AAFF0028E7D001210846FEF707
:105850001DF82846FFF7C2FF0146A068FFF79AFF30
:10586000D7E700BFE0BA0120F888012003681B6970
:10587000184703685B69184703689B6A03B11847B8
:1058800070470368DB6A03B1184770470D4B014648
:105890001B68DB0606D50C4B93F8BC3513F0040FE0
:1058A00018BF0021094B9B7A13B10846FCF73EBD97
:1058B000074B1868074B1B780BB981F00101FDF706
:1058C0005BBF00BF00000020E0BA01206488012017
:1058D0005C88012060880120BFF34F8F0549064B8B
:1058E000CA6802F4E0621343CB60BFF34F8F00BF7E
:1058F000FDE700BF00ED00E00400FA0508B572B650
:1059000000224FF0FF319300013203F16043082A77
:1059100003F56143C3F88010C3F88011F3D1FFF79A
:10592000DBFF012108B50846FEF794FEFFF7E6FF0E
:10593000EFF31183102282F312880B49DBB20A685D
:1059400001320A604FF0E02208499069C1F8CC05A5
:105950000020C1F8D005126983F31188044A136846
:1059600001331360704700BFE02E0120E0BA012030
:1059700040220120064B074A1B68516858434FF4E8
:105980007A73B0FBF3F053685B1A8342FBD970471C
:10599000D82A0120001000E010B5EFF31182102387
:1059A00083F312884FF0E0239C69196911F4803F5A
:1059B0000D4903D00120C1F8D0059C690B4BD2B230
:1059C0001868D1F8D03582F31188094A0344116868
:1059D0004FF47A7202FB01F0001BB0FBF1F00021E2
:1059E000E3FB020110BD00BFE0BA0120E02E012060
:1059F000D82A0120124B5B68C3F3080330B4EBB91B
:105A0000EFF31183D3B90F4B4FF0E0250E4819681F
:105A1000AC691A688A42FAD1D0F8CC15A142F6D303
:105A20000A4B19684FF47A7303FB01F0001BB0FBBB
:105A3000F1F0002130BCE2FB0301704730BCABE762
:105A400000ED00E0E02E0120E0BA0120D82A01207C
:105A5000F8B506460D46FFF7CDFF04460F46FFF7A3
:105A6000C9FF031B61EB0702B34272EB0503F6D3D8
:105A7000F8BD10B50446013C00D210BD4FF47A7059
:105A80000021FFF7E5FFF6E70023F7B5174F1A46A9
:105A900034210120FAF7A5FE0446386048B9144BBA
:105AA0001B780C2B03D1134B0122C3F8D4252546B8
:105AB00018E005269620FFF7DCFF0DF10702002114
:105AC0002046FBF7F7FC054660B9013EF2D1084BD2
:105AD00038681B780C2B02BF064B0222C3F8D42572
:105AE000FAF772FE284603B0F0BD00BF1094012003
:105AF000A8850120E0BA012008B50122092100682B
:105B0000FBF7CCFA6420BDE80840B2E706460B2557
:105B100080B5013D01D1FFF704FF0121771C4FF053
:105B2000320805240846FDF7B1FE00210846FDF7BE
:105B3000ADFE0120FDF79CFE0020FDF799FE01203F
:105B4000FFF7A4FE4046FFF794FF0120FDF790FE0B
:105B50000020FDF78DFE0020FFF798FE4046FFF77E
:105B600088FF7CB1013C05D14FF0FA084FF4FA7080
:105B7000FFF77FFF54EA0703DBD14FF47A70FFF79A
:105B800078FFC6E7013FF5E718B103685B6803B12A
:105B90001847FF20704718B103689B6803B1184786
:105BA0000020704770B450B106798E4207D3457912
:105BB000954204D30368DB680BB170BC184770BC16
:105BC000704710B440B184798C4205D303681B69D7
:105BD00013B15DF8044B18475DF8044B704718B1DA
:105BE00003685B6903B11847704718B103681B6A03
:105BF00003B118470020704730B568B1041D0A464C
:105C000000F114032068083454F8041C15469C4223
:105C100003C52A46F6D1012030BD10B50C4670B937
:105C20002D23002023750A4B2061C4E9063330235D
:105C3000C4E90000C4E9020084F8203010BD036804
:105C4000DB6A002BECD098470028E9D0F6E700BFCC
:105C50000615070838B5441E044D14F8011F01B994
:105C600038BDD5F83809FAF79FFDF6E7E8A9012015
:105C700013B50D4C01900D480091FFF7EBFF0C4957
:105C8000D4F83809DDE9003247F0C8FAD4F8380909
:105C9000FAF77EFD074B93F8F42512B1012283F841
:105CA000F52502B010BD00BFE8A9012008100708C3
:105CB0008D360108E0BA012008B504460748FFF711
:105CC000C9FF074BD3F83809FAF762FD054BD3F843
:105CD000B8051BF085FF20460BF060FC1410070888
:105CE000E8A90120E0BA0120034808B5FFF7B2FF98
:105CF0000120FFF7E1FF00BF201007087FB5174B19
:105D00001A78012A27D15B790A2B04D0144807B0EE
:105D10005DF804EB9EE71122002101A850F080FFFE
:105D2000A623152168468DF8003041238DF8021016
:105D30008DF80130EB238DF803300A4B5B7D8DF835
:105D40000430B2238DF8053003238DF8063020F09F
:105D5000F0FE0548DBE707B05DF804FB9C8D0120F1
:105D600039100708841601204810070810B50446AA
:105D70000948FFF76FFF05F0F7FE05F000FA074B43
:105D800000220749204683F8F525FDF7CFFC08B926
:105D9000FFF792FF10BD00BF62100708E0BA0120B4
:105DA000821B0708054808B5FFF754FF044BB3F8FA
:105DB000F60510B1BDE808405BE608BD375E070890
:105DC000E0BA012010B5074C02460B460649D4F84C
:105DD000380947F023FAD4F83809FAF7D9FCBDE8B6
:105DE0001040DFE7E8A901208D3601080FB407B5A0
:105DF00004A951F8040B0191FFF73AFFFFF7D2FF16
:105E000003B05DF804EB04B0704770B583791646B3
:105E10008EB0044603F00F02062A52D8DFE802F0E3
:105E20000415181A1D1F4B000D7813F0C0034AD03B
:105E3000402B3ED12946204611F01EFD00285ED0A1
:105E40000EB0BDE87040FDF723BC91F90050ECE7BF
:105E50000D88EAE7B1F90050E7E70D68E5E791ED55
:105E6000000A03A8FAF7F2F901462A48FDF710FCE8
:105E7000FEB1A37913F0C00F1BD1204611F04BFCEB
:105E800000EE100A03A8B8EEC00AFAF7DFF90146DF
:105E90002148FDF7FDFB204611F04EFC00EE100AF4
:105EA00003A8B8EE400AFAF7D1F901461A48FDF7FF
:105EB000EFFB0EB070BD17480EB0BDE87040FDF7A7
:105EC000E7BB0025B1E7042A29460CBF1348144854
:105ED000FDF7DEFB002EECD0A37913F0C00FE8D164
:105EE000204611F018FC0190204611F025FC019984
:105EF00002460C480EB0BDE87040FDF7C9BB03A9CF
:105F0000204611F02BFB03AA29460748FFF76EFF36
:105F1000CFE700BF2A1207080E160708C8140708A3
:105F2000E7520708DC6507087810070813B5044630
:105F3000019111F0E3FB019A0146204602B0BDE851
:105F4000104062E7004851E7951007082DE9F04F2F
:105F500087B00346FCF7A4FA064618B107B0BDE8BF
:105F6000F04FEFE705AA47491846344650F0EDFDDB
:105F7000B04605464FF0FF37DFF83091DFF830A12B
:105F8000DFF830B18DB97EB230461BF0D9FA10B1CE
:105F90004568002D5BD1B8F1000F36D139463A483B
:105FA000F9F7A0FD07B0BDE8F08F012E0ED0022E4C
:105FB00011D01EB92846FAF7A3FA074605AA3149B7
:105FC0000020013650F0C1FD0546DBE72846FAF710
:105FD00097FA8046F2E74946284650F05CFF20B920
:105FE0002A49284650F057FF08B144F001045146B1
:105FF000284650F050FF28B95946284650F04BFF2C
:106000000028DBD044F00204D8E7002C4FF0000356
:10601000304608BF03241A4619460293E4B2CDE97C
:1060200000841BF06AFC054610B939461848B7E7EA
:10603000424639461748F9F755FD39461648F9F7EB
:1060400051FD164B2946D3F8B80545F0C5FF394632
:106050001348F9F747FD5CB16979A14208D022469F
:106060001048F9F73FFD2B68E1B228469B69984735
:10607000EB6A002BE1D00C48F9F734FD0023EB620A
:10608000DBE700BFA30C0708A410070803410708BB
:10609000CC100708EB10070856110708E0BA0120DA
:1060A000081107082011070840110708361F0708C4
:1060B000A1100708A42507082DE9F3474FF0000AAF
:1060C0004FF0FF35DFF8D09001AA57465446D0462E
:1060D0002E46314950F039FD68B9BAF1040F50D05D
:1060E0003ADCBAF1020F13DC2B4632462B49012071
:1060F00046F054F80EE0BAF1040F09D8DFE80AF0D0
:10610000030D12171C00FAF7FBF9064603281BD9EA
:10611000FFF718FF02B0BDE8F087FAF7F1F905467E
:106120008F28F4E7FAF7ECF980463F28EFE7FAF713
:10613000E7F904463F28EAE70378482B03D0562BBB
:10614000E6D1012700E0002701AA494600200AF114
:10615000010A50F0FAFCBFE7BAF1050FD8D1A4014B
:1061600008F03F08902304F47C6403FB06550C4EB2
:1061700044EA080406EB450544EA4734A5F8F84527
:10618000C8E7902303FB0652054B03EB4203B3F829
:10619000F875C7F34037E2E7A30C0708D8C0012021
:1061A000E0BA012013460A46014601481EE600BF38
:1061B000841107082DE9F04F85B00546FCF770F90A
:1061C000044630B10021012005B0BDE8F04F45F094
:1061D0005DBF6FF0004287492846F9F72DFE20B9D0
:1061E00005B0BDE8F04F38F011BE6FF000428249B3
:1061F0002846F9F721FE28B9012005B0BDE8F04F87
:1062000038F06CBF6FF000427C492846F9F714FE65
:10621000034680BB7A4A82F8F00D104692F9F71DCA
:1062200092F8A254012D08D0033D052D05D9002C6C
:1062300000F0D18080F8F71DCDE092F8A35401332F
:10624000A52D13D101290ED16E4A80F8F13D00230E
:1062500080F8F01D82F8783A80F8F73D05B0BDE887
:10626000F04F38F085BF0139012449B2782B02F193
:106270001402D5D1DBE72846FAF742F9614B834691
:1062800093F9783A03FA80F60093772E00F2A7800C
:106290002846FDF717FA0746002800F08980FAF72C
:1062A0002FF90124C5B23846FDF70CFA074600283D
:1062B00000F081800134FAF723F90190E4B2384606
:1062C000FDF700FA8046002877D00134FAF718F974
:1062D0000746E4B24046FDF7F5F9814600286ED046
:1062E0000134FAF70DF90290E4B24846FDF7EAF9F5
:1062F0008246002865D00134FAF702F90FFA80F9D6
:10630000E4B25046FDF7DEF9824600285BD0013446
:10631000FAF7F6F80FFA80F8E4B25046FDF7D2F932
:10632000002852D00390FAF7EBF803990FFA80FA9D
:106330000846FDF7C7F90346002857D004F0FD04CE
:10634000FAF7DEF8042C46D1C3B2012D02D9E91EBA
:10635000052940D81BB1A52B01D0482B3BD1284C97
:106360000EB984F8F76D1421019AA52B01FB06469E
:10637000C6F89024029A86F8A254C6F89474C6F817
:106380009824A6F89C94A6F89E84A6F8A0A486F863
:10639000A3340AD100981B4B0130584483F8780A83
:1063A00094F8F73D013384F8F73D05B0BDE8F08F70
:1063B0000446054677E7019081E707468AE70290A1
:1063C00093E781469DE78046A7E75FFA88F3824618
:1063D0008046062CB9D005B0BDE8F04FB2E5772273
:1063E0002146094805B0BDE8F04FDBE60134E4B2D0
:1063F000EFE700BFA1110708A7110708551D0708FF
:1064000050990120E0BA0120AC11070810B50D4CDD
:1064100094F8F43573B194F8F5355BB10A48FFF799
:10642000E5FC0A48FFF7E2FC002384F8F43584F821
:10643000F53510BD0648FFF70DFC04F0A0FE002066
:10644000FFF73AFCE0BA0120B5110708EC11070884
:106450000A1207082DE9F04F01F020038FB08146A2
:106460000F464C4C4FF0000800934B4BD3F83809C3
:10647000FAF78EF994F806B00BF030034B454BD188
:10648000204611F0E5F8FAF7DFF80646204611F04D
:1064900001F9D6F808A005460AEB0006204611F0DF
:1064A0002DF90BF00F02062A6BD8DFE802F0043F4B
:1064B00044484D515D001AF805200078111A4A42EF
:1064C0004A41009B03B13ABB03A92046019211F057
:1064D00045F87B0615D5019A9AB903A92F48FDF70F
:1064E000D7F82F4903A849F083FF00284BD11AF8A9
:1064F0000530202B47D131462A48FDF7C9F8FFF770
:1065000051FC03A92848FDF7C3F800223146204674
:10651000FFF77BFCFFF746FC08F1010840F2472338
:106520000B349845A1D10FB0BDE8F08F1AF90520C2
:1065300090F90000C2E73AF805200088BEE73AF972
:106540000520B0F90000B9E75AF805200068B5E762
:1065500096ED007AD0ED007AB4EE677AF1EE10FA9B
:106560000CBF01220022ACE70190204611F0E4F8B4
:106570000199421C304650F057FCB0FA80F25209A3
:106580009FE700229DE7002231462046FFF73DFCB1
:10659000B5E700BF9F8C0608E8A901201112070883
:1065A000AE6507081C12070812120708F8B50C4C54
:1065B0002F250C4E0C4F2068FFF74CFB616811B182
:1065C0003046FDF765F8A16811B13846FDF760F86F
:1065D000FFF7E8FB013D04F11004ECD1F8BD00BF6A
:1065E00020840608211207082712070808B5FFF7BC
:1065F00031FBBDE80840FFF7D5BB10B504460348A2
:10660000FFF728FB2046BDE81040EFE72D120708F2
:1066100010B528F0E7FD134CD0B11348FFF7EDFF9C
:106620001248FFF717FBD4F83809FAF7B1F84FF41E
:106630007A70FFF71EFA0E4BD3F8B8051BF0D0FAAC
:1066400013F000F902210120FEF704F8FFF756F9D4
:106650000848FFF7FFFAD4F83809BDE81040FAF708
:1066600097B800BFE8A901203212070814100708E4
:10667000E0BA01205212070808B5FBF709FD83684C
:106680001BB90948BDE80840B0E70848FFF7AEFF6E
:1066900028F04EFDFBF7F2FC08B10548F2E7642054
:1066A000FFF7E7F9F6E700BF811207089512070820
:1066B000A012070808B50A480024FFF797FF094B06
:1066C000D3F83809FAF764F8074B83F8794AC3F826
:1066D000BC4A83F8C04A12F03BFF2046FFF7ECFAB1
:1066E000A6120708E8A90120E0BA012010B505228A
:1066F0001849044650F076FB60B9174B93F8F4251F
:1067000022B9012183F8F52583F8F4151348BDE873
:1067100010406BE703221249204650F063FB98B902
:106720000D4C94F8F4355BB194F8F53543B10D4850
:10673000FFF75CFB002384F8F43584F8F53510BDD1
:106740000948FFF753FFF5E70848BDE81040FFF799
:106750004DBB00BF4A1B0708E0BA0120D012070852
:10676000761D0708B5110708E6120708FA12070890
:1067700010B504460648FFF76DFA2046FFF76AFA9F
:10678000044B93F8F42512B1012283F8F52510BDCE
:1067900008100708E0BA01200CB4830607B500D53D
:1067A00051B905A904980191FFF70CFB012003B032
:1067B0005DF804EB02B070470020F8E7024B014699
:1067C000D3F83809F9F7F0BFE8A901200CB407B5F0
:1067D00010F0400009D069B92320FFF7EFFF05A9A9
:1067E00004980191FFF7EEFA012003B05DF804EB85
:1067F00002B070470020F8E72DE9F04F074687B058
:1068000016460C4615464FF0000B4FF019094FF491
:106810006178DFF8A4A0002E4BD02378287883423B
:10682000EB7844D161786A78914240D1A178AA7816
:1068300091423CD1E178CA1A51425141CDE9041349
:1068400010F004FA059B0499524619FB0383039345
:10685000AB7819FB038302936B7801934379384635
:1068600000935B46FFF7B2FF04992078043504914A
:1068700010F0ECF9E37852460499043419FB0383D1
:10688000039314F8023C19FB0383029314F8033CAE
:1068900001934379384600935B460BF1010BFFF7F8
:1068A0007BFFBBF1280FB6D107B0BDE8F08F002108
:1068B000C4E73146D9E700BF09130708F7B5064614
:1068C000FBF7EEFD054630B100222549012003B05B
:1068D000BDE8F04090E73046F9F712FE272804465D
:1068E00036DC8700701C8DF80750FCF7EBFE1C4D62
:1068F000064668B1F9F704FE002809DBC0B210F0C3
:10690000B7F928B1037905F8243001238DF8073051
:106910003046FCF7D7FE064650B1F9F7F1FD0D28D9
:1069200006D8EB1958709DF8073001338DF8073001
:10693000B91C0DF1070230462944FCF7CFFE9DF843
:106940000730042B02D0002345F8243003B0F0BDFB
:1069500027222946034803B0BDE8F04022E400BFE7
:10696000BC8D0120EE1307082DE9F04F804689B059
:106970000C46154602F1540B334EDFF8D4900692C4
:1069800094F9041000230C2202FB03F02F4FC05790
:10699000884254D00133072BF6D10C350C345D45B9
:1069A000EED109B0BDE8F08F95F904302A6899421C
:1069B000687995F806C095F808E095F807A03CD1ED
:1069C0002168914239D16179814236D1A1796145FD
:1069D00033D1217A714530D1E179A1EB0A077942AF
:1069E000794156F82A7056F82000049756F82E7010
:1069F0000791039756F82C70CDE9002002974A467C
:106A00004046FFF7E3FE0799E279404694F90430E7
:106A100056F822200492227A56F822200392A27974
:106A200056F822200292627956F8222001922268BA
:106A300000924A46FFF7B0FEAFE70021D1E7069B80
:106A4000002BB1D11946DFE708820608B485012082
:106A50001C130708F0B585B00346FBF721FD30B1E4
:106A600000224349012005B0BDE8F0407CE718460C
:106A70005E1CF9F745FD044640B21AF0EBFE0546F0
:106A800030B921463B4805B0BDE8F040FFF7AEB94C
:106A9000006801AB696803C3A86818603046FCF75A
:106AA00011FE0446002853D003782B2B05D02D2B44
:106AB00043D0F9F725FD019009E001342046F9F7AC
:106AC0001FFD0122019B02FA00F0034301930226FD
:106AD00000272046FCF7F6FD044638B3F9F710FD11
:106AE000254A0023114652F804EB5FFA83FC7045F7
:106AF00004D00133112BF6D14FF0000C51F82C309B
:106B0000984213D1102200216046F8F7C1F9022FF4
:106B100020D0032F21D0012F14BF8DF809008DF84C
:106B20000A0001370136042FF6B2D2D1012E17D850
:106B300005B0BDE8F040FFF705BA01342046F9F78B
:106B4000DFFC0122019B02FA00F023EA0003BDE70B
:106B50000126BDE78DF80C00E3E78DF80B00E0E7B8
:106B600001AB03CB286018686960A86005B0F0BD70
:106B70005891012039130708088206082DE9F04FC3
:106B8000804689B017460C46154600264FF0190A74
:106B90004FF46179DFF8B4B0002F54D06979A87848
:106BA0000791A1782B7881426A7895F803C095F80F
:106BB00004E0069345D12178994242D1617891420F
:106BC0003FD1E17861453CD12179714539D10799AF
:106BD00063795B1A59425941069B1AFB029206914E
:106BE0001AFB039303925A46CDE90103079B4046E3
:106BF00000933346CDE904CEFFF7E8FD06992379EB
:106C00005A46404606340593063514F8033C04936F
:106C100014F8053C1AFB0393039314F8063C1AFB83
:106C20000393029314F8043C019314F8013C00937D
:106C300033460136FFF7B0FD142EADD109B0BDE8E3
:106C4000F08F0021C8E73946D9E700BF4C13070889
:106C50002DE9F3478246FBF723FC064630B10022BC
:106C60003B49012002B0BDE8F04787E75046F9F7FD
:106C700047FC1328054663DC364C06278DF8076071
:106C8000474304F6C1290AF10100FCF71BFD09EB9B
:106C90000708064648B1F9F733FC03289FBFE319FC
:106CA00083F8C60A01238DF807303046FCF70AFD49
:106CB000064668B1F9F724FC0D2809D8062303FB22
:106CC000054383F8C30A9DF8073001338DF8073078
:106CD0000DF1070241463046FCF700FDFCF7F2FCDF
:106CE000064668B1F9F70CFC3B2809D89DF8073037
:106CF0000622013302FB05428DF8073082F8C40AF0
:106D00003046FCF7DFFC68B1F9F7FAFB0D2809D82B
:106D10009DF807300622013302FB05448DF8073049
:106D200084F8C50A9DF80730062B06D0002349F8E1
:106D30000730A8F80430FFF705F902B0BDE8F08786
:106D400013223146044802B0BDE8F047FFF72ABAE3
:106D5000A1C50120E0BA0120EE1307082DE9F04F8C
:106D6000074690460C4615460026DFF80CA12DED8F
:106D7000088B97B094ED008AB5EE408AF1EE10FAD8
:106D800071D0D4ED019A94ED029AD4ED038AB8F152
:106D9000000F40D095ED000A95ED01BAB4EE408A9F
:106DA000D5ED02AA95ED03AAF1EE10FA60D1F4EE4A
:106DB0004B9AF1EE10FA5BD1B4EE6A9AF1EE10FA4A
:106DC00056D1F4EE4A8AF1EE10FA0CBF4FF00109E9
:106DD0004FF0000912A8F9F739FAB0EE4B0A8346D2
:106DE0000EA8F9F733FAB0EE6A0A05900AA8F9F787
:106DF0002DFAB0EE4A0A049006A8F9F727FA049A89
:106E0000059B49460390384602925246CDE900B3AD
:106E10003346FFF7DBFCB0EE480A12A8F9F716FA82
:106E2000B0EE690A81460EA8F9F710FAB0EE490AE9
:106E300083460AA8F9F70AFAB0EE680A049006A891
:106E4000F9F704FA049B0390524600213846CDF826
:106E5000009010341035CDE901B333460136FFF709
:106E60009BFC0C2E86D117B0BDEC088BBDE8F08FD3
:106E70004FF00009AEE700BF6A13070870B505467A
:106E8000FBF70EFB064628B100222D490120BDE884
:106E9000704063E705222B492846F8F7CDFF38B943
:106EA000274B0022013043F8102B0C28FAD170BD7B
:106EB0002846F9F725FB0B2804463AD82846FCF764
:106EC00001FC064648B3F9F72BFA1D4B012503EBED
:106ED000041383ED000A3046FCF7F4FB064638B194
:106EE000F9F71EFA164B013503EB041383ED010A83
:106EF0003046FCF7E7FB064638B1F9F711FA104BBC
:106F0000013503EB041383ED020A3046FCF7DAFB8C
:106F100028B9BDE87040FFF715B80546DBE7F9F77B
:106F2000FFF90748032D00EB041484ED030AABD0EE
:106F3000EFE731460B220448BDE87040FFF732B955
:106F40001CC60120A1110708EE1307082DE9F04324
:106F5000804685B00D46164602270024DFF858907B
:106F60003EB336F8242035F82430F05B93421ED12E
:106F7000EB5B191A4B424B4119462346CDE90020E1
:106F80004A4640460391FFF721FC0399EB5B4A46D2
:106F900040460437019335F82430009323460134EA
:106FA000FFF7FAFB042CDBD105B0BDE8F08300232A
:106FB000E2E73146EAE700BF7E130708F8B504466A
:106FC000FBF76EFA054628B100222B490120BDE8E7
:106FD000F840BBE76FF0004228492046F8F72CFF45
:106FE000A8B9274B4FF47A714FF4FA62A3F8FC1B4F
:106FF000A3F8FE2BA3F8001CA3F8022CA3F8041C92
:10700000A3F8062CA3F8081CA3F80A2CF8BD204608
:10701000F9F776FA0328074627D82046FCF752FBF3
:10702000044670B1F9F76CFA012506462046FCF7D4
:1070300049FB10B1F9F764FA2DB9BDE8F840FEF745
:1070400081BF0546F2E7A6F2EE2240F2DC539A42F7
:10705000F3D8A0F2EE229A42EFD8094B03EB870354
:10706000A3F8FC6BA3F8FE0BD0E7294603220548E2
:10707000BDE8F840FFF796B8DCC60120A11107086B
:10708000E0BA01208F1307082DE9F04F834691B035
:1070900091460C4615460026DFF8F0A004F11508CD
:1070A000042209A80BAF41464FF0D2FE00238DF811
:1070B0002830D4E90232082B72F1000155D21A4669
:1070C0002E493846F8F728FDB9F1000F54D02B7837
:1070D0000793079A237893424CD1D4E90202D5E969
:1070E00002139A4208BF884244D1227D2B7D9A42E6
:1070F00040D1042205F1150140464FF067FD0028FC
:1071000038D121692B69CB1A594259411C4B52463F
:107110005846059300230493B5F912300393B5F94B
:1071200010300293174B0193079B0791009333464E
:10713000FFF74CFB079909AB52465846203505939B
:10714000237D0493B4F912300393B4F91030CDE9E0
:10715000017314F8203B009333460136FFF71CFB04
:10716000082E9BD111B0BDE8F08F07493846F8F7DB
:10717000D3FCA9E70021C9E74946DCE7E752070845
:10718000E02A07084145070897130708A2130708D4
:107190002DE9F74F0446FBF783F9074630B100228B
:1071A0006E49012003B0BDE8F04F6DE76C496FF008
:1071B00000422046F8F740FE014638B94FF480728D
:1071C000664803B0BDE8F04F4FF02ABD2046F9F7FE
:1071D00097F9054683B2072B00F2B8802046FCF7EA
:1071E00071FA824600284CD0F9F78AF901240FFA87
:1071F00080F95046FCF766FA68B14FF00008411E6E
:1072000000F1100C464611F8013F13F0DF0F3BD19F
:1072100001270134E4B2FCF755FA824600284CD02D
:107220000134F9F76DF90FFA80FBE4B25046FCF730
:1072300049FA0346002842D001340190F9F760F979
:10724000019B0FFA80FAE4B21846FCF73BFA0346BA
:10725000002836D001340190F9F752F9019B42B26F
:10726000E4B218460192FCF72DFA019A034650B396
:107270000134E4B2032C28D803B0BDE8F04FFEF788
:1072800061BE04468146B4E76145C2D0A3F1300235
:10729000D2B2092A05D9A3F16102052A07D8573BC2
:1072A000DAB2360146EA187642EA0818ABE7A3F1EB
:1072B0004102052AADD8373BF2E78346B6E782465E
:1072C000C2E70246CDE7274BD4E71FFA89F102292E
:1072D000D2D80BF2262189B2B1F5E16FCCD80AF2EF
:1072E000262189B2B1F5E16FC6D8D4B2062CC3D835
:1072F0001846019349F086F80428BDD8002FBBD06A
:107300002DB2164A019B680102EB451102F800906C
:1073100002EB4512A1F810B0A1F812A015320C75BD
:10732000114DC1E90286591E033311F8010F445D66
:1073300004F00304022C08BF203802F8010B08787F
:1073400008B19942F1D103B0BDE8F08F0722394668
:10735000064803B0BDE8F04FFEF724BFC08A012005
:10736000A1110708E02A0708016B0708C3130708E3
:107370002DE9F047814686B090460D461746002617
:10738000DFF868A0B8F1000F2DD03B782A789A4238
:10739000D7E9010C25D16A68824222D1AC68A4EBFE
:1073A0000C02544254412146009352463346059400
:1073B000CDE9010C4846FFF709FA0599AB6852463A
:1073C00048460C3702936B68019315F80C3B009309
:1073D00033460136FFF7E0F9082ED3D106B0BDE8F9
:1073E000F0870024DFE74146E8E700BFD013070835
:1073F0002DE9F8430446FBF753F8054628B100226F
:107400002F490120BDE8F843B2E72E496FF0004252
:107410002046F8F711FD014628B960222848BDE84A
:10742000F8434FF0FDBB2046F9F76AF80646C3B2B1
:10743000072B06D9294607222348BDE8F843FEF763
:10744000B1BE2046FCF73EF9074630B3F9F758F8CD
:10745000051E4FF0010418BF01253846FCF732F92C
:107460000746E0B10134F9F74BF88046E4B23846FC
:10747000FCF728F90746A0B10134F9F741F8814635
:10748000E4B23846FCF71EF908B10134E4B2032C2B
:1074900009D0BDE8F843FEF755BD0446DDE7804658
:1074A000E5E78146EDE776B2084B0C2000FB063697
:1074B00086F80C5CC6F8108CC6F8149CBDE8F883FE
:1074C000ECC60120A1110708E5130708E0BA012066
:1074D0002DE9F04F91B007468846164600240DF17D
:1074E0002C0ADFF8789004EB8405514608EB05037D
:1074F00058F805001B79029002A88DF80C3044F072
:1075000015FD4EB373197059052204A91B790DF1AD
:10751000180B049002A88DF814304FF057FBB0FA06
:1075200080F5594604A86D0944F000FD23464A46FB
:1075300029463846CDF800B0FFF748F92346013414
:107540004A4629463846CDF800A0FFF725F9202CF9
:10755000C9D111B0BDE8F08F3546EFE7F413070845
:107560002DE9F04F89B00546FAF79AFF044630B18D
:1075700000226849012009B0BDE8F04FA8E728467D
:10758000F8F7BEFF1F28074600F3BB802846A24637
:10759000FCF798F85F4ABB0006462546A3460393CE
:1075A00007EB8703A046A146D118D4505A4B0C7163
:1075B00002930194029B05AA13F801CB964602930D
:1075C0000023304616F8011B19B18C4501D00A2B57
:1075D0000CD108AE8C4533444FF0000603F80C6C18
:1075E00008D009B0BDE8F04FFEF7ACBC01330EF88F
:1075F000011BE6E709F1FF33461C032B03D8DFE844
:1076000003F02E456E7705A8F8F77AFF019009F18F
:1076100001095FFA89F9B9F1050FCBD1039A05F099
:107620000F003E4B04F00F043A44019944EA081459
:1076300017469A1803F66C4340EA01104FEA2818DF
:1076400082F86DBC1F4482F86C0C82F86EACFC7042
:1076500087F8048009B0BDE8F04F29F0ADB905A85E
:10766000F8F74EFF0546D2E74E2B14D0452B14D029
:10767000532B14D0572B14D0552B14D0442B05D199
:107680000523012101FA03F348EA030812F8013B3C
:10769000002BE9D1BBE70023F3E70123F1E7022345
:1076A000EFE70323EDE70423EBE7DFF878C00023DF
:1076B00019461CF8013B834204D0072901F101035C
:1076C000F6D15946DFF860C000231CF801EB704585
:1076D0000AD1012000FA03F34AEA030A8B4612F8A2
:1076E000010B0028E1D192E70133072BEDD1F5E73B
:1076F00005A8F8F705FF10280446B4BF0446002487
:1077000085E71F222146064809B0BDE8F04FFEF785
:1077100049BD00BF4CC7012010870608E0BA012010
:10772000EE130708158706081D8706082DE9F047A0
:10773000814686B090460D4616460027DFF860A0C9
:10774000B8F1000F2AD033882A889A4224D16C8855
:107750007188621A54425441F27821464846059491
:107760000292B278CDE900323B465246FFF72EF83E
:107770000599EB785246484604360293AB7801935C
:1077800035F8043B00933B460137FFF705F8102F0F
:10779000D6D106B0BDE8F0870024DDE74146E8E732
:1077A000FE1307082DE9F8430546FAF779FE04466B
:1077B00028B1002225490120BDE8F843B6E7284654
:1077C000F8F79EFE0F28064630DC28362846FBF7E1
:1077D00079FF1F4F0546DFF884804FEA8609284667
:1077E000F8F78EFE37F8023B984226DC012C08EBB6
:1077F000090311D0022C12D0A3F86C0C28462C21BE
:107800004FF0DBFA054668B1013501230134A3B11D
:10781000032CE4D1BDE8F88383F86E0CEEE783F81F
:107820006F0CEBE7A21E53425341EFE721460F22B4
:107830000848BDE8F843FEF7B5BC074B002243F803
:107840002620BDE8F843FEF77DBB00BFECC7012052
:1078500024870608EE1307084CC70120E0BA012070
:107860002DE9F04F144685B00646894600274FF0B3
:10787000060B284A0BFB07F54FF00008E03519F816
:1078800005A0002C42D0635DAAEB030041424141B8
:107890003046CDE900833B460391FEF797FF0399FD
:1078A0001C4A3B4630460135CDE9008A08F1010803
:1078B000FEF772FF174AB8F1060FE0D10137062F25
:1078C000D8D14FF48275134FA5F5827819F805A029
:1078D000F4B1635D3046AAEB0302514251413A468E
:1078E000CDE9008306230391FEF770FF0399062379
:1078F0003A4630460135CDE9008AFEF74DFF40F2A9
:107900000D139D42E0D105B0BDE8F08F2146C8E7D8
:107910002146ECE7101407082DE9F043804687B0B4
:1079200017460C4615460026DFF88C90002F40D0F5
:10793000B5F90030B4F90010B5F902209942B5F953
:10794000040095F906C032D1B4F9021091422ED14B
:10795000B4F9041081422AD194F90610A1EB0C0E5F
:10796000DEF1000141EB0E010591CDE90032CDE9D8
:10797000020C33464A464046FEF728FF059994F923
:1079800006304A46404608350393B4F90430029362
:10799000B4F90230019334F9083B009333460136C1
:1079A000FEF7FAFE102EC1D107B0BDE8F08300212A
:1079B000DAE73946E3E700BF241407087FB5054638
:1079C000FAF76EFD00285BD000222E49012004B09A
:1079D000BDE87040A0E72D2B03D0A3F13002092AA7
:1079E00049D8042C04DD04B0BDE87040FEF7AABA03
:1079F0002846F8F785FD04AB621C03EB440424F829
:107A00000C0C15F8013F303B092BFAD914462B78A2
:107A1000002BE0D1052CE6D1BDF80430BDF904609F
:107A20000F2BE0D8BDF90610A1F5FA7292B2B2F5AB
:107A3000FA6FD8D8BDF90820A2F5FA7080B2B0F577
:107A4000FA6FD0D8BDF90A008142CCDC8242CADB91
:107A50009142C8DCBDF90C5005F17D04A4B2FA2CAA
:107A6000C1D8084B23F8361003EBC6035A80988020
:107A70009D7104B070BD202BB5D101352246C5E7FC
:107A80000446C4E7048701202DE9F04F80468FB0FB
:107A900017460C4615460026DFF8A8B0A3882068D4
:107AA000ADF82C302378B4F902900893637894F9F8
:107AB00005A0069323790A900793B9F1000F3AD0F5
:107AC000002F3DD02868BDF828100C9080B2AB88FC
:107AD00081422A78ADF8343095F801C0B5F902300A
:107AE00095F804E02AD14B4528D1BDF82C10BDF8FB
:107AF0003400081A41424141009240465A460991D9
:107B0000CDE901C3CDE903EA3346FEF75FFE0999EB
:107B1000079B5A464046CDF810A006340635CDE9FD
:107B20000293069B0193089B009333460136FEF7B0
:107B300033FE202EB2D10FB0BDE8F08F0021DBE77D
:107B40003946E5E739140708F0B589B0044648F02E
:107B500059FC10F0FF0205D12C49012009B0BDE805
:107B6000F04091E705222A492046F8F765F930B937
:107B70001521264809B0BDE8F04047F023BC204657
:107B800001AA244902AD4EF0E0FF00244FF0FF337C
:107B9000204E079378B1062C02D1FEF7D3F933E0DB
:107BA000F8F7AEFC01AA45F8040B31460020013479
:107BB0004EF0CBFFEEE7042CEFDD029E1F2EECD83B
:107BC000039D0F2DE9D8049C252CE6D8059800F5D7
:107BD0007A73B3F5FA6FE0D80699FF29DDD8079AD2
:107BE000531C402BD9D80C4B062707FB0633A3F8B0
:107BF0007C0D83F87A5D094883F87B4D83F87E1D00
:107C000083F87F2DFFF7A0FF09B0F0BD5AC801200F
:107C1000A1110708A30C0708E0BA0120E02A070811
:107C20002DE9F04F07469BB093460C4615460026BB
:107C3000DFF804A10E930E9B5A1C01D0B3426FD102
:107C4000A6460DF1400C94F8048094F81390BEE819
:107C50000F00ACE80F00DEF800300890CCF80030E0
:107C6000237B09920A93237C0B9394F911300C9394
:107C7000A37C0D93BBF1000F5CD0AE460DF1540C0C
:107C8000BEE80F00ACE80F00DEF80030149ACCF824
:107C9000003023F07F4322F07F420F9095F804E0FC
:107CA0009A42A86895F80CC0E97C41D1F0453FD1D3
:107CB000089B0F9A93423BD10A9B634538D1099B9D
:107CC000834235D1A9EB010359425941099B5246E0
:107CD0003846CDF81C9006930A9B0F910593089B9C
:107CE000CDE903830D9B02930C9B01930B9B0093A7
:107CF0003346FEF76BFD0F99099B52463846CDF887
:107D00001C9006930A9B0593089BCDE903830D9B6A
:107D100002930C9B01930B9B00933346FEF73CFDB3
:107D2000013614341435402E85D11BB0BDE8F08FD8
:107D30000021CBE75946DFE7501407082DE9F04151
:107D40008AB004460D4648F05DFB10F0FF0211D1E9
:107D50003F4991F8F40548B94FF0FF33024601F668
:107D60003C6101200AB0BDE8F04159E76B1C6CD0C2
:107D70002B46F4E7052237492046F8F75DF838B975
:107D80004FF47E7134480AB0BDE8F04147F01ABBA9
:107D9000204601AD0024314E6A4630494EF0D5FEF2
:107DA00078B1092C02D1FEF7CDF84EE0F8F7A8FB28
:107DB0006A4645F8040B3146002001344EF0C5FEFA
:107DC000EEE7092CEFD101993F29ECD8DDF808E066
:107DD000BEF1010FE7D8DDF80CC00CF10103402B18
:107DE000E1D8049F332FDED8059E072EDBD8069DF1
:107DF0001B4A05F5742303F510739342D3D8079CEF
:107E0000072CD0D8089800F5742303F5107393421B
:107E1000C9D8099AFF2AC6D80D4B4FF0140808FBA1
:107E2000013309B2C3F8440E83F84CEE0D4883F8D1
:107E30004DCE83F84E7E83F8406EC3F83C5E83F8E7
:107E4000484E83F84F2EFFF779FF0AB0BDE8F08166
:107E5000E0BA0120A11107081CC90120A30C0708E2
:107E600080841E00E02A07084FF0FF3166E72DE905
:107E7000F04F1646154687B007460C464FF0000BEC
:107E8000194AD4F80880D4E9009A56B3AB689845EB
:107E9000D5E9000123D1814521D1AAEB0103594243
:107EA00059415B463846CDF800800591CDE9019AED
:107EB000FEF78CFC05990C4A5B460BF1010B38462A
:107EC000CDF800800C340C35CDE9019AFEF764FC46
:107ED000BBF1080F044AD4D107B0BDE8F08F0021F0
:107EE000DFE73146E8E700BF7114070870B586B0D8
:107EF000044648F087FA10F0FF0205D1214901201D
:107F000006B0BDE87040B2E705221F492046F7F7EA
:107F100093FF38B940F2FF311A4806B0BDE870400F
:107F200047F050BA204602AD0024184E01AA174966
:107F30004EF00BFE78B1042C02D1FEF703F81FE0DF
:107F4000F8F7DEFA01AA45F8040B314600200134A7
:107F50004EF0FBFDEEE7042CEFD1029A072AECD895
:107F60000B4B0C210B4801FB0233039AC3F84C2244
:107F7000049AC3F84422059AC3F84822FFF7B6FFD3
:107F800006B070BD1CCE0120A1110708A30C070884
:107F9000D8CB0120E02A07082DE9F04F8046A1B098
:107FA00017460C4615460026DFF8F8B0A6460DF138
:107FB000480C94F80C9094F818A0BEE80F00ACE8B8
:107FC0000F0023680C9323790A93A3680B93238AE9
:107FD0000D93638A0E93A38A9EE807000F93E38AAA
:107FE0008CE807001093002F5AD0AE460DF1640CB8
:107FF000BEE80F00ACE80F002B7E9EE8070053455B
:108000008CE807004AD12B790A9A934246D12B6813
:108010000C9A9A4242D12B7B4B453FD1AB680B9ACD
:108020009A423BD1169A824238D117991E9BCB1A9D
:1080300059425941109B5A464046119108930F9B53
:1080400007930E9B06930D9B05930B9BCDE9039322
:108050000C9B02930A9BCDE900A33346FEF7B6FBC7
:108060001199109B5A4640461C3408931C350F9BAF
:1080700007930E9B06930D9B05930B9BCDE90393F2
:108080000C9B02930A9BCDE900A333460136FEF711
:1080900083FB042E8AD121B0BDE8F08F0021C9E70F
:1080A0003946DEE7821407082DE9F0438DB0044617
:1080B00048F0A8F910F0FF0205D13E4901200DB0AB
:1080C000BDE8F04368E705223B492046F7F7B4FED8
:1080D00038B94FF47E7137480DB0BDE8F04347F032
:1080E00071B9204602AD0024344E01AA33494EF046
:1080F0002CFD78B10A2C02D1FDF724FF57E0F8F7E8
:10810000FFF901AA45F8040B3146002001344EF076
:108110001CFDEEE70A2CEFD1DDF80880B8F1030F63
:10812000EAD8DDF80CE0BEF1010FE5D8DDF810C0AB
:10813000BCF1070FE0D8059F214B07F5742202F52B
:1081400010729A42D8D8069E072ED5D8079D05F5FD
:10815000742202F510729A42CED8089CB4F5004FF2
:10816000CAD20998B0F5004FC6D20A99B1F5004FAE
:10817000C2D20B9AB2F5004FBED2124B4FF01C097F
:1081800009FB0833A3F8B60283F8BCE20E4883F873
:10819000A8C2C3F8A47283F8B062C3F8AC52A3F8C3
:1081A000B442A3F8B812A3F8BA22FFF77DFF0DB0CE
:1081B000BDE8F0837CCE0120A1110708A30C0708BD
:1081C00080841E00D8CB0120E02A07080FB407B531
:1081D00004A951F8040B0191FDF7F4FD03B05DF81B
:1081E00004EB04B07047F7B58479054614F0C0037A
:1081F00003D0402B18D003B0F0BD04F00F040FF0F3
:108200009BFA062C05D10146164803B0BDE8F040A4
:10821000DCE7019028460FF07EFA019A01461248E9
:1082200003B0BDE8F040D1E70024104E104F0FF02E
:1082300013FB05460F48FDF70DFD2B79A34204D82B
:1082400003B0BDE8F040FDF7ADBD14B13046FDF719
:1082500001FD2B68384653F824100134FBF718FA57
:10826000EBE700BFA4140708B4140708DB140708E1
:108270000E160708CB1407082DE9F0478CB0074607
:1082800010F8013B202BFAD000251F4CDFF880802E
:108290002E46DFF88090DFF880A001A920460FF07D
:1082A0005DF9394601A84EF0F6FDE0B101A940465E
:1082B000FBF7EEF9494601A848F09AF8F8B92046CC
:1082C0000FF01CFA114B0146007820280CBF5046D5
:1082D0001846FBF7DDF90136FDF764FD2046FFF790
:1082E00082FFFDF75FFD013540F247230B349D42CD
:1082F000D3D10EB943F0B4FE0CB0BDE8F087002135
:108300002046FDF713FEE6E79F8C06082A120708B1
:1083100016120708AE6507081C1207082DE9F04F72
:108320002DED028B8DB0067805460130202EFAD057
:10833000284648F067F8044618B1012821D12A2EB2
:108340001FD18A4D0026DFF8408240F24727884837
:10835000FEF74CF9284601A90FF000F9013601A9F2
:108360004046FBF795F9284621460B35FDF7DEFD23
:10837000FDF718FDBE42EDD10DB0BDEC028BBDE89E
:10838000F08F3D2128464EF018FD002800F0E780D0
:108390000346984613F8012D202AFAD0A8EB0508C9
:1083A0000130074610F8013B202BFAD06F4E4FF0FA
:1083B00000095FFA88F840F2472B01A930460FF018
:1083C000CDF801A848F01EF801A9024682462846C9
:1083D000F7F732FD654B044640BBC24526D10B2260
:1083E00002FB09339B7903F00F08B8F1060F31D176
:1083F000384648F007F8844205461FD35D4901A876
:1084000047F0F6FF20B15C4901A847F0F1FFF0B951
:108410003B78222B1BD17B1913F8013C222B16D160
:10842000AA1E791C30460FF033FAA5E709F10109BD
:108430000B36D945C1D143F013FE9DE73B5DA3F157
:108440006102192A9CBF203B3B550134D0E72A46E4
:108450003946E7E713F0C0030AD0402B4DD0474818
:10846000FEF786F93046FFF7BEFEFDF79BFC83E77B
:108470003B78002BF3D0424938464EF0FCFC0446D2
:10848000384647F0BFFF8442E9D13846F7F748FF46
:108490003046B0EE408A0FF03EF907EE900AF8EE53
:1084A000E77AF4EEC87AF1EE10FAD8D830460FF039
:1084B00043F907EE900AF8EE677AF4EEC87AF1EE27
:1084C00010FACCDBB8F1050F0CD118EE104A30468B
:1084D0000FF014F9B8F1050F32D8DFE808F03030AA
:1084E0003A3A3C3EB8F1040F384603D1F7F7EEFFB5
:1084F0000446ECE7F8F704F8FAE7304625460FF0B3
:10850000ABF9A246814690F804B02346AB4500D9AA
:108510001BB1BAF1000FA2D0D9E7D9F800306FF043
:108520000042394653F82500F7F786FC002805BFBE
:108530002C46012300234FF0010A0135E6E70470C1
:1085400001A91048FBF7A4F800213046FDF7EEFC26
:1085500012E70480F4E70460F2E70460F0E72846DD
:108560000DB0BDEC028BBDE8F04F85E69F8C060890
:10857000DD140708AE650708EF1407081315070890
:10858000FA140708081507081612070870B586B010
:108590000346F9F785FF044638B100221949012046
:1085A00006B0BDE87040FFF75BB903AD164E02AAF6
:1085B000154918464EF0C9FA80B1032C03D1FDF7D6
:1085C000C1FC06B070BDF7F79BFF02AA45F8040B8B
:1085D0003146002001344EF0B8FAEDE7032CEED11D
:1085E000059BDDE903451A4601932946E0B228F0D0
:1085F00013FB0028E3D0019B2A4621460348FFF7DE
:10860000E5FDDEE74CC70120A30C0708101407089E
:1086100008B50346F9F744FF40B10C4B00220C4863
:10862000A3F8F625BDE80840FDF7E0BF1846F7F7C8
:1086300067FF014630B1054BA3F8F6050548BDE8D4
:108640000840C3E5BDE80840FDF77CBCE0BA012066
:1086500023150708391507082DE9F04385B0F9F708
:1086600017FD826804462AB9224805B0BDE8F043E8
:10867000FDF7BCBF838900250188019242881E4E08
:10868000DFF888801D4FDFF88890009242681C4810
:10869000FFF79CFD15B94046FDF7A8FF3B689D42DA
:1086A00015DA3378294601351648062B06F10606F9
:1086B00096BF09EB83030022D3F8A02336F8023CCF
:1086C000009336F8043CFFF781FD092DE2D102202A
:1086D000F9F7EAFC81884388CB1A616803FB011132
:1086E000039126F05BFE03990246074805B0BDE8FA
:1086F000F0436BE581120708148201204C820120AF
:1087000050150708A9150708B81507089E1507088A
:108710008C8306082DE9F843054647F073FE0446AE
:10872000D0B9304B0127304DDFF8C8802F481E6884
:10873000FDF790FA55F8041B51B10B7833B107FAE5
:1087400004F3334202D04046FAF7A2FF0134F1E7C6
:10875000BDE8F843FDF726BB024625492846F7F752
:108760006BFB78B9204C234D2348FDF773FA54F87E
:10877000041B0029ECD00B78002BF8D02846FAF720
:1087800087FFF4E72B780026DFF85C902D2B03BFE2
:10879000013504F1FF344FF001084FF0000859F89B
:1087A000047B1FB9BDE8F84343F05ABC2246394662
:1087B0002846F7F741FB90B90120B040B8F1000F0F
:1087C00009D0F7F737FF0D48FDF744FA39460C4852
:1087D000BDE8F843FAE4F7F723FF0A48F4E7013667
:1087E000DDE700BFEC81012048870608D5150708A2
:1087F00049220708725E0708DF150708EB1507080E
:108800000E160708F41507082DE9F84F344F0546F2
:1088100047F0F8FD0446BE68C8B9324D0127DFF8BD
:10882000D4803148FDF716FAE3B205EB8302D2F8A3
:10883000401441B107FA03F3334202D04046FAF73D
:1088400027FF0134F0E7BDE8F84FFDF7ABBA024669
:1088500026492846F7F7F0FA60B9254C254D2648F9
:10886000FDF7F8F954F8041B0029ECD02846FAF774
:108870000FFFF7E72B784FF00009DFF874B02D2BCE
:1088800003BF013504F1FF344FF0010A4FF0000A35
:108890005BF8048BB8F1000F03D1BDE8F84F43F04B
:1088A000DFBB224641462846F7F7C6FAA0B90123A6
:1088B00003FA09F3BAF1000F0AD026EA03030F48BE
:1088C000BB60FDF7C7F941460D48BDE8F84F7DE4B0
:1088D00033430C48BB60F4E709F10109D8E700BF56
:1088E000708801208C830608D515070849220708DF
:1088F000CC870608725E0708DF150708EB15070826
:108900000E160708F41507082DE9F0474E4E81466C
:1089100047F078FD0446376800BB4C4D4FF00C081B
:108920004B4E4C48FAF7B4FE08FB04F35B5D5A1E4D
:10893000012393403B4206D0204618F041FC0146FB
:108940003046FAF7A5FE0134182CEDD117B942488C
:10895000FDF780F9BDE8F047FDF724BA02463F492C
:108960004846F7F769FA054678B92C46384D3C4831
:10897000FDF770F92046013418F022FC0146284624
:10898000FAF786FE1A2CF5D1E4E799F800304FF09B
:1089900000082D2B03BF09F1010904F1FF344FF04A
:1089A000010A4FF0000A404618F00AFC224605462C
:1089B00001464846F7F740FA00283BD1BAF1000FCC
:1089C0001FD0B8F1180F0BD16FF07F4333602548EB
:1089D000FDF740F929462448BDE8F047FFF7F6BB0C
:1089E000B8F1190F01D17368F0E7204B0C2202FB9C
:1089F000083898F878345A1E012393401F43376093
:108A0000E5E7B8F1180F03D1C6F800A01848DFE772
:108A1000B8F1190F01D17760F8E7144B0C2202FB73
:108A2000083898F878345A1E0123934027EA030740
:108A30003760EBE708F10108B8F11A0FB3D1BDE8D0
:108A4000F04743F00DBB00BF64880120048806088E
:108A50000D160708FC15070806160708492207081F
:108A600012160708EB1507080E1607088C83060870
:108A7000F4150708F0B585B0044647F0C3FC042898
:108A80003DD1631E2546E11C13F8012FA2F16100C0
:108A9000192898BF203A8B421A70F5D1261D1A4F1B
:108AA00015F8011B384601914EF087F920B1019964
:108AB00028464EF082F920B105B0BDE8F040FDF740
:108AC00041BAB542ECD120461DF026FE0F48FDF715
:108AD000C1F80F4C0C4901231A5D04AD013311F8A4
:108AE000010B2A44052B02F8080CF5D1002302A93A
:108AF00008488DF80C30FFF769FB05B0F0BD002881
:108B0000E4D0FDF71FFAE1E73C8906081D160708C7
:108B10009C8D01202A120708F7B50346F9F7C0FC1F
:108B2000044620B103B0BDE8F040FDF70BBA26467D
:108B300025461E4F01AA1D4918464EF006F840B9B9
:108B40000B2D18D901460B221948FDF72BFB03B05A
:108B5000F0BD44B1012C0AD001AA394600200134ED
:108B60004DF0F3FFEBE7F7F7CBFC0546F4E7F7F73B
:108B7000C7FC0646F0E7022C0ED1A6F57A73B3F5D2
:108B80007A7F05D94FF4FA624FF47A710948DCE72D
:108B9000094B03EB45039E80074B2946074803EB2F
:108BA0004503B3F90420FFF711FBD0E7A30C070836
:108BB000EE130708EC2007081810002023160708FA
:108BC00070B50346F9F76CFCC0B11F4B9E690136C6
:108BD0003046344618F0F4FA0546E8B901341A2C48
:108BE000A8BF0024204618F0EBFA0546A0B9B4420D
:108BF000F4D11648BDE87040FDF7F8BC1846F7F709
:108C00007FFC044618F0DCFA054628B921461048D6
:108C1000BDE87040FFF7DABA0B4B9C6119F0A4FA7B
:108C20000C4821462A46FFF7D1FA192C9BBF0A4867
:108C30000C21002001FB0400BDE8704098BF90F8B3
:108C4000780419F0ADBA00BF841601203016070869
:108C5000441607085A1607088C83060810B5034601
:108C60000C4C1846F9F71CFC38B10B4B0B48197823
:108C7000BDE810400131FFF7A9BA1846F7F740FCEC
:108C80000138022804D8C0B203F03EF92346E8E7D1
:108C900010BD00BFE02A070881850120771607086C
:108CA000022810B50C4614D802F040FF0948FDF721
:108CB000A4FC094B094819780131FFF787FA2146CE
:108CC0001020FDF7C7FB21462020BDE81040FDF72E
:108CD000C1BB10BDD3210708818501209A16070862
:108CE00010B503460C4C1846F9F7DAFB38B10B4BBC
:108CF0000B485978BDE810400131FFF767BA1846B4
:108D0000F7F7FEFB0138022804D8C0B203F00BF9D4
:108D10002346E8E710BD00BFE02A0708818501204F
:108D20006F160708022810B50C4610D802F058FF3D
:108D30000748FDF762FC074B074859780131FFF7F8
:108D400045FA21463020BDE81040FDF783BB10BD39
:108D50008216070881850120921607082DE9F04F39
:108D6000B64BA1B0B64A00250293B64BB649019363
:108D7000B64BB7480093B74BFFF728FAB649B74848
:108D8000FFF724FAB64BB74819684FF47A73B64E1A
:108D9000B64CB74F04F5B969DFF80CA304F2E45BF5
:108DA000B1FBF3F1FFF712FA09A8F7F75DF9B6F98D
:108DB000142309A915A844F0B9FE15A9AD48FFF779
:108DC00005FA1EF015FDAC4B64221B78B0FBF2F1E6
:108DD00004EB830302FB110289B2A848D3F8B8352B
:108DE00092B20093A64B1B78FFF7F0F9A54B3968B8
:108DF000A548B1FBF3F1FAF74BFCA44BD3F8008084
:108E00000123AB4013EA080F0BD059F8253043B1CA
:108E10001AF805205BF8251053F822209C48FAF731
:108E200037FC0135072DEBD1964DFCF7BBFF994878
:108E3000FDF7DCFBF1F702FBB0FBF5F19648FFF71D
:108E4000C5F939689548B1FBF5F1FFF7BFF9F1F7BE
:108E50002FFBB0FBF5F19248FFF7B8F9F1F742FBB1
:108E6000B0FBF5F18F48FFF7B1F98F4B1B78002B62
:108E700014BF0123022304EB8303D3F80C160791DC
:108E80001FF066FC04EB8000D0F80C2606921FF061
:108E900075FC04EB8000D0F80C3605931FF096FCAF
:108EA00004EB8000D0F80C861FF0A2FC05461FF0F2
:108EB000EFFC07461FF0D4FC04EB8000079904EB9D
:108EC0008707D0F80C0604EB85050390D7F80C064D
:108ED0000290D5F80C06DDE90532CDE90080734833
:108EE000FFF774F9724B1B68DA0319D510F0F2FA28
:108EF0000546A8B10027DFF8108201466D48FFF74C
:108F000065F9F8B220F074FB39460137B0F9022058
:108F10004046FAF7BDFBFBB2AB42F2D3FCF742FF8F
:108F2000654B664A1D88664B6649ADB21B6866484C
:108F3000C3F50073DFF8D491DFF8D4819B00634F51
:108F4000FFF744F9624A634B294663480425D31A64
:108F5000624ADFF8C0B11288DFF8BCA1FFF736F92A
:108F60005F48FDF743FB59F8041B5E48FAF790FB96
:108F70005846FCF76FFE18F8011B002940F02981C4
:108F80005948FCF767FE5948FCF764FE57F8041B84
:108F9000002940F022815448FDF728FB013DE2D131
:108FA000534B5448998BFAF773FB01201DF0FAFFDD
:108FB000054658B107EE900ADFED4F6AF8EEE77A02
:108FC00086EEA77AFDEEC77A17EE905A03201DF0C1
:108FD000E9FF034658B107EE900ADFED476AF8EE65
:108FE000E77A86EEA77AFDEEC77A17EE903A002070
:108FF00005931DF0D7FF059B58B107EE900ADFEDF2
:109000003E6AF8EEE77A86EEA77AFDEEC77A17EEAB
:10901000900A2A46009039480127B6F81813384EAE
:10902000FFF7D4F83748FCF715FE3568DFF8EC8019
:1090300025F0004525F07F0572E000BF770D070899
:109040009B0D0708800D0708720C0708890D07089B
:10905000821A0708950D0708A71607089A1A070825
:10906000E02E0120C1160708D8CB01208C8306080A
:10907000BC010120DB160708A8930120EC160708A5
:10908000A993012040420F00111707080C0000208F
:1090900021170708291707083E1707085017070860
:1090A0006217070874170708F88901208617070850
:1090B00008000020D91707081C2701200000012004
:1090C00054790120001800000D180708487301208A
:1090D000008000080040000845180708E8810120CA
:1090E0007F1807089218070808160708B01807081D
:1090F00018100020BA18070800247449CA18070875
:109100000000002007190708FE170708A8890608AD
:109110007C8801209A180708A91807080E16070866
:10912000002D5ED1FCF73EFE33685B0114D50CA820
:109130000EF018FB80B90C9B40F2462215A9934211
:109140009BBF35480B25284605FB03000EF006FAA9
:1091500015A93248FCF74AFE3148FCF77BFD2BF09D
:10916000E3F900284FD0037B427B81682D48FAF752
:109170008FFA2D4DFCF716FE2C48FCF76BFD286886
:10918000FCF709FD002842D00CA92868FCF745FD32
:109190009DF844109DF85030139A2548FAF778FA54
:1091A000109911B12348FAF773FA0E9911B12248B8
:1091B000FAF76EFAFCF7F6FD204B1B7833B104EB9F
:1091C00083041F48D4F88C16FFF700F821B0BDE8DF
:1091D000F08F5046FAF75CFAD5E65046FEF7F6FFF8
:1091E000DCE695FAA5F3B3FA83F307FA03F2062B4C
:1091F00025EA020594DD04EB83034046D3F81016FC
:10920000FAF746FA8CE70F48FCF724FDB1E70E4861
:10921000FCF720FDCEE700BF9F8C06081E1907084B
:109220003219070838190708309301205119070827
:1092300057190708751907087E1907089487012030
:109240009A190708451907088D1907082DE9F04FE5
:10925000002544482DED028B2F46A8469FED428AFB
:1092600095B0FEF7B3FF08A9E8B21DF011FE9DF816
:109270002430002B53D0129C4CB107EE904AB8EE2C
:10928000E77AC8EE077AFDEEE77A17EE904ADDF846
:1092900030904FEAE47B0D9B4FF47A7209FB0BF19F
:1092A000A9FB040604FB031141F28833C0184FF0F8
:1092B000000341EB060147F0E7FE41F28833064622
:1092C0004FF47A72DDE910A161430AFB0B1BA4FB8A
:1092D0000A01C0184FF000034BEB010147F0D4FE28
:1092E0004FF47A720E9B042D29461CBF3F18B044E0
:1092F000B3FBF2F306930A2390FBF3F203FB120095
:10930000CDE9042096FBF3F203FB126617482346CF
:10931000CDE90226CDE9009A089AFEF757FF0135FC
:109320001A2DA0D108A81DF09FFD0A9A4FF47A7358
:1093300008990F48B2FBF3F30C9AFEF747FF0A2295
:109340000C4897FBF2F398FBF2F102FB137702FB58
:1093500011820097FEF73AFF15B0BDEC028BBDE815
:10936000F08F00BFB419070800247449FB190708DF
:10937000301A0708521A07081FB5094B094A029309
:10938000094B0A4901930A4B0A4800930A4BFEF71E
:109390001DFF0A490A4805B05DF804EBFEF716BF49
:1093A000770D07089B0D0708800D0708720C07084A
:1093B000890D0708801A0708950D0708A7160708E2
:1093C000981A0708F8B500240B4D0C4E0C4F0D48A9
:1093D000FEF7FCFE6CB93268C2F50072920022B151
:1093E00057F824100848FEF7F1FE0134212CF1D182
:1093F000F8BD55F82420F2E7588101205479012066
:10940000308A0608A11A0708B71A07082DE9F3479A
:109410001A4C00251A4E1B4FDFF870801A48FEF7D1
:10942000D5FEE2792046A379F8F78AFE06EB8202A0
:1094300094F808A006EB830300F14101D2F82897C5
:10944000A288D3F8A436B2FA82F2BAF1000F0DD096
:10945000C2F11F024046CDE900A9FEF7B7FE013573
:109460000C34402DDDD102B0BDE8F087C2F11F02FF
:109470003846CDF80090FEF7A9FEF0E750820120B3
:109480008C830608F11A0708C51A0708E11A0708AD
:109490002DE9F04F0D468DB0B8490446FAF746F96C
:1094A0000646002840F0C080B5492046FAF73EF94C
:1094B0000646002840F0BA80B2492046FAF736F94D
:1094C0000646002840F0B4802046AF49FAF72EF94E
:1094D0000028064612BF1024264601240DB144F090
:1094E0002004AA4DAA4F95F8009095F80180DFF866
:1094F00014A35745C0F09E8002F036FB484602F0A8
:1095000015FB404602F06CFBA2493046FAF70EF913
:1095100008B144F0400414F01103009300F0898274
:109520009D48FDF76AF80020FFF726FF9B48FDF7EE
:1095300064F89B48FDF75AF804F03003302B02D151
:109540009848FDF75AF8984E4FF0000A9748FDF7F3
:1095500054F89748FDF751F8D6EDC77A954A20465A
:10956000F5EE407ADFF8A092CB46F1EE10FA0CBF90
:1095700001210021FDF710F906F547718E4A2046BA
:10958000FDF7ECFB8D48FDF738F8B6F9DE138C4A91
:109590002046B1FA81F14909FDF7FEF806F5777129
:1095A000884A2046FEF770FA8748FDF726F8874A72
:1095B00087492046FEF7B0F98648FDF71EF8864A2F
:1095C00006F29C412046FDF7D3FE8448FDF715F8CE
:1095D000834B844A1E68844B1F6867EA0603019325
:1095E0005BF8043B002B32D01978D1B14FF0010861
:1095F00001992046029308FA0AF811EA080F14BFED
:1096000001210021FDF7E2F866EA0701754A2046CC
:1096100011EA080F029B14BF01210021FDF7BCF8DD
:10962000704A0AF1010ADBE7012457E7022455E7F3
:10963000042453E77B88C3F30B021B04D7E9011012
:1096400048BF02EB420214374DF0A0F851E79846AC
:10965000664A67EA0603019359F804BBBBF1000FA1
:1096600026D09BF8001001B34FF0010A0AFA08FA5D
:1096700017EA0A0F0BD066EA07015B46204611EA9B
:109680000A0F14BF01210021FDF7A0F8574A16EA7E
:109690000A0F0AD0019B204613EA0A0F5B4614BF4B
:1096A00001210021FDF778F8504A08F10108D3E7BD
:1096B0004F485E46FCF7A1FF4E4ADFF850A1D2F8B2
:1096C00000904D4ADFF848B1126889EA02086FEA53
:1096D000080801273046B740013618EA070F14BFC3
:1096E0000121002119EA0707039114BF52465A4687
:1096F000019217F065FD03990346019A02902046F6
:109700000191FDF763F8002F14BF5A465246029BA1
:1097100001992046FDF740F8182EDAD13748002687
:10972000FCF76BFF364BDFF8ECA09F68DFF8E880B2
:10973000DFF8E890F3B20AEB8302D2F840B4BBF151
:10974000000F6DD0012199405B4639400CD04A464C
:1097500000212046FDF720F85B464A4600212046BE
:109760000136FDF733F8E5E7424620460191FDF763
:1097700013F85B4642460199F1E700BF141B070846
:10978000D3210708821607081B1B070881850120C3
:109790003C8607081F1B07081B2507082C1B07080A
:1097A000441B0708501B0708D8CB012019220708C3
:1097B0008B1B07089E1B07081CC60120AD1B070852
:1097C000C01B07085AC80120CD1B070804870120C9
:1097D00028940120DD1B0708ECC601207B20070828
:1097E000C8970120E61B0708EC810120F21B07083F
:1097F000171F0708E895012064880120FD1B070852
:1098000010990120148B070848870608FF1A0708DB
:10981000091B07088C830608121C0708061C07088A
:109820008B48FCF7EAFE01238A481F46DFF8DCC2BA
:10983000DFF8DCE28DF820B08DF810B08DF821B0A3
:109840008DF811B08DF822B08DF812B08DF823B0DC
:109850008DF813B013F80C200CA910F8016B0DF162
:109860003008114401F8206C13F80E10884408F8F1
:10987000106C17B1561A774277410133052BE9D1A5
:10988000002608AB744A394620468DF81460FCF770
:109890009DFF04AB704A39462046FCF77DFF6F48B8
